:020000040800F2
:1000000000A00020A53B01080D3C0108D92B0108E8
:100010000D3C01080D3C01080D3C010800000000EA
:100020000000000000000000000000000D3C01087E
:100030000D3C0108000000000D3C01086FF20008B3
:100040000D3C01080D3C01080D3C01080D3C010868
:100050000D3C01080D3C010805AA000801AA000892
:100060000D3C01080D3C01080D3C01080D3C010848
:1000700071E800080D3C010873B800080D3C010848
:100080000D3C01080D3C01080D3C01080D3C010828
:100090000D3C01080D3C01080D3C0108FDA90008BC
:1000A000EDFD000829FE0008DDFD00084DFE0008FA
:1000B0001DFE00080DFE0008FDFD00080D3C0108B6
:1000C0000D3C01080D3C01080D3C01080D3C0108E8
:1000D0000D3C010871000108650001085900010884
:1000E0007DF200080D3C01080D3C01080D3C0108A3
:1000F0000D3C01080D3C01080D3C01080D3C0108B8
:100100000000000000000000000000000D3C01089D
:100110000D3C01080D3C01080D3C01080D3C010897
:100120000D3C01080D3C01080D3C01080D3C010887
:100130000D3C01080D3C010800000000000000001B
:100140000D3C01080D3C01080D3C010800000000B9
:10015000000000000000000000000000000000009F
:1001600000000000000000000D3C01080D3C0108EB
:100170000D3C01080000000000000000000000002D
:08018000000000000D3C010825
:100188002DE9F04F2DED028B6A4F6B4B3B60AFB002
:1001980000237B6010F095FD18B910F0B5FD07F04D
:1001A800E3FC07F09FFD654A654C137843F00103B3
:1001B8001370644B4FF47002C3F88820002309932E
:1001C8000A93236843F480332360236803F40033DD
:1001D8000A93099B013309930A9B1BB9099BB3F541
:1001E800A04FF2D1236813F4003318BF01230A93F8
:1001F8000A9B012B68D0534E534BF360636ABB6074
:10020800636ADFF874B1DFF87481DFF874A143F032
:1002180080736362636943F4FC032EAD6361032357
:100228008DF86A3041F6FF7325F8503D4FF0904045
:1002380029460EF00DFC4FF6FF7358462946ADF8D7
:1002480068300EF005FC414829460EF001FC404894
:1002580029460EF0FDFB3F4829460EF0F9FB2946DA
:100268003D480EF0F5FB28460CF0ACF81A9B3B4ACB
:10027800B3FBF2F33A4A3B4913603B4B00221A6046
:100288005A603A4B5960F02186F823109A60384E2C
:1002980007221A60B368CAF8003098E80300636957
:1002A80085E8030043F4802363610823CBF8183002
:1002B8001A981BA90EF0CCFBDAF8003013F0080FDF
:1002C800A8F10C0829D163E02A4B12221A6063684E
:1002D800636063686360636843F480636360636852
:1002E80023F47C136360636843F4E8136360236852
:1002F80043F0807323602268114B9001FBD55A6844
:1003080022F003025A605A6842F002025A60636897
:1003180003F00C03082BFAD16DE796F88E31012B08
:1003280036D8044B96F88F219B6813F0805900F05B
:10033800D3852DE000010020DB730008F433002092
:100348000010024000ED00E00005FA050008004832
:10035800000C0048001000480014004840420F00FC
:10036800882B00203F1901008C2B002010E000E0B2
:10037800E01100200020024000040048BC8401086D
:10038800E42F0020BD4B002283F88F2107F05CFE8C
:1003980064200EF05EFFBA4800214FF48C7215F00D
:1003A800C0FEE369B74843F00703E361A36943F478
:1003B800E123A361636943F4C023636100F5887492
:1003C800837B416890F80FE003F00702DB0801EB3C
:1003D80083039200196A4FF00F0C0EFA02FE0CFA12
:1003E80002F221EA02021A62196A10304EEA010288
:1003F800A0421A62E4D10022A349002353540132D7
:10040800112AF9D1A14AFF2199540133072BF9D1B7
:100418009F4BDAF800409F4A1A609F4800213C220F
:1004280015F07FFEC4F3801905234FF0000E9B4A98
:1004380099481EF802100C2202FB0EF21154B9F171
:10044800000F07D11E3901299FBFFF2103F1FF3398
:100458001154DBB20EF1010EBEF1050FE7D1904A3F
:1004680096F805B013708F4B8F4983F800B08F4B07
:100478007B62C0330B608E4B8E4A03EBCB03A10625
:100488005B7848BF0123936200238B4A40F2DC511A
:1004980022F813100133082BF7D113A800211C22CE
:1004A80015F03FFE14F4007A1DBF844B1995039391
:1004B800CDF80CA0BBF10E0F03D00BF0EF03082B07
:1004C80002D101238DF85E30022006F0DBFD18B161
:1004D8004088003018BF0120C4F340038DF8523023
:1004E800C4F340338DF84C30C4F3C03300F001003E
:1004F8008DF84F3014F400638DF851008DF8549046
:1005080007D096F8823103F1FF3EDEF1000343EB9A
:100518000E038DF85030C4F300438DF85530BB6A94
:10052800B6F84401ADF862001AF1000A18BF4FF09E
:10053800010A003318BF01238DF85730C4F3005364
:100548008DF85830B6F84631ADF85C30B6F852310F
:10055800ADF85A3004F00101C4F38043C4F3C0027B
:10056800E40448BF45488DF85330B6F8503144BFCD
:10057800B0F84C01ADF86200B3F5FA7FADF8603021
:1005880084BF0023ADF862304D4896F8D23187F821
:100598002C30002387F82D3043709DF85E308DF89D
:1005A8004D10002B8DF84E208DF856A00CBF00235F
:1005B800022301B902B1013308EB83084FF00009A7
:1005C800D8F81430A3F1020A203304933AF8023F12
:1005D8004FF6FF72934200F0B1819DF85110DAB2E4
:1005E8001B0ADEB279B12748364C00EB021041688D
:1005F800A14208D10189B1F5806F00F09B81B1F566
:10060800006F00F097819DF8541031B111011D4819
:1006180040582D49884200F08D819DF8551079B1D8
:100628001101184C6018645828498C4200F08281E6
:100638004168B1F1904F03D1817B082900F07A819C
:100648009DF8521051B10F4800EB02104168B1F10A
:10065800904F03D10189102900F06C819DF84F104B
:10066800B1B30848174C00EB02104168A1422FD1E2
:100678000189042900F05E812AE000BFE011002012
:10068800D82B00202CA701080C0100201D010020F8
:1006980094280020D01300209828002065AD010878
:1006A800B5110020280A00206C2D0020F011002030
:1006B800CCAA01080001002020110020B084010804
:1006C8002D0100200004004800040040002C0140D7
:1006D8009DF8501051B1BE4800EB02104168B1F1CD
:1006E800904F03D10189202900F02481199C7CB105
:1006F800B74F216807EB02177868884208D1398913
:10070800A088884200F01681E088884200F01281B3
:10071800022B02D19DF84C3003E0012B04D19DF847
:100728004D30002B00F006819DF85710A84B17019B
:1007380059B19DF85E1041B9A2F10E01012904D802
:10074800D959A448814208BF04269DF85810DC19DD
:1007580031B19DF85E1019B9043A032A40F2D280EB
:10076800012E49D1DFF878820693D919FF2291F832
:100778000DE088F8742088F875204868C8F8844027
:1007880001F108020989ADF868104FF0000B022149
:100798008DF86B1088F878B01AA98DF86AE0059280
:1007A80088F830B0C8F834B0C8F838B0C8F83CB0E9
:1007B800C8F870B088F876B088F877B00EF048F9C5
:1007C800069B059AD85991785A460BF095FA204617
:1007D800594632460FF08CFB7F4BC8F888307F4B68
:1007E800C8F88C30C8F890B0204608F1880108F1A4
:1007F8008C020FF0D3FB9DE0022E4BD15FFA89F3F8
:100808001C2101FB03FC764BCDF81CC003EB0C0B41
:1008180001238BF8783006936D4B8BF87990D919B2
:100828004FF0000891F80DE048688BF87A8001F1E4
:1008380008020989ADF868108BF882801AA9CBF8EC
:1008480084408DF86AE005928DF86B600EF000F92F
:100858005F4B059AD859917842460BF04DFA069BA2
:1008680020461A4641460FF043FB5D4BDDF81CC09D
:100878005C4ACBF8882003EB0C015B4ACBF88C2050
:100888008831CBF8908020460A1D0FF087FB09F1CC
:1008980001094FE0032E33D19DF85330504E534F8A
:1008A8003BB196F82E80204608214FF6FF720023B0
:1008B8001AE0BDF8602096F82E80BDF86230B2F5D7
:1008C800FA7F0BD94A49B1FBF2F22046082192B2CD
:1008D8000EF0E7F8474B47F828000AE04649B1FB15
:1008E800F2F22046012192B20EF0DBF8434B47F8B2
:1008F8002800C36096F82E30013386F82E3019E0B0
:10090800042E17D1364EBDF85A2096F82D703A4B62
:1009180093FBF2F22046BDF85C30012192B20EF052
:10092800C0F896F82D3006EB87070133C7F8580151
:1009380086F82D30049B9A457FF448AE284E304BFC
:1009480096F82D2086F878212E4A1778A7F11702F5
:100958000024022A1C709E461BD8736A2344D3EDD8
:10096800007AF5EE407AF1EE10FA03D1B36A002B63
:1009780050D126E0244A04EB020C0FCB8CE80F0080
:100988009EF8003010340133C02C8EF80030E4D1CA
:10099800ECE71E4B13F837808EF8008003EBC70393
:1009A800D3F80490B9F1000FE0D04445DEDA164AD6
:1009B800230103EB020C4B440FCB01348CE80F00EE
:1009C800F3E7134B1A6812F4805F984648D141E068
:1009D8002CA7010800400140B9E6000899E7000883
:1009E80000010020FDE7000891E60008A42B002084
:1009F80000127A00B9E7000840420F00A9E7000892
:100A0800D42B0020280A002064090020CCAA010861
:100A1800E42F00202B4B2C4A13F83700107003EBFF
:100A2800C7035C68002CCCD000238342C9DAC3EB2F
:100A3800C3016218DFF89C80D2F8009041F8089052
:100A480001EB080C9188ACF8041092798CF8062018
:100A58000133EAE707F0EF03082B1C4B20D121E014
:100A68009EF80020012AF5D9194B03EB0212103227
:100A780010339342EED053ED047AB6EE007A67EE67
:100A8800877A43ED047A53ED057A67EE877A43ED6A
:100A9800057A53ED037A67EE877A43ED037AE7E741
:100AA8000E2F08D11A7842F010021A70182F13D19D
:100AB8000EF052FE10E01A7822F010021A70192F68
:100AC800F5E700BF78930108F82C0020D81900201A
:100AD8006C090020F92C00200EF022FED8F8003016
:100AE800B14CB24F580358BFB14BB2485CBF01225A
:100AF8001A70B14A137843F0040313704FF400439B
:100B0800ADF8683063694FF0020943F400234FF0F1
:100B1800010B8DF86B9029468DF86AB063610DF072
:100B280097FFA64BA64A1A6000200EF0B1FBE369B6
:100B380043F48043E361236943F480432361636999
:100B480043F4802363617B6A23F470037B627B6ACE
:100B580043F4A0037B627B6A23F070637B627B6A49
:100B680043F0A0637B627B6A23F070437B627B6AFD
:100B780043F0A0437B627B6A23F470237B627B6A29
:100B880043F4A0237B624FF460431A938DF86C9072
:100B980003234FF00009384629464FF4805A8DF850
:100BA8006D3004938DF86E908DF86F900BF07CFD8E
:100BB800049B8DF86D3038462946CDF868A08DF82D
:100BC8006CB08DF86E908DF86F900BF06DFD236909
:100BD80043F480432361236923F480432361794BE1
:100BE8009A8822F480521204120C9A809A8892B23F
:100BF80042EA0A029A801A8802F4415242F4457283
:100C080042F003021A809A8822F470621204120CCD
:100C180042F4E0629A809A8B22F400621204120C69
:100C28009A8307221A821A8892B242F040021A80E6
:100C3800C7F818A0D8F8003003F41073B3F5107F84
:100C480000F09E80604B614F1F606369DFF85C9124
:100C580043F480236361E36943F40013E361236B86
:100C680023F010032363236B43F010032363D9F8A5
:100C7800203023F07063C9F82030D9F8203043F0D1
:100C88008063C9F82030D9F8203023F07043C9F8C0
:100C98002030D9F8203043F08043C9F820304FF095
:100CA80000084FF0020C4022484629464FF0030B3B
:100CB8008DF86CC0CDF818C01A928DF86E808DF83A
:100CC8006F808DF86DB00BF0EFFC80224846294606
:100CD8001A920BF0E9FC3A68DFF8089122F0010259
:100CE8003A6039683A4A0A403A603A4A3A613A6898
:100CF80042F001023A60C7F80880C7F80C80C7F8CC
:100D08000880BA6842F40042BA603A683A607A6881
:100D180022F0784222F400427A603A6842F00102F6
:100D28003A60D9F800502C4F05F400434FF0100AF0
:100D38000493524605F4006338464146059315F07E
:100D4800F0F94FF6FF72DDF818C00E9215F00205A3
:100D58008DF83DC08DF83E808DF83F808DF83CB011
:100D680042D02EA94FF0904041F880AD0BF09CFC8A
:100D7800012507233D7087F80180FB70BD7033E0C3
:100D880016490A784B4616481F561F2F02BFFF27E1
:100D98001F5402F1FF3203F10C0308BFD2B23C2BFF
:100DA800F1D10A704EE700BF00100240000400486D
:100DB800900E002000080048F4330020043400207E
:100DC80059EE000800380040EC10002000540040A4
:100DD800FFE0CF007A25E00000290020B5110020AF
:100DE80098280020E42F0020049B7BB12EA904231F
:100DF80041F8803D92480BF057FC0C233B710723C8
:100E0800FB7101237D711D44BB71EDB2059B83B15C
:100E18002EA9202341F8803D4FF090400BF044FC70
:100E280002233B730723FB7301237D731D44BB73AC
:100E3800EDB2E36A834823F4F873E362E36A43F4A8
:100E4800D873E362636943F0805343F0020363613C
:100E58000BF067F91AA80BF039F97B4B1A937B4B07
:100E68001B93012D4FF0000394BF1A4680221F9256
:100E78004FF48072734C20924FF4806221922022AA
:100E8800204622921AA94FF400521C931E932392D3
:100E98002493ADF874500BF026F9236843F001034E
:100EA80023606B4CA36823F04053A360A36843F00E
:100EB8008053A3600A200EF0CCF9A36823F0804386
:100EC800A360A368A360A36843F00043A360A2687B
:100ED8005F4B002A31DAFAE7531E092B3FF658AA6E
:100EE800D8F858002860294658460DF0B1FD4FF44F
:100EF8000063CBF818303C200EF0ABF996F88F3130
:100F08009945BFF63FAADFF838B108224FF40063CD
:100F1800CBF8182078200492ABF8283003930EF011
:100F28008DF9049A039BABF828207820CBF8183069
:100F38000EF084F909F10109E0E79A68454922F0C1
:100F480040529A609A6842F000529A608868424A11
:100F5800024042F468328A60D968404A0A4042F442
:100F68000052DA601A6B013D22F00F0215431D632F
:100F7800002101237A189078002800F084805C1CF6
:100F8800042B17F801E0D278DFF8C4C0E4B20ED819
:100F980003EB4303DCF830505B001F20984025EA40
:100FA80000000EFA03F30343CCF8303031E0092B8C
:100FB8000ED80620053B4343DCF834501F209840E8
:100FC80025EA00000EFA03F30343CCF8343020E09E
:100FD8000E2B4FF006050ED8A3F10A006843DCF883
:100FE80038801F23834028EA03050EFA00F32B43B9
:100FF800CCF838300DE00F3B05FB03F0DCF83C8003
:101008001F23834028EA03050EFA00F32B43CCF88C
:101018003C30BEF1090F0E4822D983698569AEF1CB
:101028000A0303EB43034FF0070E0EFA03FE25EA0B
:101038000E05856185699A402A43826122E000BFD6
:101048000004004808040240400100501029002014
:101058000001005000030050E010FCFF07C0FFFD36
:10106800436945690EF1FF3303EB43034FF0380E34
:101078000EFA03FE25EA0E054561456903339A40D9
:101088002A4342612346043110297FF473AFBC4BD5
:101098009A6842F001029A601A461168B84BC9076B
:1010A800FBD5DA68B74C22F00202DA60DA6842F05F
:1010B8000202DA60DA6842F00102DA609A6842F005
:1010C80004029A60B4F85831002B41F07E80B4F9DC
:1010D8005A21002A41F07980B4F95C21002A41F0B4
:1010E8007480D9F800309B031FD5C8200EF0B1F8E2
:1010F800AE200AF0F4F908B10AF0F6F9A24D86F824
:101108007901C8200EF0A5F8A04BC6F87C31002163
:101118000C22284615F005F80223EB700CF00DFFA1
:101128000EF070F89A4B0344AB609A4B9A481B68D0
:10113800B4F86081B3F85630049300210C2294F877
:101148005FB194F8675194F8687114F0EAFF934B13
:10115800069318460021142214F0E3FF904A0592E2
:10116800002111708F49C6F880110EF01EFE059AF5
:101178008246002838D0069B8B4919608B495960F4
:101188008B49D960B8F5807F8A4919618A4B01D1AA
:1011980000211CE0B8F1BB0F01D9012117E0B8F11B
:1011A800610F01D9022112E0B8F1290F01D90321F9
:1011B8000DE0B8F1130F01D9042108E0B8F1090FC7
:1011C80001D9052103E0B8F1000FE1D0062119701B
:1011D80004231370794B02221A70794A136843F07A
:1011E800010313605B460EE001200EF0ADF82FE21C
:1011F8004FF0010B0BFA03F140F2B2320A4042B150
:10120800012B5FD900236F490022092B0A70F9D8F6
:10121800EEE711F04D0FF3D0624A0593C6F880212E
:101228000EF0C3FD059B0028EAD0062168200A4677
:101238000DEB00030DF022FD9DF86D1001EA0B0285
:101248009DF86B1001EA0B0101FA0BF343EA8201E6
:101258009DF8692002EA0B030B430AD05BB25B4599
:1012680001D1002302E0022B0ED1012386F884313C
:1012780011E00EAB68200C215A460DF0FFFC9DF8DA
:10128800383013F00F0303D103200EF05DF802E0AD
:10129800042BEAD1E5E7404B4B4A1A604B4A5A60A7
:1012A80096F88421002A0CBF6F226E221A72454BD1
:1012B80004221A70414B03225A70414A136843F0C2
:1012C80002031360042F00F2D180DFE817F0050055
:1012D800EC009900050099000A200DF0BAFF77206C
:1012E800A02101220EAB0DF0C9FC002800F0888077
:1012F8001E21012277200DF03DFD4FF42F600DF0E7
:101308009DFF4FF0000BABF160010027C9B202222C
:101318001AAB77208DF868708DF869700DF0AEFC07
:101328009DF868209DF8693043EA0223284A02F5AF
:10133800C3712BF801300BF1020BBBF1100FE2D196
:10134800B2F8943103F00F0103F47F43A2F894310B
:1013580001203A4622F0010EB644BEF886E1BEF1FD
:10136800000F18BF002012F0010F06D05FFA8EFEA2
:1013780087EA0E074FF0080E2CE087EA1E27F9E7E8
:1013880000010050E0110020C4290020661300204D
:10139800404B4C0030110020683000205C1B0020BE
:1013A800DC070020D484010891FC000819FB000820
:1013B800A1FA000890C1793D0000002088000020B3
:1013C800D41900201C34002005FD00085BFB000830
:1013D8000001002017F4004F18BF87F4C057BEF172
:1013E800010E4FEA4707F5D10132102AB2D1654AFA
:1013F8000B43A2F8943118B9C7F30337B94238D070
:1014080096F896B15F4FBBF1000F40F0CD861420DF
:101418000DF01FFF07F297137620D02101220DF05F
:101428002DFC97F89731582B3DD107F5CC738821BF
:10143800182276200DF022FC31227620F4210DF0BE
:1014480099FC012387F896314F4B504A9A60504ACD
:101458005A6045F6D8125A804E4ADA604E4A1A61E6
:101468004E4AA3F800B05A6100F09EBE012F13D176
:1014780019E0454B42F210721A805A80484A5A6065
:10148800484A9A60484ADA60484A1A61484A5A61A2
:10149800BAF1000FB4D00327464B474A9F70136830
:1014A80043F004031360444F3B689A0702D5434B4B
:1014B8001B68984718F0FF0F0AD13B6813F0020F1A
:1014C8004FF07D0240F2712308BF4FF4FA7302E037
:1014D8004FF47A731A461344013B93FBF2F3013B32
:1014E800DBB203FB022286F8B431354B1A60354B68
:1014F8001B689847344A0023022D1370934604D082
:10150800032D20D0002D40F056862EAB002203F884
:10151800502D2E4AC6F8B8211E200A2101220DF0AE
:10152800ADFB80B19DF86830482B0CD1284B294A77
:101538001A60294A5A60BAF1000F04D004238BF8C4
:10154800003002234EE02EAB4FF0000803F8508D18
:101558000C20414601220DF091FB80B19DF86830C6
:10156800482B40F05A861A4B1C4A1A601C4A5A608B
:10157800D046BAF1000F00F05086032332E08046CF
:1015880000F04BBE00010020700600206DAC000882
:101598006FAC00083FAE0008E5AE00086FAA00086F
:1015A800C7FA000809FB0008BDFA0008F9FA0008A4
:1015B800E1F8000888000020D419002068300020D5
:1015C800903000205C1B00201D340020EC840108B2
:1015D8004C0600205DB0000849AE0008C5AF000801
:1015E80031AF0008BD4AD3703B6843F008033B6045
:1015F800BB4B93F854210AB1BA490A7093F85521A4
:101608000AB1B9490A7093F856310BB18BF800301A
:101618003B68B64913F0080F00F0C985BDF9100002
:10162800DFEDB36A642290FBF2F302FB130212B2FD
:1016380007EE902AB8EEE77A07EE903AF8EEE77AE6
:10164800E7EE267AB2EE047A67EE877AC1ED007A81
:10165800A84A137843F002031370A74B08229A6133
:101668000A25A54EB38A9BB283F00803B3821920DA
:101678000DF0EFFD01200DF00BFE19200DF0E9FD36
:10168800013D00200DF004FE15F0FF05E9D1082307
:101698009A4FB3613B681B0705D5994B1B68984760
:1016A800984B01221A70984B9FED988A1B68984DA9
:1016B8001B7B00EE103AB8EEC00A20EE080A06F0CE
:1016C80055F92B8807EE903AF8EEE77A27EE800A6C
:1016D80014F036FF8F4B9FED907A18802B888F4D32
:1016E80007EE903AF8EEE77A8D4BC7EE277A284650
:1016F800FF211B229FED8B7AC7EE877A9FED8A7AAE
:10170800C3ED007A894BD3ED047A894B67EE887A6A
:1017180067EE877AC3ED007A14F003FD0021297083
:101728003968844B012211F0020F18BF6A701A70D1
:101738001FBF03221A700222AA704E0748BF1A78E8
:10174800284641BF551C1D700325855411F00A0F0A
:101758000CD01A7804218154511CC9B2052545546E
:10176800D11C0232D2B2197006218154D9F8002056
:10177800950641BF19784D1C1D70072548BF455473
:10178800110608D51978092545548D1C0131C9B2AF
:101798001D700A254554524D6E79082E01D00E2E23
:1017A80008D1197801F1010E83F800E04FF00B0E13
:1017B80000F801E0197812F4803F4FF00C0C00F8A3
:1017C80001C001F1010E1CBFDFF868C102315FFAE8
:1017D8008EFE83F800E01FBF8CF800104F494FF0D1
:1017E8000E0C01F80EC0510741BF197801F1010E26
:1017F80083F800E04FF0100E48BF00F801E01978B8
:1018080001F1010E5FFA8EFE4FF0120C12F4806F98
:1018180083F800E000F801C00ED095F81CC2BCF1B6
:10182800000F09D0DFF80CC102318CF800103B49D9
:101838004FF0130C01F80EC0197812F4007F4FF026
:10184800140C00F801C001F1010E1CBFDFF8E4C060
:1018580002315FFA8EFE83F800E01FBF8CF800109B
:101868002E494FF0150C01F80EC0182E13D1197817
:101878004FF0160E00F801E001F1010E5FFA8EFE3E
:101888004FF0170C00F80EC001F1030E0231C9B277
:1018980083F800E04654110341BF19784E1C1E70AE
:1018A800192648BF4654D60541BF1A78511C1970ED
:1018B8001A2348BF8354002198221F4814F031FC92
:1018C8000AF0DFFA1D4B1E4A1A601E4BB4F84E117F
:1018D80019801D4900230B8038E000BF88000020D4
:1018E800E0110020DC0700201C340020782D0020A7
:1018F8008988883CF433002000040048D41900206B
:101908004C060020640600206808002035FA8E3C4A
:101918002C000020840800200AE81C41F91000204F
:101928009807002000401C46BD3786355C1B002008
:1019380064080020F8100020F0270020C40F0020C1
:1019480066130020C80F0020C43300208B7097490D
:101958000A60B4F8941188B2954A22F8130001334A
:10196800122BF9D1934E3368D8045CBFB5F89A01AD
:1019780010801B0740F1C68095F88E41062C00F2B6
:10198800BB80DFE804F004070E3D5878780045F284
:10199800F05201E042F6F822874B1A800AF00EFB5B
:1019A800A9E007EE901ADFED856A834BB8EEE77A77
:1019B800DFED837AE7EE267A42F6F8221A800023D2
:1019C800FCEEE77A7F4A17EE901A42F823100133AB
:1019D800122BF7D17C4A7D4911607D4A4020137053
:1019E80005F02AFC002800F0878001234FF0070942
:1019F80090F90000774A8DE808024021764B75E09F
:101A08006D4B42F6F8221A806F4B744A1A60704B7D
:101A1800102240201A7005F00FFC00286CD001231A
:101A28004FF0000890F900006D4A8DE80801402148
:101A38004FF4E1335AE0604B42F6F8221A80624BC9
:101A4800684A1A60624B082240201A7005F0F4FBBD
:101A5800002851D001234FF0000C90F90000624A91
:101A68008DE8081040214FF4E13305F0BBFA5F4BD5
:101A7800C3F8BC013CE0504B5D485E49DFF8A481E7
:101A8800DFF8A4C142F6F8221A80514B5A4A4FF0A7
:101A98000C0E83F800E0062C4FF0000303700B7067
:101AA80013700AD01B2388F80030544B8CF800E0E0
:101AB80005221A704FF4E13407E0212388F800303A
:101AC8004E4B8CF800E01C704D4C3F4B4D4A1A6051
:101AD800402005F0B1FB78B101234FF0000E4A4ACF
:101AE80090F9000040218DE80840234605F07AFA75
:101AF800003018BF012028B9082005F0FBFF324B41
:101B0800424A1A603368324A13F4804F1FBF0821D3
:101B180011702D493E4818BF086042F20101194072
:101B280003F0010003F4005481B1234944F6206E08
:101B3800A1F800E024B1082111702349354C0C604C
:101B480020B10C211170204933480860117818061B
:101B5800A1F10401517040F1A48024482F4CDFF812
:101B6800CC90C0F8C0914FF000084146152200F50E
:101B7800E270DFF8BCA084F80180C4F80480C4F8DF
:101B8800088014F0CEFAA9F105034046CAF80030DF
:101B980008F050FC224B02201B68E36005F04CFB68
:101BA800002847D1802005F0A5FF72E0B833002057
:101BB80020300020E42F0020D2080020CDCCCC3FDC
:101BC8000000B0C4C83200203C000020BD27010836
:101BD8008C28002065290108A0860100A927010892
:101BE800B9280108952701086D280108000100207F
:101BF800B4330020C9270020C8270020EC27002084
:101C080090D0030065BD000879BD00081D280108B3
:101C1800F12701080D280108FD270108B407002055
:101C280008300020EB270020B3330020D013002019
:101C3800D407002090F805E06378C8490C2202FB1D
:101C480003125278724504D00133DBB2042BF4D965
:101C580000236370DAF8003062781B7890F900008E
:101C6800002B4FF00C0303FB021314BF4FF0030EBD
:101C78004FF0010E00225B78CDF800E001920221BE
:101C880005F0B0F9B64B186000288BD0012008F099
:101C9800D1FBB44B1868B44B00F5C5721A6008F054
:101CA80077FC336813F4007F0DF1680857D0AF4C08
:101CB800039B2360AE4BAF485A6942F480225A61B5
:101CC8009A6942F001029A61039B1B88ADF8303093
:101CD8004FF0010902230CA98DF833308DF83290AA
:101CE8000CF0B6FE2368A3485B88ADF830304FF09F
:101CF800000A0CA98DF832A00CF0AAFE2368484609
:101D0800197A0AF087FA236858680AF0D3F9236821
:101D18005B681A93404610238DF86D308DF86CA0DF
:101D28008DF86E900FF0ACFC23685B7A8DF8383034
:101D38000EA803238DF839308DF83AA08DF83B9022
:101D48000FF080FC8C4B8D4A1B683C3B13603B6852
:101D580043F010033B608A4B4FF0FF321A60894A08
:101D6800894B1360894A8A4F803313603368002493
:101D7800D9033C7040F1B0800EF0ECF9DFF83CC2BA
:101D8800DFF8ECA1CDF814C040F22A334FF0010976
:101D98001A4660462146049387F8009014F0C1F96A
:101DA800DAF814207B4F4FF0904042F40032CAF822
:101DB8001420426A22F00F024262426A032142F072
:101DC800060242624FF4807B02228DF835100CA97E
:101DD8008DF8342003928DF83640CDF830B08DF868
:101DE80037900AF061FCDAF81810039A41F40061A0
:101DF800CAF81810398821F45C710904090C398073
:101E08001D21F96238463A850EA93C866022C7F83A
:101E180014900E92ADF83E401094ADF84440ADF8E1
:101E28004640ADF84840ADF84A40ADF83C900AF05D
:101E38008BFABA6942F00802BA617A6C42F400423D
:101E48007A64DAF8142042EA0902CAF81420AAF6D9
:101E5800E47A50460AF065F940460AF037F9049BDF
:101E68004D4AADF874308023DDF814C01A9241460B
:101E780010221F9350464FF40053CDF86CC01C92AB
:101E880023931E94CDF880B02194229424940AF0D0
:101E98002AF9FB6843F40073FB60DAF8003043F07A
:101EA8000203CAF800300BA80C238DF82C308DF8EB
:101EB8002D908DF82E408DF82F900FF0C3FB214602
:101EC800364B1A68364B43F8212001312029F7D1C7
:101ED8000CF0E0FC0CF0DEFC33685A0540F18B8016
:101EE800304C314BD4F80495C3F80090042005F029
:101EF800A3F90421C4F8080505F07AF92B4B84F8F6
:101F08000C050820C3F8009005F096F9284B294FD6
:101F18001860082105F06CF9002184F80D052C22C1
:101F2800384614F0FEF88E237B704FF07C0BE023CC
:101F38004FF07D0AFB7087F800B087F82BA01E4F82
:101F48002C220021384614F0ECF88A237B701020EC
:101F5800A023FB7087F800B032E000BF8885010835
:101F6800C02900203011002020100020B0070020D8
:101F7800001002400004004808300020AC07002090
:101F880050110020A01A00200C140020042A002060
:101F9800910E0020002C0140342C014004850108DA
:101FA800920E002000010020C8190020201A0020ED
:101FB8006C1A0020F0190020251A0020D9020020F0
:101FC80087F82BA0C4F8109505F036F91021C4F84D
:101FD800140505F00DF984F818052020C4F81C959F
:101FE80005F02AF92021C4F8200505F001F984F844
:101FF80024050BF079FE8D4A138823F040031B0457
:102008001B0C1380138823F038031B041B0C13804C
:1020180013889BB243F04003138000249F2332208F
:102028008DF838308DF839408DF83A408DF83B40BE
:102038000DF00FF98DF869407D4C4FF4805704225C
:10204800278540460EA90FF0C7FAA7619DF86A20B8
:102058009DF86930120242EA03429DF86B301A4338
:10206800744B9A42744B17D008D874498A420CD0E2
:1020780001F51A4102318A4209D01CE070498A42AE
:1020880005D001318A4207D015E0202200E08022E5
:102098001A804FF4807202E04FF480721A805A80DE
:1020A8009A88198812029A604A43DA60654A0121BF
:1020B80082F8251504E000221A805A809A60DA60B6
:1020C800DC6814B3E40AA1464FF0000AA24509DA15
:1020D8000AEB04077F10F8024146102209F0B0F914
:1020E8000F2807DC08F020FC564B4FEAC922C3F83A
:1020F80028250AE0002358F82320013261D1013352
:10210800042BF8D1B9463C46E0E733684E4A13F44D
:10211800002318BF012313700DF074F84B4B18609F
:102128006B79052B02BF4A4B4FF4C8721A80494B92
:102138004FF47A721A80484BC8221A80474A13789B
:1021480043F008031370464A137823F00203137010
:10215800326840F6020313406BB1424B42491960A2
:10216800424B03211970424B012119704149002348
:102178000B8041490B80930341BF404B04221A71E5
:10218800DA7844BF42F00102DA70AB6833603C4B46
:1021980001221A703B4A137863F07F0313702FB043
:1021A800BDEC028BBDE8F08F0427FFF775B900235B
:1021B8000B60FFF74DBA012D7FF61AAA1D46FFF7EF
:1021C80099B907F1010A27469DE71BB207EE903A35
:1021D800DFED2D6AB4F95A312C4AF8EEE77A07EEAA
:1021E800103A67EEA67AB4F95C31CDED1A7A07EEAB
:1021F800903AB8EEC77AF8EEE77A002127EE267A09
:1022080067EEA67A11701AA821498DED1B7ACDEDDB
:102218001C7A05F0B3FBFEF764BF012D7FF6E8A931
:1022280000258BF80080FFF770B900BF0038004028
:102238000004004818BA20001C00002015202000C7
:102248001740EF00000100208C300020A408002077
:10225800D60F00201634002014340020D81900208E
:102268001F340020C019002058130020241A002011
:1022780080000020C0100020C2100020C4290020C7
:10228800900E0020F433002035FA8E3C70000020B8
:10229800DC280020954A2DE9F04F1568944C05F587
:1022A8009C4320332DED028B2360924B196889B033
:1022B80011F4804F0592984605D110F019FC10B919
:1022C8002379013323718C4B1F78C7B18B4A12686D
:1022D800954240F2DF80013F1F70DBE0D9F8003003
:1022E8008748072D98BF595D864B88BF29461B68CC
:1022F8009847032D0BD904EB45050137E880804B3F
:10230800DFF81C921E78FDB2AE42E7D820E0D9F87B
:10231800002005F10E0302EB83039988DA88002870
:10232800E9D04FF47A73401A5843531A90FBF3F0EC
:1023380040F6C90300F57A70984205DC40F2EE23B6
:102348009842B8BF184601E040F6CA0080B2D2E70A
:102358000F23277984F82A3094F82B30019303252A
:1023680094F82C30B7FBF5F505EB45057D1B039379
:10237800D9F800300293DFF8B0A1EBB2049300253E
:10238800B54254DA6049019B31F815B04FEA450966
:1023980053B910F0ADFB28B1039B002B08BF4FF0D9
:1023A800000B01E0DDF804B0029B988A584502D87A
:1023B800D88A58450ED2E8B210F044FB032D834664
:1023C800DFBF94F82AE00120A8402EEA0000D8BF19
:1023D80084F82A0010F08CFB18B14C4829F800B09A
:1023E80021E0049B94F876002AF813B028B9022F4C
:1023F80015D93F49012081F87600BAF80210BAF8D9
:1024080000000844BAF804100844414980B229F889
:10241800010000B2032190FBF1F080B200E05846C1
:102428003A4929F8010001350AF1060AA8E794F8A3
:102438002A203848384BA2F10F014A424A4184F811
:1024480090206AB1354A1268520109D40268D968E5
:102458009A60521AC82A1DD9012283F8212019E04E
:1024680002689868DA605B68121A9A4288BF2A4B39
:102478004FF0000184F82B1088BF83F82110002545
:10248800B54207DAE8B210F0DDFA204B23F8150060
:102498000135F5E7D8F80030DF0405D51F4B1B6878
:1024A800DE0701D410F02AF9059B19681C4B18683F
:1024B800837A002B3AD0013B144D027B35F8133058
:1024C8001AB1C3F53B6308339BB21BB2A3F57A7309
:1024D800B3F57A7FA8BF4FF47A7323EAE37307EE64
:1024E800903A9FED107AF8EEE77A58E00034002031
:1024F800180F0020E42F0020C0330020BC33002038
:102508008C2800203C0000201E0F002020300020D6
:10251800900F002008300020C4330020F410002061
:10252800B833002000007A44460F0020D8F8002075
:10253800150440D5D4F89420934E8A1A002A3ADB21
:1025480001F59C422032C6F89420904AC07A557909
:102558008F4A32F8152096F89850013592B292FBBE
:10256800F0F205F00F0086F89800304480F89920C2
:102578001A468848185C01330244102B92B2F8D1ED
:1025880012B292FBF3F31BB2642BA8BF642323EAB5
:10259800E37307EE903A9FED807AF8EEE77AC7EE9C
:1025A800877A7E4A9FED7E7A67EE877AFCEEE77A35
:1025B80017EE903A1380D8F800307A4F13F4807FE2
:1025C80000F00981784BDFF8E491994205D999F830
:1025D800022012B9012289F8022099F80220002A63
:1025E80000F0F980714A3E7892F821506A1E5542EF
:1025F80055416F4A1168002DC1F38063C6F3800608
:102608000193924614BF4FF0000B4FF0030B99F85B
:102618002020052A00F2D980DFE802F0034D527528
:1026280084A1002E3AD0D4F8AC00B4F8B0100CF065
:10263800A4FD012809D15F495F4A09681268C98861
:10264800642000FB0122C9F81020019B6BB1594A94
:10265800126812794AB110F09DFA032289F82020F5
:102668004FF47A72C9F81C20D1E7002D40F0AD80F4
:10267800514AD9F8101010684C4A88420AD9029277
:1026880010F088FA029A032182F8201040F6B83137
:10269800D161BCE7012182F82010B8E7019B4FF413
:1026A800806013B105F016FA01E005F002FA002285
:1026B800C9F8102089E0002D46D110F06BFAA6E782
:1026C80025B1052289F82020012000E0284666B1BE
:1026D800D4F8AC20D189394A11805180918035498C
:1026E80009684988D1804FF0020B334A1168D9F83C
:1026F8001420914201D8002E64D147F23052C9F813
:102708001C20032221E03A7842F002023A700FF0CE
:10271800F5FF294AD9F81C1012680A44C9F818208C
:10272800042212E0244A9DB11168D9F81820914278
:102738004BD9234A12781AB9DAF80020D30744D4BF
:102748003A7822F002023A70052289F820205EE7E2
:102758001268D9F81C100A44C9F8182035E0154940
:10276800154A09681268C988642000FB0122C9F863
:1027780010204FF48060002289F8202089F8032077
:1027880005F097F943E700BF180F00200029002043
:1027980010290020B10F00200000C8425411002069
:1027A80000C07F441F340020404B4C00C43300203D
:1027B800F4100020F03300200830002020300020E2
:1027C8001800002000287FF422AFBBF1000F02D0D0
:1027D80058460CF07BFD934D05F5C370B5F84E11C6
:1027E8000CF0CBFC834668B910F0C6F98E4BC3F8E1
:1027F80000B0C3F804B0C3F808B08C4B00221A60CC
:102808005A609A603B785E0736D5D8F80030D8060B
:1028180032D5874B1B78D9062ED4864B1B7893B1BB
:1028280095F8DE31BBF1000F15D17BB1824B1A68E8
:10283800D4F8B4309B1A002B08DA0FF05FFF7F4BF7
:1028480083F8B8B018E0BBF1000F0DD110200CF0E0
:102858003DFD01230EE03BB1774A12684FF47A71CF
:1028680001FB0323C4F8B43094F8B83023B10CF05A
:1028780015FD002384F8B830002295F8DCA195F8FE
:10288800DD11B5F896E1B5F898C113466C4E01967E
:1028980036F912009B087045C4BF63F07F03DBB2B2
:1028A80001326045B8BF43F04003042AEED194F8E2
:1028B800B92062489A4205D190F8BA20F92A04D87A
:1028C800013200E0002280F8BA2084F8B930594B70
:1028D8005C4E1A789946E2B93368DA0708D5BBF135
:1028E800000F16D13B78DB0713D50FF061FD10E020
:1028F8003B7858070DD5514B93F82B304BB1524BC1
:10290800DB7833B911B10FF0F9FE02E0BBF1000F2B
:10291800F9D094F8BA30494ADFF840B1142B40F0A6
:10292800AF8099F800301AF1000A18BF4FF0010A79
:102938006BB392F8B9305F2B11D13B7803F00403E5
:1029480003F0FF0113B10FF0D9FE08E00B2003914B
:1029580002920CF0BBFC029A039982F8BA10BAF101
:10296800000F14D094F8B9307D2B10D13B7803F0C8
:10297800040303F0FF0213B10FF0C0FE07E00B20C1
:1029880002920CF0A3FC2D4B029A83F8BA203B78F4
:1029980003F0040303F0FF01002B71D194F8B93060
:1029A800264A572B16D1294B4FF47A721A80D8F839
:1029B8000030190601D507F04DFE254B1B685A0754
:1029C80042BF244A0A21118013F0080358D1224A31
:1029D800138055E0D8F80000400717D55A2B15D1B9
:1029E80092F8BB302BB1012382F8BB1082F8BC30BF
:1029F80046E092F8BD3083F0010382F8BD300BB198
:102A08000C2000E00D200CF061FC39E05D2B00F09B
:102A180019855B2B00F018855E2B21D1032000F06F
:102A280014BD00BFE0110020182B0020E01A002080
:102A3800D81900201800002008300020180F0020A6
:102A480020300020F4100020C43300201634002069
:102A5800D419002014340020D01100203011002097
:102A6800562B01D105F0F0FA99F80030002B00F050
:102A7800018594F8B9306F2B40F0F6840FF098FC7C
:102A8800D8F80030580736D594F8BD30B74A93B116
:102A98003B7859070FD5019BB3F90610B5F8963165
:102AA800994208DD336813F0010302BF3221A2F80E
:102AB800C01082F8BD303368DA030DD594F8C2200F
:102AC800AA4B2AB993F8BB2012B93222A3F8C02026
:102AD800012384F8C2300EE094F8BB30A34A53B106
:102AE8003B7803F0040303F0FF0123B9012382F8C4
:102AF800BB1082F8BC30DBF800A0002333600AF179
:102B08007B090AF1CB0B99F8002099F8013019F8E4
:102B1800010C9A420BD249460CF0F8FA38B119F870
:102B2800022C012303FA02F233681343336009F1DC
:102B38000409D945E7D18E4B1B7843B18D4B8E4E96
:102B48001A6812F0020F994640F038832FE30AF111
:102B5800CA060AF589793278737816F8010C9A4210
:102B680025D231460CF0D2FA08B3B37896F804E0CF
:102B7800824A96F803A07D480C21013B01FB0E41D7
:102B880003EB43031344D1F8C8209A420FD0C1F88D
:102B9800C830002390F8F420C1F8CC30012303FAA0
:102BA8000EF322EA030381F8C4A080F8F430063655
:102BB8004E45D0D1724B1E68724B1B68039394F834
:102BC8002B300493704B029300230193029B1B68E4
:102BD800002B00F0E18293F800A0BAF1000F00F09A
:102BE800DB82029A039952688A1A002A0CDB01F5E3
:102BF800FA7202994A60019901228A4094F8F41005
:102C080021EA020284F8F420049A002A00F0C4821F
:102C1800029A597812F8042C0432D2B2002940F0F2
:102C28007A825A4931F91210B5F8942102F1C80094
:102C3800814202DD93F802B015E0C83A914203DA06
:102C48009978C1F1000B0EE0019A0123934094F8A2
:102C5800F42022EA030384F8F430039B029A03F574
:102C6800FA73536098E294F8F430019A1341DB0741
:102C780000F19282BBF1000FCCBF022001200CF0C2
:102C88004BFB0AF1FF33DFF8E490132B00F27C8250
:102C9800DFE813F01400250037004B0064008400BF
:102CA800E7004A01B101DF010F027A024B005A0026
:102CB8008400E7004A01B9001C01810196F80090E0
:102CC800D944B9F1FA0FA8BF4FF0FA0929EAE9790E
:102CD800304686F800900CF0FFF901200FE096F8D6
:102CE8000190D944B9F1640FA8BF4FF0640929EAEB
:102CF800E979304686F801900CF0EEF90220494651
:102D0800D4E196F803A0DA44BAF1640FA8BF4FF0F3
:102D1800640A2AEAEA7A86F803A03046D9F8F81055
:102D280004F090FA03205146C0E1717959446429AE
:102D3800A8BF642121EAE17171710D200CF04EFAEF
:102D4800BAF10D0F00F02082317959446429A8BFE7
:102D5800642121EAE17131710E20A7E1B17959446A
:102D680081F30801B1710520A0E100BF180F002010
:102D780021340020F4100020D4190020DC8601083A
:102D88005811002008300020E00F002020300020DB
:102D980000007A440000C84200000000D9F8FC3066
:102DA8001A78022A20D107EE90BAB8EEE70A5FED4A
:102DB800077A93ED097A80EE270A30EE070AB5EE16
:102DC800C00AF1EE10FA07D4B4EE670AF1EE10FA71
:102DD800C8BFB0EE670A01E01FED110A83ED090ACA
:102DE8000F200CF0E5F90AE099785944C829A8BFE2
:102DF800C82121EAE17199700F200CF0EFF9BAF1BE
:102E08000F0F00F0C181D9F8FC301A78022A1ED1C0
:102E180007EE90BAB8EEE78A5FED227A93ED080ADA
:102E280088EE278A38EE000AB5EEC00AF1EE10FAED
:102E380007D4B4EE670AF1EE10FAC8BFB0EE670A1D
:102E480001E01FED2B0A83ED080A122056E159789C
:102E58005944C829A8BFC82121EAE1715970122034
:102E680024E1D9F8FC301A78022A20D107EE90BA6A
:102E7800B8EEE70A5FED397A93ED0C7A80EE270A0F
:102E880030EE070AB5EEC00AF1EE10FA07D4B4EE38
:102E9800670AF1EE10FAC8BFB0EE670A01E01FED4D
:102EA800420A83ED0C0A10200CF082F90AE0197B23
:102EB8005944C829A8BFC82121EAE1711973102013
:102EC8000CF08CF9BAF1100F00F05E81D9F8FC30E3
:102ED8001A78022A1ED107EE90BAB8EEE78A5FED9B
:102EE800537A93ED0B0A88EE278A38EE000AB5EE7E
:102EF800C00AF1EE10FA07D4B4EE670AF1EE10FA40
:102F0800C8BFB0EE670A01E01FED5D0A83ED0B0A4A
:102F18001320F3E0D97A5944C829A8BFC82121EA67
:102F2800E171D9721320C1E0D9F8FC301A78022A6D
:102F380022D107EE90BA1FED6A0AF8EEE77A87EE1B
:102F4800800AD3ED0F7A30EE270AB5EEC00AF1EE0B
:102F580010FA09D45FED717AB4EE670AF1EE10FA4F
:102F6800C8BFB0EE670A01E01FED750A83ED0F0ACE
:102F780011200CF01DF90AE0997D5944C829A8BF11
:102F8800C82121EAE171997511200CF027F9BAF1ED
:102F9800110F00F0F980D9F8FC301A78022A20D1F4
:102FA80007EE90BA1FED860AB8EEE78A88EE008A27
:102FB80093ED0E0A38EE000AB5EEC00AF1EE10FAEB
:102FC80009D45FED8C7AB4EE670AF1EE10FAC8BF47
:102FD800B0EE670A01E01FED900A83ED0E0A142097
:102FE8008CE0597D5944C829A8BFC82121EAE1715C
:102FF800597514205AE0D9F8FC301A78022A1ED1E3
:1030080007EE90BAB8EEE78A5FED9E7A93ED0A0A6A
:1030180088EE278A38EE000AB5EEC00AF1EE10FAFB
:1030280007D4B4EE670AF1EE10FAC8BFB0EE670A2B
:1030380001E01FEDA70A83ED0A0A09205EE0D978AE
:103048005944C829A8BFC82121EAE171D9700920CB
:103058002CE0D9F8FC301A78022A1ED107EE90BA73
:10306800B8EEE78A5FEDB57A93ED0D0A88EE278A08
:1030780038EE000AB5EEC00AF1EE10FA07D4B4EE45
:10308800670AF1EE10FAC8BFB0EE670A01E01FED5B
:10309800BE0A83ED0D0A0A2030E0597B5944C8293D
:1030A800A8BFC82121EAE17159730A200CF096F8EB
:1030B8006AE0D9F8FC301A78022A22D107EE90BAD1
:1030C8001FEDCD0AB8EEE78A88EE008A93ED100A64
:1030D80038EE000AB5EEC00AF1EE10FA09D45FED39
:1030E800D37AB4EE670AF1EE10FAC8BFB0EE670AF9
:1030F80001E01FEDD70A83ED100A0B200CF058F8F9
:1031080042E0D97D5944C829A8BFC82121EAE17104
:10311800D9750B20CAE7012936D19878BA4B33F90B
:103128001230B3F5617F05DB40F633029342A8BF46
:10313800134601E04FF46173BAF10C0F24D14FF438
:10314800966292FBF0F0B14AA3F5617393FBF0F33A
:103158005FFA83F913784B4516D0B9F1040F34BFE1
:103168004B4602231370AA4A0AFB035303F2B673B1
:10317800136004F093FD504649460CF02FF809F10E
:103188000100C0B20CF0C8F8019A0123934094F8EA
:10319800F420134384F8F430019B01330193029B1C
:1031A8000C330293019B042B7FF410ADC6E4D8F8CE
:1031B8000030D80510D5974BDB786BB13368990789
:1031C8000AD5954B1B8813F0010A0AD10FF0D4FCDD
:1031D800012004F07FFC04E0012004F06AFC0123D4
:1031E80000E00023D9F8002052070DD563B1012073
:1031F80004F05FFC884B1B88980708D40FF0BCFCD0
:10320800022004F067FC02E0022004F052FC33685C
:1032180013F00A0F29D0D9F80030D9060BD57E4B08
:103228001B885A070AD4042004F054FC7B4B1B88E3
:10323800A4F8003102E0042004F03BFCD9F8003087
:103248009B0607D5744B1B88580606D4402004F00B
:1032580041FC02E0402004F02CFCD9F8003059066B
:1032680042BF6E4B1B88A4F8023133689A0609D412
:10327800D9F800301B0540F194804FF4807004F0B9
:1032880029FC92E0664BDFF890A11B7813F0020F3F
:1032980053D0644B1B78042B4FD9D9F8003013F462
:1032A800007B0FD0BAF80030DE063AD4102004F0C4
:1032B80011FC202004F0FDFB5B48011D07F01EF9FE
:1032C80002232AE0BAF8006006F01006B6B22EB162
:1032D800102004F0EEFB012684F804B1D9F8003080
:1032E800580512D5D4F8083150495A89B1F9003037
:1032F800002BB8BF5B42934207DAB1F90230002BCA
:10330800B8BF5B429342C0F20881BAF80030990610
:1033180008D5202004F0CDFB002384F804310126D1
:1033280000E0002694F80C31BBB90E200BF0CEFF5C
:103338003F4B012283F80C210FE0BAF8003003F06C
:103348003003002B94D0102004F0B3FB202004F0AD
:10335800B0FB002384F8043101E0002E88D0354BFF
:10336800002003F1280603F15004334A002122F813
:103378001010324A596022F810100432716022F895
:10338800101000221A609A603260B2602260616098
:10339800A26014331436143400287FF469AF012076
:1033A800E3E74FF4807004F084FB6B79082B01D0BD
:1033B8000E2B02D1402004F07CFBD8F800305A05CF
:1033C80040F1C18095F81C321BB93B7813F0040F0B
:1033D80003E0D9F8003013F4002F0BD0184B00226B
:1033E8001A703C2008F032FE002800F0AC800EF085
:1033F80001FDF6E70AF078FC09B0BDEC028BBDE8E8
:10340800F04F08F03EBD00BF2030002048300020BB
:1034180058110020C43300209C1A0020D01100202D
:10342800D8190020DE19002060110020D8110020D2
:10343800180F00202810002018340020A0100020A9
:1034480091280020012000E002205FFA80F909F1AC
:10345800FF3385F8B43704F087FB04F043FC484693
:103468000BF05AFFFFF70CBBBAF1000F02D07E2B0E
:103478003FF404AB94F8B930972B06D1344B4FF492
:10348800C872A3F8BE20FFF7FBBAA72B06D1314AB2
:10349800137843F004031370FFF7F2BA0022BB2B32
:1034A800079201D1022303E0B72B04D14FF6FE7334
:1034B800ADF81E3009E0BE2B01D1022303E0BD2B7D
:1034C8001AD14FF6FE73ADF81C30DBF80030BDF8AA
:1034D8001C10B3F858200A44A3F85820BDF81E1051
:1034E800B3F85A200A44A3F85A2004F0ADFD00238B
:1034F80084F8BA30FFF7C4BA792B04D1164AD378C6
:1035080023F0010306E07A2B7FF4BAAA124AD37893
:1035180043F00103D370FFF7B3BABAF800309B0643
:103528003FF500AF202004F0D5FA0C480C4B011DE4
:103538001A685B684360026006F0E0FF044B0126EE
:1035480083F80461EEE609B0BDEC028BBDE8F08FAC
:10355800180F0020D8190020C42900206811002065
:10356800E01900202DE9F04FC14BB3F90610C14B0B
:103578002DED028B1F687A8989B0914201930EDB89
:10358800B1F5FA6FFC79BDBF8B1A6343A2F5FA64F3
:10359800C4F16404BCBF93FBF4F4643400E0642415
:1035A800B54AB64BB2F894A192F95E211868049016
:1035B80092B20592054600220293AD4B33F91230C0
:1035C8000393CAEB030303F2F31640F2E630864294
:1035D8004FEA420B03D8002BB8BF5B4201E04FF41F
:1035E800FA73022A049E4FF064002FD096F811E176
:1035F800BEF1000F04D07345CCBFCEEB030300230C
:10360800DFF8C0E293FBF0FC6FF063093EF81C8022
:103618009B4E09FB0C390CF1010C3EF91CE00FFA2A
:1036280088FCCCEB0E0E0EFB09FE9EFBF0FEC6449A
:1036380026F80BE0BE1836797343924E93FBF6F3E7
:1036480064339BB2634393FBF0F02EE096F812E1EB
:10365800BEF1000F04D07345CCBFCEEB03030023AB
:10366800DFF84C8293FBF0F06FF0630C0CFB003931
:1036780038F910E00130002B38F91000CEEB0000CB
:1036880000FB09F9BDF8140099FBFCF9CEEB090918
:1036980019FB00F97A48A0F80490B879B8BF5B42E2
:1036A8004343784893FBF0F064306B78764E4FF0E4
:1036B800640E434393FBFEF3B354744EEB7A4343D7
:1036C80093FBFEF3B3546B7D6D4E5843704B90FBE8
:1036D800FEF0022A98546F4B0FD183F802E0039B47
:1036E80053450EDB644CB4F89621914215DBB1F5D5
:1036F800FA6FA8BF4FF4FA6110E09C54039B53453E
:1037080004DA36F80B305B4226F80B300132032A14
:1037180005F101057FF451AFE4E71146891A4FF42A
:103728007A73DFF8A4E1564D59436FF063036427B9
:10373800C2F5FA62B1FBF2F191FBF7F23EF8120022
:1037480003FB0211013203B23EF91220D21A51438F
:1037580091FBF7F30344F3804F4B1B885F0635D585
:103768004E4B4F4A1B881288DFED4E7A9B1A1BB2CC
:1037780008EE103AB8EEC88A28EE278AB0EE480A52
:1037880004F0F4F8F0EE408AB0EE480A04F08BF842
:10379800B5F9023006EE903AB5F90030F8EEE66A6F
:1037A80007EE903A20EE667AF8EEE77AA7EEA87A66
:1037B80067EE807ABDEEC77AE6EEA87A17EE103A81
:1037C800FDEEE77A2B8017EE903A6B80364D2B682A
:1037D800980740F1A180354B354F1A687B6945F24F
:1037E8000721D31A8B4240F397807A6109F072F867
:1037F800304BDFF8D8901A78032A9846B9F8003089
:1038080022D10A2B2AD90023282088F800300BF06F
:1038180020FD09F05FF8284B188809F045F8274B78
:103828001A68D37890FBF3F001300828244BA8BF1E
:1038380008201870537980B213FB00F33B83137987
:1038480013FB00F0788309E00A2B07D803231C4AEE
:1038580088F80030002313703B837B8398F800308E
:10386800144A012B3DD033D3022B4CD054E000BF77
:103878002030002058110020E011002030110020D5
:10388800D81100200CFEFFFFF41A0020B61000200B
:10389800081B0020142B00209C1A0020D0110020A7
:1038A8001A10002035FA8E3CE42F00200034002046
:1038B800A8100020241A002018290020C019002070
:1038C80080000020782B0020A61A0020C4190020B0
:1038D8003A8BB9F800309A421EDD012388F800308F
:1038E8000FE0B9F800107B8B8B4202DD02231370C6
:1038F8000FE0A34B1B8B0133994202DD00231370A9
:103908000AE0082006E07B8BB9F8002001339A42D0
:10391800E3DC07200BF0DAFC2D68290577D5994BF5
:10392800974F1A68FB69C3EB020845F207239845CD
:103938006DDD954BB6F906B0D3F80090FA6199F8A9
:103948000A30B4F84E11914E012B4FF47A70ABF552
:103958007A7B98FBF0F803D042D3022B20D041E0C9
:103968008B4B396A5A7B8B4B33F812204FF0080E79
:1039780092B291FBFEF3C91A8B18BA843B6240F6E7
:10398800E44293FBFEF39BB25343B9F80820C2EB21
:1039980013335843B9F9063090FBF3F0306021E057
:1039A8007D4BB9F808A01B78C6F800A05A0719D5AE
:1039B8007A480BF0E2FB20B915F0100F18BF4FF052
:1039C800000B32220BFB0BF393FBF2F3B9F9062041
:1039D8005B445A434FF47A7392FBF3F3534400E089
:1039E80000233360D7E90A0133686D4A03FB08F8FE
:1039F8004FF47A7398FBF3F810EB080041EBE87189
:103A08000023C7E90A010FF0FDF8664B1860664EFF
:103A18003368DB0427D52F0622D5644B1B789D0716
:103A28001ED5634B187804281AD90022614BD71881
:103A38000521951C4FF00A0E122AD154E9B287F8D5
:103A480001E004D0B0EB510F2A46EFD800E0142172
:103A58005A18322002F8010CFF225A540F2000E0B5
:103A68000A200BF033FC544D2A68002A50D0534BDF
:103A7800534F186839688142984649D8514BDFF846
:103A8800509119785268E1B94FF0010A83F800A003
:103A9800B9F80030D35C23B350460BF0F9FB4A4B1E
:103AA80083F800A00FF030F8B9F80030CBB92B68D4
:103AB8001B78053B534514D80BF0A4FB434B186007
:103AC8000FE04FF0000A83F800A0B9F80030D35C8B
:103AD8003BB150460BF0DCFB3B4B83F800A00FF0EA
:103AE80013F82A68B9F8003052683948D25CFE2ABF
:103AF80001D100230BE0FF2A02D10BF0CFFB07E036
:103B0800D8F800500A2111FB02523A6001330380B1
:103B1800214D2B78580703D52E4B08221A8571E0C2
:103B28003268D1075CBF43F001032B701F4B1B7831
:103B38001F075EBF2B7823F001032B70D60248BF06
:103B48002B78214A44BF23F001032B70224B1B68BA
:103B580013F0040F02D02149098851B92049098876
:103B680009B1980705D41F4B1B88003318BF0123E0
:103B7800D3B3022313702B7823F001032B7038E0A2
:103B8800A810002000340020C0190020CC19002003
:103B980000290020102900201F340020661300206F
:103BA800407E0500D0190020F4100020D81900200C
:103BB800DE19002074300020A02B002008300020DF
:103BC800982B0020942B0020E83300204832002056
:103BD8009C2B002000040048D41900201434002035
:103BE800D60F0020163400202978C90758BF0223B1
:103BF80013700BF007FBB44B1B68C01A002801DBDD
:103C08000EF082FFB14F0AF06FF83E78002E00F0F8
:103C1800AC80AF4B1A689846002A00F02387D8F882
:103C280000000BF0F5FB002800F01C87A84BA94CFE
:103C380018680BF0EAFB092801D03F2852D14FF051
:103C4800000A2668DFF8C892554636B1A248D9F866
:103C58000010324612F0B2FA10B9CA4605B94D46FC
:103C68009E4B09F110099945EFD3EDB1D5F800C085
:103C7800DAF8009023681CF803E019F8030070458F
:103C880012D15A1C944958B92D2B09D8DFF844E2AF
:103C9800CEF800204FF0200E01F803E0885403E02E
:103CA80001F803E02260E5E723680BB1554510D021
:103CB8008B480EF099F9554507D855F8100B0EF0BA
:103CC80093F909200EF088F9F5E786480EF08CF98B
:103CD800002623689E42A2D27F4B985D0EF07CF9A5
:103CE8000136F6E72368002B40F0A286042840F04E
:103CF800D886794809F076FA00F0B4BED8F8000002
:103D0800DFF8ECA10BF084FB28B3DAF800000BF025
:103D18007CFBDBF8003093F848100246A9BB242846
:103D28006CD1012283F84820DBF80030DFF8E4A1E9
:103D380093F84820062AE1D193F8490000F040FFA3
:103D48008346002800F083800EF0A2F8D9F80030EE
:103D5800002283F84820644B93F83530002B40F05C
:103D680055864C36982E00F07D86604BF21892F8F6
:103D78004A100129F5D1DFF89C91F358C9F80020C1
:103D88005B4ACB4613609046B8E7012904D14D2819
:103D980014BF00220222C5E7022904D13C2814BF1F
:103DA80000220322BEE703290CD140284FF000016E
:103DB80002D983F84810B7E758711971D971987109
:103DC8000422AFE7042906D1997983F849004A40CB
:103DD8009A710522A6E70529A6D15879197988424A
:103DE800987906D950409871481C18710B441A727A
:103DF8009AE790420CBF0622002293E72B783D49B0
:103E0800580791D4232ADAF8003013D101203870EA
:103E18002F480491036034480392036336480EF038
:103E2800E3F830480EF0E0F80499039A0B7843F071
:103E380002030B70314B1B681B78934201BF304B58
:103E4800304A1A60304B04BF304ADA606CE7DAF85F
:103E5800002092F849304C2B00F08A8400F28680CA
:103E6800332B00F0DD8421D8292B00F04D8409D8AC
:103E7800252B00F02584272B00F02884232B40F0E5
:103E88000C860AE22D2B00F0508407D82B2B40F02B
:103E980004860DF0CFFF607100F0B3BD2F2B00F04A
:103EA8002B85312B00F03D8500F0F7BD3E2B00F04F
:103EB800E68046D8372B00F0E6842DD8352B00F065
:103EC800278200F0EABD00BFEC3300202134002037
:103ED80064300020002A0020D0290020B892010870
:103EE8003BA9010840A90108A8100020F0270020DC
:103EF800801A00201F34002070A90108942800208F
:103F0800FC9F0020EFBEADDE00ED00E00400FA05E6
:103F1800D89001087C1A0020392B00F0E4833C2B50
:103F280040F0BB85DFF84884D8F800A00DF082FF88
:103F38008AF80000D8F8003018780BF0A9FC00F0D7
:103F480060BD432B00F07D8406D8412B40F0A58549
:103F58004FF0000800F069BC442B00F01785482B8F
:103F680040F09B8506F01EFD00F04BBDD12B00F004
:103F780068831FD8CC2B00F00B820ED8C82B61D0D9
:103F880004D84E2B00F01E8400F087BDC92B00F02A
:103F98003183CA2B7DD000F080BDCE2B00F01D836D
:103FA800C0F01283CF2B00F04782D02B00F00183A2
:103FB80000F073BDD82B00F001810BD8D32B3BD078
:103FC80027D3D42B00F07C82D62B40F066854FF0A7
:103FD80000086AE2F22B00F0C18212D8EF2B40F001
:103FE8005C85DFF88C83D8F800A00DF02DFFAAF8C7
:103FF8005A00D8F800800DF027FFA8F8580000F004
:1040080000BDF32B00F0C784FA2B00F0EF8200F01C
:1040180044BD2B7803F0040303F0FF08002B40F0A5
:10402800F0840DF007FF022884F8B40740F2C78235
:10403800CB4B83F8B487C2E20DF006FFC94B18805A
:1040480000F0DFBC92F805804FEA5808B8F1120F6B
:1040580003D907F0F7FF00F0D4BC4FF0000AC245BF
:1040680007D20DF0F1FEC04B23F81A000AF1010A3D
:10407800F5E7BE4B012283F8342000F0C2BC0DF0F6
:10408800D9FE84F8DE010DF0D5FE84F8DD0100F0DC
:10409800B8BCB74B1A681278022A4FF0000A984643
:1040A80070D1D8F800B00DF0C5FE07EE900AF8EE12
:1040B800677AB2EE048AC7EE887A0BEB8A0BCBEDEF
:1040C800087AD8F800B00DF0B5FE07EE900A9FED1B
:1040D800A97AF8EE677A0BEB8A0BC7EE877ACBEDF5
:1040E8000B7AD8F800B00DF0A5FE07EE900A9FED08
:1040F800A27AF8EE677A0BEB8A0BC7EE877A0AF199
:10410800010ABAF1030FCBED0E7ACAD1BAF1070F43
:10411800D8F800B01CD10DF08DFE07EE900AF8EE2D
:10412800677AC7EE887ACBED117AD8F800B00DF02F
:1041380081FE07EE900AF8EE677AC7EE887ACBED33
:10414800127AD8F800B00DF075FE8BF84C0012E02A
:104158000DF070FED3448BF80100D8F800B00DF0D4
:1041680069FED3448BF80B00D8F800B00DF062FE5E
:10417800D3448BF815000AF1010ABAF10A0FC5D128
:1041880000F03FBCD8F800B00DF054FED3448BF8D3
:104198000100D8F800B00DF04DFED3448BF80B00A9
:1041A800D8F800B00DF046FED3440AF1010ABAF17E
:1041B8000A0F8BF81500E5D100F023BC8246DFF822
:1041C800B0819FED6D8AD8F800B00DF03DFE07EE86
:1041D800900AF8EE677A0BEB8A0BC7EE887ACBED7C
:1041E800087AD8F800B00DF02FFE07EE900AF8EE26
:1041F800677A0BEB8A0BC7EE887ACBED0B7AD8F887
:1042080000B00DF021FE07EE900AF8EE677A0BEB8E
:104218008A0BC7EE887A0AF1010ABAF1030FCBEDCF
:104228000E7ACCD1BAF1070FD8F800B01CD10DF036
:104238000BFE07EE900AF8EE677AC7EE887ACBEDA8
:10424800117AD8F800B00DF0FFFD07EE900AF8EEED
:10425800677AC7EE887ACBED127AD8F800B00DF0FD
:10426800F3FD8BF84C0012E00DF0EEFDD3448BF813
:104278000100D8F800B00DF0E7FDD3448BF80B002F
:10428800D8F800B00DF0E0FDD3448BF815000AF122
:10429800010ABAF10A0FC5D1B3E30DF0CBFD13281B
:1042A80083463FF6D6AEDFF8C8A0DAF800800DF0F6
:1042B800C1FD0023314A0C2101FB0322117A8142FE
:1042C80022D10FFA8BFB08EB8B08137888F879302A
:1042D8000DF0B0FD88F87A000DF0ACFD88F87B0091
:1042E8000DF0A8FD264B274A1A6088F87C00264B5B
:1042F800DAF800001860002179300AF02DFF234B0E
:1043080080F0010018707CE301331C2BD2D1A0E6A9
:104318000DF090FD0B2882463FF69BAE144BD3F868
:1043280000800DF087FD03283FF693AE062303FBBC
:104338000A8888F8CE000DF07DFD88F8C9000DF0D8
:1043480079FD88F8CA000DF075FD88F8CB000DF0EE
:1043580071FD88F8CC000DF06DFD88F8CD0050E3B4
:10436800E01100201810002020300020A8100020A4
:10437800301100200000C84200007A444887010834
:104388001010002020130020141000201800002016
:104398005379092B7FF65DAE019BD3F800800DF0B1
:1043A80049FD019B88F80000D3F800800DF042FD1C
:1043B80088F801000DF03EFD019B64281B68A8BF2A
:1043C800642018710DF036FD019B64281B68A8BF96
:1043D800642058710DF02EFD019BFF281B68A8BFB3
:1043E800FF2098710DF026FD019B6428D3F800800A
:1043F80028BF642088F807000DF01CFD019B88F891
:104408000200D3F800800DF015FD019B88F8030029
:10441800D3F800800DF018FDDAF80030A8F80A008B
:104428005B790A2B40F2ED82D84BD3F800800DF06F
:1044380001FD88F80800E4E20DF006FD6FF4AF62B4
:1044480083189BB2C62B98BFA4F894010DF0FCFC0E
:10445800A4F840010DF0F8FCA4F842010DF0F4FCBA
:10446800A4F844010DF0F0FCA4F8D6010DF0E2FC2C
:1044780084F8EB010DF0DEFC0DF0DCFC84F8EC01B7
:104488000DF0D8FC84F883010DF0D4FC84F8900179
:104498000DF0D0FCBE4BD3F800800DF0D5FC00EB3E
:1044A80080004000A8F856001DE10DF0CDFCB94B86
:1044B80023F8180008F10108B8F1080FF5D1A0E2B7
:1044C80053790F2B7FF4C5AD0DF0B4FC0728804657
:1044D8003FF6BFAD029BD3F800A00DF0B5FC0E234C
:1044E80003FB08F8C244029BAAF81901D3F800A0FC
:1044F8000DF0AAFCC244029BAAF81B01D3F800A045
:104508000DF0A2FCC244029BAAF81D01D3F800A03A
:104518000DF090FCC244029B8AF81F01D3F800A05A
:104528000DF088FCC244029B8AF82001D3F800A051
:104538000DF080FCC244029B8AF82101D3F800A048
:104548000DF078FCC244029B8AF82201D3F800A03F
:104558000DF084FCD044C8F8230152E20DF06AFC47
:104568000F2880463FF675ADC8EBC8080DF062FC11
:1045780004EB080303F1D00883F8D0000DF05AFCCF
:1045880088F801000DF056FC88F802000DF052FC86
:1045980088F803000DF04EFC88F804000DF04AFC82
:1045A80088F805000DF046FC88F806000BF0D4F8F2
:1045B80027E22B785B0700F124820CF0A5FB03F0BF
:1045C800D3FA03F08FFB1CE22B78580700F119820D
:1045D800714B4FF4C8721A8013E22B78590700F117
:1045E80010826E4A137843F0040328E02B785A07A8
:1045F800E5D552E20DF01EFC684B1A7810B142F076
:10460800020201E022F002021A700DF013FC644B62
:10461800DFF8AC8118700DF021FCC8F800000DF02F
:104628001DFCC8F804000DF00FFC5E4B18800DF05F
:104638000BFC5D4B5D4A1880137843F0020313703E
:10464800DFE10DF0F7FB03900DF008FC83460DF059
:1046580005FC82460DF002FC80460DF0F5FB0DF0DE
:10466800F3FB0DF0E7FB039BA3B9514B1020C3F8F4
:1046780000B0C3F804A003F01CFA484A137843F0CA
:1046880001031370B8F1000F00F0BB81494BC3F868
:104698000080B6E1102B40F0B481474BC3F800B05E
:1046A800C3F804A0B8F1000F02D0424BC3F8008051
:1046B8004148424B0222011D1A7005F01FFFA0E17C
:1046C800A0600DF0CBFB03F01DFA9AE10DF0BCFBE6
:1046D800A4F858010DF0B8FBA4F85A010DF0B4FB8A
:1046E800A4F85C018DE10DF0A5FB84F878010DF0CC
:1046F800A1FB84F87C010DF09DFB84F87B010DF093
:1047080099FB84F87D017CE10DF09EFBA4F87E0105
:104718000DF09AFBA4F880010DF08CFB84F882015F
:104728000DF092FBA4F884016BE10DF083FB84F893
:104738008E010DF089FBA4F898010DF085FBA4F813
:1047480094010DF081FBA4F896010DF073FBDAF8E3
:10475800003084F88F015B79082B40F252810DF00C
:1047680073FBA4F89A010DF06FFBA4F89C0148E1D3
:104778000DF060FB84F8D4010DF05CFB84F8D501E2
:104788000DF062FBA4F8D6013BE100BF58110020F0
:10479800301100204A300020D60F0020D819002000
:1047A800DE190020DC190020DA1900205E11002033
:1047B8006011002070110020681100201C100020DA
:1047C800E019002092F805800323B8FBF3F8B8F14C
:1047D800120F3FF63EACDFF8E4A34FF0000BC345E1
:1047E80080F00F810DF026FB8AF89E010DF02CFB5E
:1047F80040F2ED23984205DD40F6CA039842A8BF6F
:10480800184601E040F2EE20A0F2EE2019230BF149
:10481800010B90FBF3F00AF1020A8AF89D01DEE72A
:104828000DF008FB84F89001EBE00DF003FB04EBBE
:10483800080308F10108B8F1080F83F88601F4D1DC
:10484800DFE00DF0F7FAC4F808B060710DF006FB70
:1048580003F058F90DF0EEFA84F88E010DF0F4FA31
:10486800A4F858010DF0F0FAA4F85A010DF0ECFA8A
:10487800A4F85C010DF0E8FAA4F87E010DF0E4FA62
:10488800A4F88001BDE053794FF0070AB3FBFAF2B0
:10489800C2EBC2029A1A12F0FF0F7FF4DAABB3FB35
:1048A800FAFA0AF1FF3A5FFA8AFABAF1FF0F00F052
:1048B800A8800DF0BFFA5FFA80FB4FFA8BF002F088
:1048C800E1FB804600283FF4C4AB80F800B00DF04F
:1048D800BBFAA8F802000DF0ADFA88F804000DF054
:1048E800A9FA88F805000DF0A5FA88F807000DF078
:1048F800A1FA88F80600D4E7DFF8C08208F1400A78
:104908000DF0A2FAA8F8AC020DF094FA88F8AE02FD
:104918000DF090FA08F1040888F8AB02D045EFD101
:104928006FE00DF087FA1F2880463FF692ABD9F862
:1049380000305B79082B7FF48CAB0DF085FA08F119
:104948008A0804EB880800F03F00A8F806000DF07C
:104958007BFAB8F80630800100F4FE501843A8F836
:1049680006000DF067FA000188F804000DF062FAFD
:1049780098F8043000F00F00184388F804000DF090
:1049880059FA88F805000BF0E5FB3AE0784B01226C
:1049980083F8352035E00DF04DFAFF2882461BD10B
:1049A80000238DF81F309DF81F30072B29D89DF85C
:1049B8001F00704A9DF81F3052F8300002EBC30305
:1049C80001215B68994089B2042202F06DFA9DF8D2
:1049D8001F300133DBB2E4E707283FF63AAB00208B
:1049E8000DF07AFA0DF054FAD8F800000AF007FD35
:1049F80018B932200AF02DFCF6E74FFA8AF002F0D7
:104A080061FA00200DF068FAFFF79EB95A4B9859E1
:104A18000AF0F5FC18B932200AF01BFCF6E70AF098
:104A28005BFE03F077F8554B554ADA60FFF799B902
:104A38000C2838D00A283FD1524D53480DF0D4FAEB
:104A48002846232111F0A3FB08B1401B20602368EE
:104A5800002B54D14B4823600021302211F061FB18
:104A68003B781BBB494B1B689B060FD5484B4049FD
:104A78001B688A6B9A1A002A08DB464A1278042AAD
:104A880082BF03F5123303F5F8738B63424B9B68BF
:104A9800002B67D04148984764E007F0D3FAFFF746
:104AA80053B90C2804D13E480DF09EFA3D480DE05C
:104AB8007F2812D1FFF7B3B80D28BDD07F2809D1C0
:104AC800013B304A384823600021D1540DF08CFA5C
:104AD800FFF7A5B82F2B3FF6A2A8A0F12002D2B26B
:104AE8005E2A3FF69CA813B920283FF498A85A1CC0
:104AF8002260244AD0540DF06FFAFFF790B85A1E7E
:104B0800A95C202901D11346A2E71E4A236000218F
:104B1800D154264B264DD3F800A0D5F800B0DFF8C5
:104B28006490584611F041FB0646324648465946BD
:104B380011F044FB1F4A28B919F8063053445B7832
:104B48005B0703D010359542E7D306E0954204D2BF
:104B5800701CEB684844984702E017480DF044FA87
:104B6800002377E709B0BDEC028BBDE8F08F00BFEA
:104B7800A8100020C0AC0108F027002000ED00E0DC
:104B88000400FA05D0290020E3BA0108D41900204E
:104B980000340020DE1900205C1B0020E4100020F7
:104BA80045A9010840A901086CA901089000002046
:104BB800D8900108B892010850A90108E011002016
:104BC8002DE9F0472DED028B4D28A0B0044600F0EA
:104BD8004F8600F2BD80302800F0CC8651D82228BC
:104BE80000F09C8423D8032800F00E8214D80128F2
:104BF80000F0FE81022840F0288704200DF06CF9AF
:104C080043200DF034F94C200DF031F946200DF019
:104C18002EF94C2000F052BE042800F0FE81052831
:104C280040F013871A200DF057F9002405E22828D0
:104C380000F0EC8515D8242800F0D385262840F00C
:104C48000487D34C06200DF047F9B4F858010DF04D
:104C580046F9B4F85A010DF042F9B4F85C0100F0D5
:104C6800BDBD2C2800F0E5852E2800F052862A28A4
:104C780040F0EB8601200DF02FF9C54B587900F074
:104C88001DBE3D2800F002831ED8362800F0278676
:104C98000BD8322800F00C86342840F0D6864820FD
:104CA8000DF01AF9002500F05BBC3A2800F0C38229
:104CB8003B2800F02C84382840F0C78604200DF0EB
:104CC8000BF9B34C00F093BD452800F0AB8627D80C
:104CD800402800F0F685422840F0B786AC4C1020FA
:104CE8000DF0FAF860790DF0C2F8A0680DF000F93F
:104CF80094F88E010DF0BBF8B4F858010DF0EFF8F8
:104D0800B4F85A010DF0EBF8B4F85C010DF0E7F8CF
:104D1800B4F87E010DF0E3F8B4F8800100F05EBD50
:104D2800472800F05D86C0F04A864B2840F08D8603
:104D3800974C04200DF0D0F894F8D4010DF097F8B2
:104D480094F8D5010DF093F8B4F8D60100F046BDFB
:104D5800702800F0F18200F2E580692800F04B82AB
:104D680000F2B680662800F0A58100F2A6806428CB
:104D780000F07C81652840F06886864C0B200DF099
:104D8800ABF820880DF0ABF86268834B9A420CBFF1
:104D98002089608980B20DF0A2F8804B1B68C3F3AC
:104DA800C000C3F38002800040EA4200C3F340021F
:104DB8001043C3F3401240EAC20003F01003184343
:104DC8000DF08DF8764B1A88E368247C02F0080110
:104DD80003F4475949EA010903F4804149EA010902
:104DE80003F4004149EA010903F4803149EA010961
:104DF80003F4003149EA010903F4802149EA010971
:104E080003F4002149EA010903F4801149EA010980
:104E180003F0007349EA0303DFF8A49199F80090BE
:104E280012F0010FC9F3800914BF4FF002084FF0C8
:104E3800000843EA090312F0020F43EA080314BF0B
:104E48004FF0040C4FF0000C12F0040F43EA0C0C66
:104E580014BF4FF0100E4FF0000E12F0400F14BFA9
:104E6800202700274CEA0E0E12F0100F14BF4FF443
:104E7800007600264EEA070712F0200F14BF4FF401
:104E8800806500253E4312F4807F14BF4FF4006014
:104E98000020354312F4007F14BF4FF400110021A5
:104EA800284312F4806F41EA000114BF4FF0806379
:104EB8000023002019430346E8E0672800F0228118
:104EC800682840F0C28510200DF006F8002489E11A
:104ED8006C2800F0A38117D86A2800F003846B2897
:104EE80040F0B38505200CF0F7FF2E4B18880CF026
:104EF800F6FF2D4B18880CF0F2FF264B93F876003E
:104F080000F0010000F0DABC6E28224D00F0998113
:104F180000F2EA8106200CF0DFFF686E0CF0E8FF73
:104F2800224B86E1782800F0FA8018D8742800F01F
:104F380038830AD8722800F09583732840F0858555
:104F480008200CF0C9FF0124C5E3762800F0EA83A5
:104F580000F268832F200CF0BFFF154CCFE2A42885
:104F680000F008842ED87B2800F06F82A02840F03B
:104F78006C850C200CF0B0FF0E4B18680CF0B8FFD5
:104F88000D4B18680CF0B4FF0C4B186800F059BDB5
:104F9800E0110020E810002000540040D41900203F
:104FA8009C1A0020521A0020541A0020C811002010
:104FB80017870108ACF7FF1FB0F7FF1FB4F7FF1FF3
:104FC8001F340020F12800F0E680FE2800F0F98365
:104FD800F02840F03A85B34C04200CF07DFFA36C18
:104FE800B3F85A000CF07BFFA36CB3F85800F5E354
:104FF80003200CF071FF00200CF039FF20460CF064
:1050080036FF0D2000F05ABC0CF066FF01200CF0B2
:105018002EFF0A200CF02BFFAAE306200CF05CFF01
:1050280053200CF024FF52200CF021FF46200CF0F6
:105038001EFF33200CF01BFFCFE39B4B185D0134A0
:105048000CF015FF0B2CF8D10024984B185D013497
:105058000CF00DFF082CF8D10024954B185D013495
:105068000CF005FF072CF8D100F0EDBC07200CF080
:1050780033FFE7200CF0FBFE8E4B58790CF0F7FE5F
:1050880000200CF0F4FE042000F0DBBCA3420AD29E
:10509800894A9D5C012202FA05F50D421CBF9A401F
:1050A80010430133F2E70CF023FF824B93F8B40767
:1050B80000F004BC12200CF00FFF804B1B88B3F5E6
:1050C800806F8CBF0825012500247D4B33F914001F
:1050D80090FBF5F0013480B20CF001FF032CF4D101
:1050E800704CA08D0CF0FBFEE08D0CF0F8FE208ECD
:1050F8000CF0F5FE608E0CF0F2FEA08E0CF0EFFEC8
:10510800E08E6BE310200CF0E7FE00246D4B185D79
:1051180001340CF0ACFE102CF8D100F094BC7020D7
:105128000CF0DAFE00265F4D0E24AB6C744323446A
:105138000136B3F819010CF0D2FEAB6C2344B3F876
:105148001B010CF0CCFEAB6C2344B3F81D010CF032
:10515800C6FEAB6C234493F81F010CF088FEAB6CC1
:10516800234493F820010CF082FEAB6C234493F89F
:1051780021010CF07CFEAB6C234493F822010CF067
:1051880076FEAB6C1C44D4F823010CF0B1FE082E5B
:10519800C9D100F058BC7020464C0CF09DFE04F1BB
:1051A800700594F8D0000CF062FE94F8D1000CF071
:1051B8005EFE94F8D2000CF05AFE94F8D3000CF07E
:1051C80056FE94F8D4000CF052FE94F8D5000CF07A
:1051D8004EFE073494F8CF000CF049FEAC42E0D103
:1051E80000F031BC384B185D01340CF040FE102C37
:1051F800F8D100F028BC354D2878400000F0FE00BA
:105208000CF06AFE00242B789C4280F01C84304B02
:1052180033F814000CF063FE0134F4E72D4C06203B
:105228000CF05AFE20880CF05AFE60880CF057FEED
:10523800294B1888D2E204200CF04EFE194B986EC8
:10524800FFE307200CF048FE244B1888FF28A8BF6E
:10525800FF20C0B20CF00BFE214B186880F3100041
:1052680080B20CF03CFEB5F86C000CF038FE114B27
:1052780093F883211B4B186822B10A23584380F303
:10528800100001E000F30F0080B2A7E2094C0220F1
:105298000CF022FE94F8DE010CF0E9FD94F8DD0133
:1052A8000CE300BFE8100020A8A90108B4A9010870
:1052B800BDA90108E0110020F91000202C000020F1
:1052C800C211002020110020341100208C28002059
:1052D80020300020DC2F0020D0110020C41900202D
:1052E800D0190020CC1900200B200CF0F5FD2B6FF5
:1052F80018780CF0BCFD2B6F58780CF0B8FD002620
:105308002B6FC44C3344013618790CF0B0FD032ED2
:10531800F6D1236FD8790CF0AAFD236F98780CF09A
:10532800A6FD236FD8780CF0A2FD236F58890CF0E6
:10533800D6FD236F187AC1E2B64C1E200CF0CCFDC6
:10534800A36C1B78022B4FF000056BD1A36C03EB09
:10535800850393ED080AB2EE048A20EE080A11F0DC
:10536800EFF880F30800C0B20CF081FDA36CDFED0C
:10537800AA7A03EB850393ED0B0A20EE270A11F0B6
:10538800DFF880F30800C0B20CF071FDA36CDFED0C
:10539800A37A03EB850393ED0E0A20EE270A11F09A
:1053A800CFF880F30800C0B201350CF060FD032D82
:1053B800CCD1072DA36C23D193ED110A20EE080A56
:1053C80011F0BEF880F30800C0B20CF050FDA36CD9
:1053D80093ED120A20EE080A11F0B2F880F30800E3
:1053E800C0B20CF044FDA36C93F84C3000EE103AB8
:1053F800B8EE400A11F0A4F880F30800C0B20BE040
:105408002B4458780CF033FDA36C2B44D87A0CF05D
:105418002EFDA36C2B44587D01350CF028FD0A2D78
:10542800C7D110E3A36C2B4458780CF020FDA36C73
:105438002B44D87A0CF01BFDA36C2B440135587D06
:105448000CF015FD0A2DEDD1FDE23C200CF044FDD9
:105458000024704D9FED718AAB6C03EB840393EDD0
:10546800080A20EE080A11F06BF880B20CF037FD3C
:10547800AB6C03EB840393ED0B0A20EE080A11F0E2
:105488005FF880B20CF02BFDAB6C03EB840393ED5B
:105498000E0A20EE080A11F053F8013480B20CF01D
:1054A8001EFD032CD5D1072CAB6C16D193ED110A38
:1054B80020EE080A11F044F880B20CF010FDAB6C35
:1054C80093ED120A20EE080A11F03AF880B20CF0B7
:1054D80006FDAB6C93F84C000BE0234458780CF0B5
:1054E800FEFCAB6C2344D87A0CF0F9FCAB6C23447B
:1054F800587D01340CF0F3FC0A2CD4D1A3E214F843
:10550800010F002800F09F820CF0B1FCF7E70120A2
:105518000CF0E2FC3F4B9B6C1878CFE150200CF06C
:10552800DBFC00253B4B9C6C3D4B04EB85040C21BC
:1055380094F8792001FB0233013593F838000CF018
:1055480096FC94F87A000CF092FC94F87B000CF02E
:105558008EFC94F87C000CF08AFC142DE2D172E2E7
:105568002C4B9C6C062303FB0544013594F8CE00B4
:105578000CF07DFC94F8C9000CF079FC94F8CA0092
:105588000CF075FC94F8CB000CF071FC94F8CC008E
:105598000CF06DFC94F8CD000CF069FC0C2DDFD1FB
:1055A80051E24FF00008012600271A4B1A7C974257
:1055B80027DA11330024FA5C194D0C2305F1300168
:1055C8006343595C914207D12B44586B10F0EDFDB1
:1055D80082462EB9B14605E001341C2CECD10EE010
:1055E80080440CE0D1450ADA0C2303FB04535B6BBF
:1055F80013F809000CF03BFC09F10109F2E7013747
:10560800D3E7002E00F01F825FFA88F00CF064FCEC
:105618000026C9E7E81000200000C84200007A44CC
:1056280018870108C64D287C0CF056FC00242B7CFA
:105638009C4280F00882C34BE65C0021C2480C22E1
:1056480000F1300702FB01F3DA5DB24205D10344F1
:1056580093F838000CF00BFC02E001311C29EDD165
:105668000134E4E7B94C16200CF036FCB4F8940188
:105678000CF035FCB4F840010CF031FCB4F84201F0
:105688000CF02DFCB4F844010CF029FCB4F8D60158
:105698000CF025FC94F8EB010CF0E9FB00200CF071
:1056A800E6FB94F8EC010CF0E2FB94F883010CF0B3
:1056B800DEFB94F890010CF0DAFB00200CF0D7FB2D
:1056C8009F4B9B6C0A20B3F9563093FBF0F080B2E5
:1056D8000CF005FC8BE0E0B201340CF0C8FB092C9F
:1056E800F9D1B0E110200CF0F7FB994B994C1878E0
:1056F80000F002000CF0BBFB974B18780CF0B7FBDE
:1057080020680CF0F5FB60680CF0F2FB934B1888EE
:105718000CF0E5FB924B18880CF0E1FB884BB3F8D2
:1057280074005BE00CF086FB074612200CF0D4FBFB
:10573800834C17B9A66FE56F07E0102F13BF00253C
:10574800D4F88060D4F884502E4638460CF08FFB8D
:1057580030460CF0CDFB28460CF0CAFBD4F8880084
:105768000CF0C6FB00200CF0BAFB00200CF0B7FBD5
:105778000020A3E0724D95F88C0080000130C0B283
:105788000CF0AAFB95F88C000CF071FB00242E4657
:1057980096F88C309C4280F05681724D285D0CF052
:1057A80066FB05F11003185D0CF061FB05F12003A1
:1057B8003035185D0CF05BFB285D0CF058FB0134AC
:1057C800E6E708200CF088FB00200CF088FB00209E
:1057D8000CF085FB00200CF082FB00200CF07FFB16
:1057E80031E104200CF078FB584B986829E194F8D3
:1057F80078010CF03CFB94F87C010CF038FB94F831
:105808007B010CF034FB94F87D0157E04F4C0720E6
:105818000CF062FBB4F87E010CF061FBB4F8800177
:105828000CF05DFB94F882010CF021FBB4F88401C4
:10583800D4E7464C0C200CF04FFB94F88E010CF08A
:1058480016FBB4F898010CF04AFBB4F894010CF07C
:1058580046FBB4F896010CF042FB94F88F010CF06B
:1058680006FBB4F89A010CF03AFBB4F89C01B5E7D2
:105878003D4C3E4D207800EB4000C0B20CF02CFBB4
:10588800002623789E4205F1020580F0DC8015F899
:10589800020C0CF0ECFA15F8010C00EB800000EBA0
:1058A800800000F2EE2080B20CF019FB0136E8E728
:1058B80001200CF011FB254B93F890010CF0D7FA5E
:1058C800C1E008200CF008FB0024204B23440134DD
:1058D80093F886010CF0CBFA082CF6D1B3E0184BFC
:1058E8001A4C93F8CD00C0EBC000C0B20CF0F4FA2B
:1058F80004F1280594F8F20100231D4AD25C904275
:1059080000F0A5800C333C2BF7D10834AC42F1D120
:1059180099E040200D4C0CF0DFFA04F14005B4F892
:10592800AC020CF0DCFA94F8AE020CF0A0FA0434E5
:1059380094F8AB020CF09BFAAC42F0D183E000BFC4
:10594800E8100020F910002018870108E011002055
:10595800D8190020E0190020DE190020DC190020E9
:10596800DA190020751100208C2800207E130020F1
:1059780098280020E020444C0CF0AEFA04F1800591
:10598800B4F82E0200F03F000CF0A9FAB4F82E0289
:10599800C0F386100CF0A3FA94F82C0200090CF05E
:1059A80066FA94F82C0200F00F000CF060FA043448
:1059B80094F829020CF05BFAAC42E1D143E0334C95
:1059C8000D200CF089FA05F007FD0CF050FA20883C
:1059D8000CF08EFAE0680CF08BFA04F0EDFE30E083
:1059E8000CF03CFA054684200CF076FA28460CF0B8
:1059F8007FFA264BDC6805F18003A3428CBF641B49
:105A0800802404F091FF28462246694605F018FDD7
:105A180000240546AC4216DA1DF804000CF027FAFB
:105A28000134F7E713200CF057FA0024184B185DDF
:105A380001340CF01CFA0B2CF8D100200CF058FAA9
:105A480000200CF055FA012018E0002016E00CF0B8
:105A58000EFAB4F8F4010CF042FA94F8F6010CF0DE
:105A680006FA94F8F7010CF002FA94F8F9010CF030
:105A7800FEF994F8F8010CF0FAF946E720B0BDEC0D
:105A8800028BBDE8F08700BFE01100201C00002059
:105A9800A8A901082DE9F047D14CD24F237886B048
:105AA8000646002B00F0F8813A686368D31A7C2B0D
:105AB80040F2F281237A6260013323724FF00008CA
:105AC80008F12400C64DC0B208F0C2F805F10A0377
:105AD80033F9183007EE903AC34B1B88B8EEE77AD3
:105AE80007EE903AF8EEE77A08F10108C7EE277A50
:105AF8009FEDBE7A67EE877AFDEEE77ACDED037A01
:105B0800BDF90C0008F092F8B8F1030FD8D1302095
:105B180008F09EF8B5F9100008F088F808F090F839
:105B28002B7A9A072CD16A6841F288339A4218D99D
:105B3800102008F08DF84FF06408686990FBF8F0C1
:105B480000B208F073F8212008F082F8686990FB29
:105B5800F8F308FB13000028B8BF404200B208F071
:105B680065F8142008F074F8B4F9180008F05EF825
:105B78001C2008F06DF8002008F058F808F060F8CC
:105B8800237ADFF85C825B0740F06381022008F02B
:105B98005FF8D8F81C00DFF86C926423323090FB71
:105BA800F3F000B208F042F80320B8F9265008F0E4
:105BB8004FF88F4B1B7813F0040F4FF0050A95FB35
:105BC800FAF5ADB20DD008F5D770314609F0D5FA1F
:105BD80028B9D9F8003013F0100F18BF002528B2E3
:105BE80005E0D8F808389889B0FBFAF000B208F058
:105BF8001DF8D9F800309E076ED5DFF80C92B4F87E
:105C08000E6899F80030B4F80C28754D36014FF03D
:105C18006408B6B208FB02325B00B2FBF3F346EA53
:105C28000326B6B2C3F303231E43062008F010F878
:105C380030B207F0FBFFB4F80E3899F800100133C2
:105C48009BB293FBF1F201FB1233A4F80E38D4F89F
:105C580010389B7B012B05D1392007F0F9FFB5F9E6
:105C68000C081AE0B5F80C586E233A205D43152647
:105C780007F0EEFF95FBF6F5AEB2B6FBF8F528B2E5
:105C880007F0D4FF08FB15653B2007F0E1FFA8B239
:105C9800451D0A2095FBF0F000B207F0C7FF282049
:105CA80007F0D6FFD4F814380A2093FBF0F000B2BE
:105CB80007F0BCFF042007F0CBFFD4F808389B8915
:105CC80013B106F0C9FD04E0454BD3F8180880F37A
:105CD800100000B207F0AAFFD4F81C38404E9D0609
:105CE80040F1AC8096F8203898071DD5112007F0B0
:105CF800AFFFB6F822083F4B4FF4F365684390FBBB
:105D0800F3F000B207F092FF192007F0A1FFB6F8F0
:105D180022084543642095FBF0F595FBF0F300FB62
:105D2800135000B207F082FF94F82038B4F82458D2
:105D380013F0020F08BF0025012007F089FF28B2E1
:105D480007F074FF092007F083FF002007F06EFFBB
:105D5800294B94F826581A88B2F5967F0AD9204B11
:105D68001B7A03F00F03072B04D842F20F759542F4
:105D780028BF1546052007F06BFFD4F810385B7B69
:105D88000BB928B21CE0A5F1200307EE903A9FED6D
:105D98001B7AF8EEE77AF6EE006AC7EE877ABEEE6F
:105DA800007AF5EEC07AF1EE10FA58BFB0EE667AD6
:105DB80077EE877AFDEEE77ACDED037ABDF90C0030
:105DC80007F034FF94F82028054B910703D493F883
:105DD8002728012A1CD1012384F82738084834E0F1
:105DE800B8110020083000202C00002000007A4460
:105DF8001F340020A0860100820000206666E63F6E
:105E0800E0190020E42F0020800000208096184B25
:105E1800D3F810385FED036A93ED017AD3ED027A77
:105E280027EE267A67EEA67ABDEEC77AFDEEE77A08
:105E38008DED047ACDED057A04A806E0B74A92E81C
:105E4800030004AB83E80300184607F011FF07F0CE
:105E5800F7FE237A282B1FD1B14B00221A723C2659
:105E68003B684FF47A70B3FBF0F8172007F0F0FEA8
:105E7800B8FBF6F5B5FBF6F006FB1050000200B2D1
:105E880007F0D4FE182007F0E3FE06FB158000B2E9
:105E980007F0CCFE07F0D4FE94F83038A04D002B64
:105EA80000F05D8109F0AEF9D5F834389D4AC31A7F
:105EB8009342064640F2C680002385F83A3885F8B2
:105EC8003C38B5F80C38DAB21B0A85F8562885F83C
:105ED800573885F84C2885F84D38D5F864283B683C
:105EE8009A1AD5F86838D97B4FF47A734B439A429B
:105EF8000ED38D4B1B68C5F8643895F86C38013B98
:105F0800012B9FBF102385F83A38022385F83C38C7
:105F18000A20D4F8142892FBF0F284F854281212BC
:105F280084F8552894F82028D4F8183893FBF0F30F
:105F380084F858381B1284F85938920794F8263890
:105F4800774984F8873803D42D2381F8883877E097
:105F5800042BD4F82898D4F82C78DFF8DC81734A1D
:105F68008CBF3323322381F888384FF0060C704BEE
:105F780099FBF3F097FBF3F308FB009108FB037818
:105F880003EB83030CFB01F103EB830391FBF2FEAC
:105F9800642502FB1E119B0091FBF5F184F879182A
:105FA80009120CFB08FC84F87A189CFBF2F143FAFE
:105FB80081F39BB202FB11C292FBF5F284F87E28B2
:105FC800121284F87C3884F87F281B0AB4F8222837
:105FD80084F87D382423534393FBF5F5B4F89A38B5
:105FE80084F8803800EB80001B0A00EB80008000FA
:105FF80084F881380A22B4F82438B3FBF2F303F5A5
:10600800FA739BB240FA8EF080B284F882381B0A89
:106018004FEAD97984F87708FF0F000A84F8745892
:1060280084F88338C5F30725B4F89C3884F8769843
:1060380084F8780884F87B7884F8755884F8893867
:10604800C4F8346894F89E88354DB8F1000F0DD126
:10605800D5F8A40809F0DCF9012807D90228354F3A
:1060680000F05B8202F05EFD0123BB70D4F8A82823
:106078002B4D002A73D095F89E783FB1D5F8B038EB
:1060880040F6B731F31A8B4219D868E00123D5F8E6
:10609800A40885F89E3800F092FFD5F8B43893F933
:1060A800000002238DE8880008213A464FF4964301
:1060B80000F098FF85F8B878C5F8A4084DE095F881
:1060C800AC78CFB9D5F8A408C5F8A87885F89E7833
:1060D80000F075FFD5F8B43893F9000001238DE876
:1060E800880008213A464FF4964300F07BFFC5F834
:1060F800A40802F017FD30E0013FFFB285F8AC7844
:1061080095F8B81895F8B938C7B94A1C013385F815
:10611800B82885F8B938D5F8A4081CE0A48801087F
:10612800B81100203F0D03000830002040420F0046
:10613800809698002C000020806967FF12F8017B88
:10614800C5F8A828781885F8B8080133D5F8A40840
:1061580085F8B938394609F05EF9C4F8B06894F89A
:10616800BA38A14DDBB1D5F8BC38C3B1D5F8C038C1
:10617800ABB1C5F8C4381B689C4AC5F8C838D5F80F
:10618800CC381344187AFEF71BFD0BF081FED5F8C6
:10619800CC380133092B88BF0023C5F8CC38944D7F
:1061A80094F8D0282E68904B002A00F0F181D3F89B
:1061B800D428002A00F0EC8193F8D838013B012B51
:1061C80000F2E681D4F8D408874F09F021F9E0B14C
:1061D800D7F8D40809F019F997F8D938D5F8009004
:1061E8007E2B80460ED102231B2887F8D83809D188
:1061F800D7F8D40809F00CF920B90123C7F8DC98BE
:1062080087F8E03884F8D988DCE7D7F8DC282B68E9
:106218009B1A41F6583293421ED9032387F8D8387F
:10622800B6E1744A32F8130010B903464FF403601C
:106238000133B0F5C06FDBB279D01ED9B0F5006F6D
:106248007FD032D9B0F5036F3FD184F8E138D4F864
:106258001C38654F99063FD494F8E01894F8E13853
:10626800002900F057812A68921B012AD9D984F89D
:10627800E138002384F8E0388AE1B0F5007F43D0A4
:1062880007D8B0F5807F49D0B0F5887F00F08D80C1
:10629800E6E7B0F5806F00F0B180B0F5826F00F0EE
:1062A800F680B0F5047FDBD123E0B0F5E26F00F0B3
:1062B8008D80B0F5E46F00F08E80B0F5E06FCFD13F
:1062C80084F8E138B4F90A1089E0B0F5046F76D0A3
:1062D800B0F5026FC4D106E197F820389A07BBD50C
:1062E800B7F8221824234B431233642193FBF1F1AE
:1062F8000AE184F8E138404B3B4F1B689B07ABD55C
:10630800B7F80C380A21FEE084F8E1383A4B364FEA
:106318001B681905A0D5D7F81418F5E084F8E138FA
:10632800D4F81C38304F5A0796D57969ECE084F8D0
:10633800E138314B2C4F1B681B058DD5D7F8181841
:10634800E2E0D4F81C18284A84F8E1388F0683D58F
:1063580092F8201888077FF57FAFD90712D5D2F8B1
:106368002C3883EAE371002BA1EBE37101EB5101B7
:106378004FF01902B1FBF2F1ACBF41F0004141F01E
:1063880040410FE0D2F8283883EAE371A1EBE371CA
:10639800002B01EB51014FF01902B1FBF2F1B8BF2C
:1063A80041F080414FF400608CE084F8E138D4F883
:1063B8001C380D4F5B077FF54FAF3969A4E0B4F97E
:1063C800181084F8E138642359437BE084F8E138F5
:1063D800B4F90C1003E0B4F90E1084F8E1382C235A
:1063E80091FBF3F16EE000BFB8110020A48801080A
:1063F80008300020AAAA0108E42F002084F8E13818
:1064080094F8E238644A0133DBB2032B88BF0123D6
:1064180082F8E23894F8E21842F2107359435F4B5D
:106428001B78D80748BF01319A0748BF02315F0778
:10643800B4F8E43848BF0431D80748BF0A319A078E
:1064480048BF14311F0648BF2831D80548BF283136
:106458005A0748BF64311F0748BFC831980548BF6D
:1064680001F5C8719A0648BF01F57A71DF0648BF81
:1064780001F5FA61580648BF01F57A614FF480606A
:1064880002F01CFB444B002283F8E028E4E6D4F831
:106498001C18DFF8048184F8E13811F0200717D0C0
:1064A80098F8202812F0020F14BF4FF47A710021D7
:1064B80012F0010F14BF4FF4FA6300230B4494F851
:1064C8002618194402F0FAFA002384F8E038C3E6E3
:1064D800334B1B6819067FF5BFAE394602F0EEFA5A
:1064E80088F8E078B8E684F8E138D4F81C382A4F00
:1064F8009A067FF5B1AE97F820389B077FF5ACAECA
:10650800B7F824386421594302F0D8FA002387F8F1
:10651800E038A1E684F8E1383AE0BB7823B1C5F861
:10652800A06887F80280A1E5D5F8A038F31AB3F57A
:106538007A6FFFF49BAD0123D5F8A408BB7008F06F
:1065480064FF0746D5F8A40808F05FFF7F067FF4CC
:106558008DAD8A2802D08E280DD087E5D5F81C3855
:1065680098067FF583AD95F89E38002B7FF47EADB5
:1065780005F66D0306E095F89E38002B7FF476AD9E
:1065880005F63803C5F8A8382D2385F8AC386DE52D
:1065980006B0BDE8F08700BFB81100201F34002006
:1065A800E42F0020F8B504460E461746002520467D
:1065B80020210FF0ECFD0446D0B1013420460FF045
:1065C8004BFEB0F5617F05DB40F634039842A8BF67
:1065D800184601E04FF46170A0F56170192390FB33
:1065E800F3F00DB9307000E070703B7801333B7008
:1065F8000DB90125DBE72046F8BD30B505460C4648
:106608001346294622460248BDE8304001F01CB92D
:106618009CAB01087FB504780646E4B9354B1B6886
:1066280003EB8403192193F87B0093F87C6093F8BB
:10663800792093F87A304FF4617511FB005011FB03
:106648000651009001912C482146013401F0FCF8D4
:10665800142CE3D14BE00FF0FFFD1328054641DC75
:10666800244B701C1C68202100238DF80F300FF07C
:106678008EFD1E35064670B1013630460FF0ECFD32
:106688001A289FBF04EB850358709DF80F3001331B
:1066980098BF8DF80F30304620210FF078FD064660
:1066A80070B1013630460FF0D7FD0D289FBF04EBBF
:1066B800850398709DF80F30013398BF8DF80F301F
:1066C80004EB85043046E11C0DF10F02FFF76AFF69
:1066D8009DF80F30042B0AD0601C002104220FF013
:1066E80020FD04E0054800211322FFF786FF04B0CF
:1066F80070BD00BF30110020BBAB0108D0AB010852
:1067080001480BF071BC00BFD6AB01082DE9F0437E
:1067180004788FB00546002C59D17B4B00211422F8
:1067280009A807AED3F800800FF0FBFC072230461B
:1067380000210FF0F6FC05A80023A700059308EB3D
:10674800070583801A467149B5F802E031F813C08D
:106758001CEA0E0F0AD00DF1380C0E3102F1010EB1
:106768006244595C02F81C1C5FFA8EF20133072B55
:10677800E9D100210B46664AB5F802E011F802C0DB
:106788001CEA0E0F0AD00DF1380C063203F1010E87
:1067980063448A5C03F8242C5FFA8EF301310629DE
:1067A800E9D118F807305B498DE841006A78029210
:1067B80009A81A0903F00F0301F031F821465648D9
:1067C80009AA013401F040F8202CA6D198E00FF076
:1067D80043FD1F28044600F3868028462021E4B2A2
:1067E8000FF0D5FC1F2C02D9FFF78AFF88E0464B33
:1067F8001B6803EB8404451C0021204604220FF08B
:1068080090FC0027454B09AE304600210A2217F8B4
:1068180003905FFA87F80FF084FC002315F8012B2A
:1068280032B10A2B04D04A4502D0F2540133F5E7BD
:106838004A455ED108F1FF33032B09D8DFE803F09E
:106848001005023F0DF1230134E00DF123011EE094
:1068580030460FF001FD2378C0B243EA001006E08D
:1068680030460FF0F9FC237800F00F001843207031
:1068780031E00133062B0AD0244800F11B069E5D47
:106888009642F6D103445A7D63881343638011F816
:10689800012F02B30023EFE70133072B0AD01B486F
:1068A80000F10E069E5D9642F6D130F813206388FB
:1068B8001343638011F8012F6AB10023EFE73046D4
:1068C8000FF0CAFC0F2804DC30460FF0C5FC6070DE
:1068D80001E0002363700137052F93D1012409F0EB
:1068E80039FC6CB980E70E4800211F22FFF785FEAE
:1068F80006E02046002104220FF013FC0024EEE7F6
:106908000FB0BDE8F08300BFA01A0020B8880108C6
:10691800CD880108E4AB0108F3AB0108D988010868
:10692800D0AB0108F8B50478064674B9304DB5F80F
:10693800C221B5F8C4312F482146013400F084FF44
:10694800042C05F10405F2D1F8BD2B490FF0F2FB38
:10695800A8B9274B4FF47A714FF4FA62A3F8C21121
:10696800A3F8C421A3F8C611A3F8C821A3F8CA1133
:10697800A3F8CC21A3F8CE11A3F8D021F8BD304656
:106988000FF06AFC032805462BD8304620210FF06B
:10699800FEFB044630B1013420460FF05DFC0126B1
:1069A800074600E00646204620210FF0F0FB10B90C
:1069B800BDE8F840A4E601300FF04EFC012EF7D1F7
:1069C800A7F2EE2240F2DC539A42F1D8A0F2EE226E
:1069D8009A42EDD8064B6E3503EB85035F819881AB
:1069E800F8BD064800210322BDE8F84005E600BFCF
:1069F800E0110020FFAB010812AC010810BC01082F
:106A08002DE9FF4104780546002C39D17348744DAF
:106A18000BF0EAFAD5ED047AF5EE407AF1EE10FAC9
:106A280000F0D88021466F4800F00EFF95ED040A6B
:106A3800684600F089FD01466B4800F005FF95EDBA
:106A4800050A684600F080FD0146674800F0FCFE34
:106A580095ED060A684600F077FD0146624800F0A9
:106A6800F3FE95ED070A684600F06EFD0134014615
:106A78005E4800F0E9FE0C2C05F11005CAD1A9E02A
:106A88005B4905220FF09AFB40B9554B03F1C00250
:106A9800002143F8101F9342FAD19BE0284655493C
:106AA80004220FF08BFB04462846002C40D12021FD
:106AB8000FF06DFB002800F08D80451C28460FF074
:106AC80074FB07464C4B53F824601EB94B480BF037
:106AD8008BFA7FE028463146FAB20FF06FFB01349B
:106AE8000028EFD13E4B03F1C0029E46002143F837
:106AF800101F9342FAD1424B03EBC4029846D2F8D6
:106B080004C0BCF1000F04D131463E4800F09CFEA1
:106B180057E0002718F834309F42F5DA3B010EEBB6
:106B2800030563440FCB103585E80F000137F1E703
:106B38000FF092FB0B28064647DC284620210FF071
:106B480026FB054650B10135284600F073FC244B5E
:106B580003EB061383ED040A012400E004462846EB
:106B680020210FF014FB054648B10135284600F0F6
:106B780061FC1B4B03EB061383ED050A0134284621
:106B880020210FF004FB054648B10135284600F0E6
:106B980051FC134B03EB061383ED060A0134284618
:106BA80020210FF0F4FA10B9FFF7AAFD12E0013026
:106BB80000F040FC0A4B032C03EB061686ED070A8F
:106BC800F2D11148FFF71CFF04E0104801210C2204
:106BD800FFF713FD04B0BDE8F08100BF18AC010851
:106BE800E011002033AC010839AC010887B901086D
:106BF80012AC01083DAC0108B892010842AC01088A
:106C0800CCAA010851AC01086FA90108D0AB010852
:106C1800F0B5047887B006461CBB514B19680623AB
:106C280003FB0411192091F8CA5091F8CB7091F820
:106C3800CE2091F8C9304FF4617610FB056510FB42
:106C480007600095019091F8CC000290C831454842
:106C5800497903912146013400F0F6FD0C2CDCD172
:106C68007CE00FF0F9FA0B28044672DC3C4B701CF0
:106C78001D68202100238DF817300FF088FA06468A
:106C880080B1013630460FF0E7FA03289FBF06238C
:106C980003FB045383F8CE009DF817309CBF0133E3
:106CA8008DF81730304620210FF071FA074680B171
:106CB800013738460FF0D0FA0D289FBF062303FB93
:106CC800045383F8C9009DF817309CBF01338DF831
:106CD800173006266643A9193846CA310DF117023E
:106CE800FFF760FC20210FF052FA074670B1013718
:106CF80038460FF0B1FA14289FBF9DF8173076195F
:106D0800013386F8CC0098BF8DF81730384620211B
:106D18000FF03DFA78B101300FF09EFA0D289FBFB1
:106D2800062303FB045383F8CD009DF817309CBF5E
:106D380001338DF817309DF81730062B0ED0062238
:106D480002FB04500021C9300FF0EBF9FFF7D8FC23
:106D580004E0054800210B22FFF74FFC07B0F0BD07
:106D6800301100205DAC0108D0AB01082DE9F347D4
:106D7800047806464CB9204601A90AF029FF0134D7
:106D8800FFF7F4FF122CF6D180E00FF065FAC5B2D8
:106D9800112D76D83F4C05F1CC0704EB4703701C46
:106DA800202193F806803C4E0FF0F1F9034630B9E4
:106DB800A8F10202D2F1000848EB020848E006F107
:106DC800260800F1010A597840460FF0E0F968B149
:106DD800032D8CBF03230023C8EB0000334453FA70
:106DE80080F090F82A90B9F1030F02D1FFF788FCE0
:106DF8004CE0A9F10203D3F1000850464FF02001FE
:106E080048EB03080FF0C3F9D8B1B8F1000FEDD083
:106E180001300FF021FA40F2ED2380B2984205DDEF
:106E280040F6CA039842A8BF184601E040F2EE2097
:106E380004EB4703A0F2EE20192290FBF2F0D87180
:106E480002E0B8F1000FD1D104EB470383F80690B4
:106E580004EB4704A3791E4496F82620B8F1000FE6
:106E68000AD0E3790D48294640F2EE24192505FB9E
:106E7800034300F0E9FC09E02946094800F0E4FC76
:106E880004E0084800211122FFF7B7FB02B0BDE873
:106E9800F08700BFE0110020B88801087DAC010828
:106EA8008FAC010810BC010807B50123ADF8041028
:106EB80001A98DF806208DF8073007F0C9FD03B049
:106EC8005DF804FB2DE9F843054672B64FF090468D
:106ED8004FF480614FF40079318530460422A6F8DA
:106EE8002890FFF7E1FF304601224946FFF7DCFF13
:106EF8002B4850F8354000EBC5002368426801254F
:106F0800570005FA07F848EA030395402360A5618E
:106F1800C6F818904FF090431B8A5B05FAD4236893
:106F280048EA030323604FF090434FF40072A9B27C
:106F380021851A850822C3F8182440F605534FF016
:106F48009040028A560512D4013BF8D122680323E7
:106F5800BB4022EA030323604FF400710222FFF7CB
:106F6800A3FF62B63220BDE8F84308F072B9A56104
:106F780020460422FFF798FF4FF090431A8A5205E3
:106F8800CDD5228A92B21542064A4FF400704FF0CE
:106F9800080115BF9861188591611185ECE700BF5C
:106FA800C0AC01080004004810B50446204608F0AB
:106FB80026FA18B90A2008F04CF9F7E710BD0022A4
:106FC80007490C2303FB02135968814204D10022AC
:106FD800C2621A725A6070470132052AF0D17047AE
:106FE800982800202DE9F74389469DF82880114606
:106FF8001A469DF82C30064600250C2068431D4F84
:10700800C419C057B04202D1207A20B12BE0013513
:10701800052DF2D127E0022E0FD005DC56B1012E46
:1070280021D1009314480AE01E2E0DD01F2E1AD12C
:10703800012009E00093114801E0114800934346FC
:1070480004F034FC044605E004F00CF9414604461B
:1070580008F0D2F94CB10C2303FB0575267185F8AD
:1070680008906C6001E0002000E0204603B0BDE815
:10707800F08300BF982800200044004000380140F9
:107088000048004010B5084B1968002201EBC20304
:1070980093F90240844201D1981C10BD0132052A9F
:1070A800F4D1002010BD00BF94280020F0B502786C
:1070B80087B08AB94A4C04F1280694F8F2210023D3
:1070C8004849595650B281426ED00C333C2BF7D107
:1070D8000834B442F1D181E0002204920592451CA3
:1070E8000FF0BAF8C4B260B2FFF7CCFF074618B188
:1070F8008DF81040012400E00446284620210FF0B6
:1071080046F8054638B1013528460FF0A5F8013490
:10711800ADF81200E4B20026284620210FF037F817
:10712800B0B3451C28460FF097F800222E4951F8B5
:10713800223083425FFA82FE04D00132082AF5D158
:10714800002300E0734651F82320824220D1022E0A
:107158000FD0032E12D05A1E012ED2B204D0042A08
:1071680013D88DF814300EE0042A0ED88DF8153097
:1071780009E0052B09D88DF8173004E09A1E052A76
:1071880003D88DF816300134E4B20136042EC3D189
:10719800052C04D807B0BDE8F040FFF7B1BA04AB3E
:1071A80003CB3860796019E094F8F7010E4B94F836
:1071B800F65153F82000B4F8F421009094F8F9013E
:1071C80053F82000019094F8F80153F82000029039
:1071D80053F82530054800F037FB79E707B0F0BDD4
:1071E800E011002098280020949001089EAC010826
:1071F80038B1438811EA030003D08B420CBF012049
:107208000220704730B50A4B0A491C680A79042ADB
:107218000AD8134604EBC303551CEAB29D882842DA
:10722800F5D00A71981C30BD0A71002030BD00BF2E
:1072380094280020A01A0020014B00221A71E1E7CF
:10724800A01A00202DE9F047877890F803C0214D57
:10725800BBB2C7F1640E03EB83065C42C3F178004E
:107268005FFA8EFE7600CCF16408A4B280B2A3B2B5
:107278000FFA83F9B9F1000F05DC002B14BFBA46E9
:107288004FF0010A00E0F24613FB03F303FB0CF294
:107298001AFB0AF392FBF3F3434403FB09F30A22B4
:1072A80093FBF2F333449BB225F8023FB1F8009008
:1072B8004A880A34C9EB020AA4B21AB202FB0AF2DB
:1072C8004FF47A73844292FBF3F34B442B80CED174
:1072D800BDE8F087A41A0020F0B50124B0FBF4F54E
:1072E8008D4201D34C43F9E70026D4B1B0FBF4F545
:1072F80004FB1500B4FBF1F41EB9002D01DC002CD1
:10730800F3D1092D03F1010EEFB204DD002A14BFF9
:107318003725572500E030253D441D70013673465A
:10732800E3E71C70F0BDF0B50124B0FBF4F58D4225
:1073380001D34C43F9E70026D4B1B0FBF4F504FBC4
:107348001500B4FBF1F41EB9002D01DC002CF3D1BB
:10735800092D03F1010EEFB204DD002A14BF372511
:10736800572500E030253D441D7001367346E3E79C
:107378001C70F0BD03685A1C0260197070472DE933
:10738800F843089E002B07468846144614BF4FF062
:1073980030094FF02009334613F8012B0AB9254666
:1073A80003E0002CFBDD013CF6E7002D04DD384648
:1073B8004946C047013DF8E724EAE4743546A01B76
:1073C800284415F8011B11B13846C047F7E7BDE856
:1073D800F883024B186808F01EB800BFD8100020C8
:1073E80090ED017A07EE901AB5EE407AF1EE10FAB8
:1073F80001BFF8EEE77A9FED0E7A67EE877AB7EE6F
:10740800007A04BFC7EE277AC0ED017A90ED017AC1
:10741800D0ED007A30EE877A30EE670AC0EE870A40
:10742800E0EE807AB0EE670AC0ED007A704700BFE0
:10743800DB0FC94010B50278202A034600F101008D
:10744800F9D0092AF7D02D2A03D10346BFEE000A46
:1074580004E02B2A08BF0346B7EE000ADFED387AAE
:107468001A46134612F8010BA0F13001CCB2092CD0
:107478000AD807EE101AB8EEC77AF2EE046AA7EE39
:10748800A67AF0EE477AECE72E2816D1F2EE046AD7
:107498001146B0EE666A0B4611F8012B303AD0B2AD
:1074A80009280AD807EE102AB8EEC77A87EE267A96
:1074B80066EE866A77EE877AEDE71A7802F0DF02E1
:1074C800452A35D15A782D2A02D10233012004E009
:1074D8002B2A14BF013302330020013B002213F88A
:1074E800011F3039CCB2092C03D80A2404FB02123C
:1074F800F5E7B2F59A7F28BF4FF49A721346B7EEB4
:10750800007A072B05D9DFED0F6A083B27EE267AAC
:10751800F7E702F007032BB1F2EE046A27EE267AAA
:10752800013BF8E7F0EE476A20B1C7EE877A03E03F
:10753800F7EE006A67EEA67A20EE270A10BD00BFB4
:107548000000000020BCBE4C30B52DED028B87B08A
:10755800B0EE408A0C220021054603A80EF0E1FD9A
:10756800B5EEC08ADFED2A7AF1EE10FACCBF38EE1C
:10757800278A38EE678ADFED277A28EE278A694658
:10758800FDEEC87A17EE904A84EAE470A0EBE47046
:107598000AF01EFB002CACBF20232D2368468DF873
:1075A8000C300EF002FE012807D130238DF80D3083
:1075B8008DF80E308DF80F300CE0022805D13023FD
:1075C8008DF80D308DF80E3004E0032804BF302309
:1075D8008DF80D30694603A80EF0CAFD03A80EF019
:1075E800E4FD0338C4B2224603A928460EF00AFE79
:1075F80000232B55284608490EF0BAFD03AB284650
:1076080019190EF0B5FD284607B0BDEC028B30BD48
:107618006F12033A00007A4400AD010870B50646BF
:1076280015460846B6FBF2F414B12046FFF7F6FFFC
:1076380005FB1464024B1B5D00F8013B70BD00BFE5
:1076480002AD01082DE9F04F814689B08A461646F9
:107658001C4600253178002900F0DD80252902D05C
:107668000136484675E07278302A08BFB278A2F130
:10767800300319BFB71C4FF0000BF71C4FF0010B7C
:10768800092B4FF0000819D8A2F13003D9B2092903
:1076980005D80A2202FB083817F8012BF4E7A2F1F3
:1076A8006103052B02D8A2F1570305E0A2F14103BB
:1076B800052B03D8A2F137030A2BEADD6C2A31D156
:1076C8003A78642A07F1010600F083800BD8252A4E
:1076D8003DD003D8002A00F09E80BBE7582A0CD082
:1076E800632A19D0B6E7732A22D002D86E2A37D077
:1076F800B0E7752A5CD0782AACD1271D2068A2F1A2
:10770800580462424FF01001624155E02CD9582AC2
:1077180032D0632A2AD13E4648462178271DD047D1
:1077280001350FE0642A64D00ED9732A14D13E467D
:10773800236800934846514642460023FFF71FFE40
:10774800271D05443C4685E7252ADFD13E464846A5
:107758002521D04701357DE70AD86E2A06D13E4655
:10776800236804341D6075E7002A54D03E4671E74B
:10777800752A26D0782AF9D1A2F1580304F1040C0D
:107788005A422068CDF80CC04FF010015A4105ABA1
:10779800FFF7A2FDDDF80CC03E46644605AB00933A
:1077A8004846514642465B46FFF7E9FD054451E726
:1077B8002068271D0A21002205ABFFF7B4FD3C46CF
:1077C800ECE704F1040CCDF80CC020680A21002273
:1077D800DDE72068002804F1040708DA2D238DF876
:1077E800143040420DF115030A210022E5E705ABEC
:1077F800FAE72068002804F1040C0ADA2D238DF832
:10780800143040420DF11503CDF80CC00A210022B6
:10781800BEE705ABF8E7284609B0BDE8F08F0EB41F
:107828000FB505AB019053F8042B0649039301A843
:10783800FFF708FF019B00221A7004B05DF804EB03
:1078480003B070477D7300080FB413B50B4904AB40
:1078580008680B4953F8042B09680193FFF7F2FEF7
:107868000446084B186807F0CAFD0028F9D02046DE
:1078780002B0BDE8104004B0704700BF040100200A
:1078880000010020D810002080EAE073A3EBE07329
:107898008B4206DB002801DD401A704702D00844FD
:1078A800704700207047FDEEC07A17EE903A2033FB
:1078B800402B43D8DFED237AB4EEE70AF1EE10FA55
:1078C80004DDDFED217A30EE670AF3E7DFED1F7A9A
:1078D800B4EEE70AF1EE10FA04D5DFED1B7A30EECC
:1078E800270AF3E7DFED1A7AB4EEE70AF1EE10FAA9
:1078F80004DD30EE670A37EEC00A0AE09FED157A1C
:10790800B4EEC70AF1EE10FA44BF30EE270A37EE9C
:10791800400A60EE007ADFED106A9FED107AA7EE5C
:10792800A67ADFED0F6AE7EE876A9FED0E7AA7EE7B
:10793800A67A20EE276AA6EE070A70479FED0A0A84
:10794800704700BFDB0F4940DB0FC940DB0F49C060
:10795800DB0FC93FDB0FC9BF9A7C2E36FAAF4FB990
:107968003587083CA4AA2ABE00000000DFED027A91
:1079780030EE270A97E700BFDB0FC93F38B52DED7A
:10798800068B90ED008AB0EE480A0C460546FFF7D4
:10799800EDFFB0EE40AAB0EE480AFFF784FFD5ED40
:1079A800018AB0EE409AB0EE680AFFF7DFFFB0EE4A
:1079B800408AB0EE680AFFF776FFD5ED02AAF0EE2E
:1079C800408AB0EE6A0AFFF7D1FFF0EE409AB0EEB7
:1079D8006A0AFFF768FF60EE0A6A69EE297AF0EE34
:1079E800665AE7EEA85A29EE8A6A29EE007A69EE05
:1079F800889A29EE489A28EE400A28EE0A8AC4EDA9
:107A0800035AF0EE465AE7EE685AE6EEA87AA6EE72
:107A1800687AC4ED009AC4ED028A84ED059A84ED73
:107A2800088ABDEC068B84ED010AC4ED045A84ED86
:107A3800067AC4ED077A38BD10B52DED048B8AB0EF
:107A480090ED009AD0ED028A90ED018A044608462E
:107A580001A9FFF793FFDDED047A9DED017A68EE49
:107A6800277AE9EE077A9DED077AE8EE877A9DEDA9
:107A7800027AC4ED007ADDED057A68EE277AE9EE40
:107A8800077A9DED087AE8EE877AC4ED017ADDED94
:107A9800067A28EE278ADDED037AA9EE278ADDED3E
:107AA800097AA8EEA78A84ED028A0AB0BDEC048B95
:107AB80010BD074B1A8822EA0000904210B51880C2
:107AC8001C4602D0012007F027FC208810BD00BF0B
:107AD8009C1A0020064B1A881043904210B5188053
:107AE8001C4602D0012007F017FC208810BD00BFFB
:107AF8009C1A0020024A936823EA000090607047AD
:107B0800E0110020024A936818439060704700BF54
:107B1800E011002008B5104B1A780023D9B2914221
:107B280007D20E4951F82310096800200860013374
:107B3800F4E7322007F08DFB094B1B685A0309D57F
:107B4800084B9B685B0305D440F2DC50BDE8084055
:107B580007F07FBB08BD00BFD42B0020A42B00205A
:107B6800E42F0020E01100202DE9F3410AF0AAFFDC
:107B7800454A6A2313704FF4FC635380BE23137184
:107B8800EF2382F8DD37002382F8DE3719461646E0
:107B9800F25C0133B3F5FC6F81EA0201F8D13A4B8C
:107BA80083F8DE17394B1A69120604D5384A5A6029
:107BB80002F188325A6004270020013F17F0FF07BE
:107BC8004FD0324B3422DA60002444B1002356F8F7
:107BD8000480019304F0C2F90428EED117E004F000
:107BE800BDF90428E9D1294D2B6943F002032B6123
:107BF800284B6B612B6943F040032B6104F0AEF90D
:107C08002B69042823F002032B61DFD0D5E71F4D31
:107C18002B6943F001032B6104F1006303F57E3304
:107C28001FFA88F21A8004F099F9042810D11A4B27
:107C380023440193019B4FEA1848A3F8008004F0FD
:107C48008DF92B69042823F001032B6105D0B4E7D3
:107C58002B6923F001032B61AFE70434B4F5FC6F03
:107C6800B3D10A4A1369042843F08003136102D18F
:107C780009F027F810B9052007F066FB0AF00CFF99
:107C880002B0BDE8F08100BFE011002000200240F2
:107C98002301674500F8030802F8030810B50E4CE5
:107CA800206807F019FA2068047A002202FB02F320
:107CB800193B634303F6C4135343192193FBF1F3B0
:107CC800064921F812300132072AEFD10449BDE8EC
:107CD8001040FFF7B7BA00BF58110020A8100020C5
:107CE800201300202DE9F04108F0EBFF10B9042023
:107CF80007F02AFBAF4CB04D0AF0E4FEAF494FF451
:107D0800FC6220460EF002FA94F8B437022B84BFC6
:107D1800002384F8B43794F8B4274FF4CC7101FBEE
:107D280002F3E018234400F53B70286093F8400301
:107D380003F54E73022801FB024284BF002018722B
:107D480092F840339E4A13700C2202FB03439D4A6B
:107D580003F2B6731360A26846F2090313401BB915
:107D68004FF40050FFF7CEFEA368D80703D54FF4B1
:107D78000050FFF7BFFEA368590409D50820FFF794
:107D8800B9FE4FF40050FFF7B5FE0120FFF7B2FE31
:107D9800A3681A0706D54FF40050FFF7ABFE012081
:107DA800FFF7A8FEA3689B0402D54020FFF7A2FEB8
:107DB800012284F81D2294F8DC217E4B2AB193F825
:107DC800E02112B1002283F8E0217F4B7F4E1E6034
:107DD8004FF0000C674604EB0C03B3F8F4E14FEAEC
:107DE8005E0101F077314FEA9E0303F03333C1EBB4
:107DF8000E00C11A4FEADE0303F01133CB1A03EB6E
:107E080023131EF0010803F00F324FF0FF0392FB1B
:107E1800F3F3C3EB032318BF0137A2EB030318BF27
:107E2800FFB2012B0ADD022B40F0C180B8F1000F30
:107E380000F0BD801EF0BC0F00F0B9800CF1080CFA
:107E4800BCF1280FC7D1013F012F00F2B080FFF726
:107E580025FF302200215E485E4F0EF062F95E4B2E
:107E6800D5F800801F605D4B002108F17900C3F848
:107E7800008007F071F95A4B80F001001870594BD7
:107E880007F126021A60584B07F1DC021A6098F8CD
:107E9800000007F0FDFC2868544B00F5C5721A6015
:107EA80002F076FB524B94F8D401DFED526A07F1E9
:107EB80094021A606421504BC82211FB00225A60B8
:107EC80000229A60DA601A615A619A61DA6183F86D
:107ED800202083F82120494B07F12C021A602B68D7
:107EE800474A93ED187A03F219111160454A03F2D3
:107EF80089111160444A07F108011160434A17606B
:107F0800434A07F1A0011160424A07F1AA01116032
:107F1800414967EE266A0E60B4F86211B6EE007A3F
:107F280007EE901A87EE267AB4F86411101DF8EE61
:107F3800677AC2ED027A07EE901A93F85C10117115
:107F480093F87810517194F8DF111174F8EE677A8C
:107F5800B3F81611C2ED037A07EE901A2F4908609C
:107F680053612F4A03F1640111602E4A2E4982EDB4
:107F7800007AF8EEE77A9FED2D7A2D4A0B60C7EE6E
:107F8800277A2C499FED2C7A67EE877AC2ED007A22
:107F980003F168020A60294903F211130B60284BA8
:107FA8001F60284BBDE8F0411A600AF075BD03F068
:107FB800A9FF4CE7E01100203011002000F8030869
:107FC8004830002058110020B833002066130020E4
:107FD800DC0F0020201300201010002014100020B7
:107FE80018000020E00700200406002020100020D0
:107FF800F0330020DB0F4940C4330020380800204C
:10800800082A00204C0A0020F02C0020F42C002024
:1080180060090020C01A0020240A002068080020F7
:10802800A00800209C080020A80700200000614448
:108038005C0900209C0700204C3D0F444C0900209F
:10804800540900209406002008B5FFF78DFDFFF7BE
:1080580049FE0120BDE8084007F05EB9344B354AB7
:108068001B68126810B51A60334A11685960516864
:108078009268DA60314A99601168196151689268AA
:108088009A612F4A59611168D961516892685A6298
:108098002C4A196211881985518859859188D28886
:1080A800DA85294A998511881986518859869288CE
:1080B8009A86264A1188D98651881987194692883E
:1080C80021F83A2F224A10780022824206DA214CFF
:1080D80034F8124021F8024F0132F6E71E4A12889E
:1080E800A3F864201D4A1288A3F866201C4A118848
:1080F800A3F86C1051889288A3F87020194AA3F845
:108108006E1012689A66184A3B21126892FBF1F2C7
:10811800B2F5967FC8BF4FF0FF325A67134A1288EC
:10812800A3F87820124A5289A3F85E2010BD00BF38
:10813800B030002000340020542B0020602B002099
:108148006C2B0020D811002014110020C21100202F
:10815800D42B00203411002018290020CC10002036
:108168001A110020CC110020040000205411002016
:10817800201100202DE9F8430E4B93E880030546B3
:108188000E460024B44213DA7B1933F9140008EBC5
:10819800050333F9142009EB050333F914301344AC
:1081A800022293FBF2F3C01A09F06EF90134E9E7F1
:1081B800BDE8F883B030002070B5472008F09EFB7A
:1081C800174B1B681B0307D5164B174A5B681068CB
:1081D8001B68C01A09F048F9144E154C154D307833
:1081E80009F042F923682868C01A09F04DF9636854
:1081F8006868C01A09F048F90F4B188809F034F973
:108208000E4B188809F030F90D4B188809F02CF935
:10821800337823742B68A3606B68E36070BD00BF7C
:1082280034320020B030002000340020DE19002055
:108238009C300020E0190020DC190020DA19002009
:108248005C1100207FB5264C264E274D2749284A29
:10825800284B20B128480088B0F5805F31D230889B
:10826800ADF8040028781E4D91F8201012788DF88A
:1082780006008DF807108DF808201B788DF8093056
:1082880001A8294606220DF031FF30B30198BDF848
:1082980008302860AB80532008F030FB208809F0B4
:1082A800E3F8A07809F0E0F8E378019323790293E2
:1082B80001A86379039309F03BF80F4B00221A8059
:1082C8000BE03088208091F82010287812781B78ED
:1082D800A070E17022716371DDE704B070BD00BF6A
:1082E800D81A00209C1A0020D8190020C433002076
:1082F800430F0020A80F002054320020A0F17D0376
:10830800012B70B504460D460A4E05D830687D210C
:1083180007F081F884F020043068214607F07BF8E4
:1083280035B12B881C4404EB142404F0FF042C8082
:1083380070BD00BF8C1A00200A4A138801331380CD
:10834800094A136801331360084A138801339BB242
:10835800202B01BF00231380054A138808BF01336F
:1083680013807047543200203C32002040320020F5
:108378004232002038B53A4B1B78083B012B0546A2
:108388000C466BD8452008F0B9FA284608F0B6FA2A
:108398000C2D23D004D80A2D0AD014D835B138BDF5
:1083A8000E2D4BD02ED3FF2D50D038BD206849E07C
:1083B800207808F0A3FA62796378002A14BF802035
:1083C8000020184300E0207808F098FAA07808F018
:1083D80095FAE07808F092FA20793BE0B4F90000C9
:1083E80009F037F8A07808F089FAE07808F086FAFA
:1083F800B4F9040009F02DF8B4F90600BDE83840D6
:1084080009F027B8637820788BB180F0800008F0F5
:1084180075FAA468E0B208F071FAC4F3072008F00E
:108428006DFAC4F3074008F069FA200E12E008F06C
:1084380065FA6068BDE8384009F026B8206809F098
:1084480013F86068BDE8384009F00EB8054809F02F
:108458001FF80020BDE8384008F050BA38BD00BF0A
:108468008C30002027AD01082DE9F04FBE4BBF4FDF
:108478001A888BB00193002A40F0A980B7F8DA0770
:10848800BB4E42F20103C21A50425041FFF7DAFED6
:10849800FFF7E4FD3468492008F030FAB54B25466B
:1084A800186808F0E1FF55F8040B08F0DDFF2846CE
:1084B80003F0DAFC04F1100003F0D6FC04F11C0907
:1084C8004FF01008AC4D01232A6803FA08F3134251
:1084D80003D0D9F8000008F0D7FF08F10108B8F177
:1084E800130F09F10409EDD104F1280003F0ACFCE5
:1084F800B7F84031B4F92E00C01A08F0B5FF2B6860
:10850800DB0408D59D4BB4F864001B88181AC0F327
:108518000D0008F0A9FF2B68980403D5B4F866008D
:1085280008F0A2FF2B68590503D504F16C0003F08D
:108538008BFC2B681A0502D5A06E08F0A5FF2B68E6
:108548005B0402D5606F08F09FFF2B68180403D501
:10855800B4F8780008F088FF04F13000A04603F072
:1085680073FC04F1360003F06FFCB7F8403138F9BA
:108578003C0FC01A08F078FF0127814B1B789F42F7
:1085880008DA38F9020FB4F93C30C01A08F07CFF59
:108598000137F2E72B68990505D5B4F95E00A0F21A
:1085A800DC5008F071FF326876487260B260121AC7
:1085B8009110754A4A43531C032293FBF2F202EBD3
:1085C80042029A1A7C2303FB02033360D6E16F4B05
:1085D8006F4A1B6811688B4206D00AA9002041F82F
:1085E800203D1360FFF7C6FE019B97F8DA171B883A
:1085F80097F8DB070B44013BB3FBF0F200FB1233A7
:108608008B4280F086815A4F0120FFF71BFEFFF74F
:1086180025FD50203E687D6808F070F9BA683B680F
:1086280010681B687A6803441068A3EB400008F0E0
:108638002BFF6A6873689B1A0293AA68B3689B1A2F
:108648000393EA68F36802A89B1A049303F00CFCEE
:108658002A6933699B1A02936A6973699B1A03939F
:10866800B369AA6902A89B1A049308F061FE06F18F
:108678001C0B05F11C0810243F4901220B68A2407D
:108688001A428A4606D0DBF80000D8F80030C01A33
:1086980008F0FAFE0134132C0BF1040B08F104085E
:1086A800EAD106F1260005F12601002331F9024F2F
:1086B80030F9022F121B02AC44F823200133042B9B
:1086C800F4D103214FF000094FEA89035FFA83F9D7
:1086D80002AB53F821206AB102F108000F2802D832
:1086E80049F0010906E08032FF2A94BF49F00209E7
:1086F80049F0030911F1FF31E6D2484608F0FEF8C7
:1087080000240DF1080BA04609F00302022A16D036
:10871800032A1DD0012A4ED1B8F1000F05D1DBF88C
:1087280000402401E4B2904645E0DBF8000000F088
:108738000F00204308F0E2F84FF000083BE0B8F1E2
:10874800000F0CD0DBF80000C0F3031020432CE02E
:10875800B8F1000F1ED19BF8010008F0CFF89BF884
:10876800000008F0CBF826E040320020E01100209D
:10877800B03000203C32002034320020303200205B
:10878800D42B0020BC300020DF7BEFBD4832002016
:1087980044320020DBF80000C0F30330204308F027
:1087A800ADF8DBF80000C0F3071008F0A7F8DBF815
:1087B80000402401E4B20BF1040B06AB9B454FEAE1
:1087C8009909A1D1B8F1010F02D1204608F096F815
:1087D800DAF8003013F480541FBFB6F86420B5F8F7
:1087E8006410521A029218BF01249A040AD50AAAE0
:1087F80002EB8401B5F86600B6F86620121A41F853
:10880800202C0134580513D502AA02EB840C06F17A
:108818006A0E05F16A0000223EF9021F30F9028F44
:10882800C8EB01014CF822100132032AF4D10334B9
:10883800190508D50AAA02EB8400A96EB26E521A6D
:1088480040F8202C01345A0408D50AAA02EB840007
:10885800696F726F521A40F8202C013418040BD536
:108868000AAB03EB8402B5F87810B6F878305B1AD7
:1088780042F8203C013400E0FCB1012C03D10298FD
:1088880008F002FE19E0631E002002AA400052F818
:108898002320C0B20AB140F00100013BF5D508F031
:1088A8002DF84FF0000802AB53F8280008B108F083
:1088B800EBFD08F10108A045F5DB30200321FFF7A7
:1088C80059FC36200321FFF755FC2F4B3C20197823
:1088D800FFF750FCDAF80030990506D5B6F95E00C6
:1088E800B5F95E30C01A08F0CFFD3A6827487B68B2
:1088F8007A60121A9110264ABB604A43531C03221D
:1089080093FBF2F202EB42029A1A7C2303FB020366
:108918003B60204B1B681A0630D51F4C1F4D226840
:108928002B689A420BD162686B689A4207D1019B07
:108938001B88102B11D11A4B1B885B060DD14820C0
:1089480007F0DCFF206808F09FFD606808F09CFDD8
:1089580023682B6063686B600EE0124A0F4B117836
:108968002A7C914208D1104A99681068884203D13C
:108978005268DB689A4201D0FFF71EFC08F0C6FC7B
:108988000BB0BDE8F08F00BFD42B0020BC30002016
:10899800DF7BEFBDE42F0020601100209C30002019
:1089A80042320020DE190020E01900202DE9F84F9E
:1089B8000C9E3A4CC2EB030B0B9BF61A636800291A
:1089C80014BF4FF0060A4FF0040A013305469046DB
:1089D80013D1236853455ED2314A324852F82320D6
:1089E800032B98BF294608F0BDFD63680133636017
:1089F8002D4B002205469A7113E0002511E02B4A01
:108A08001278954240DA0B9BE3B109FB06F2995CB8
:108A180001228A40264909680A4213D16368013352
:108A28006360D4F804900A9B1C4F9945E7DB2BD16F
:108A38000A2007F063FF3B6801333B604FF0FF33C8
:108A48007B6021E0184A917921B12C2007F056FF6C
:108A5800013501E001219171226809FB0BF308EB54
:108A6800030752B958F8030008F012FD97F90410EB
:108A78004B1C0544D2D00F4802E03A440E48117905
:108A880008F070FD0544C9E7206850452CBF002058
:108A98000120BDE8F88F0020BDE8F88F4C32002097
:108AA800A88D010832AD0108D81A00208C000020DA
:108AB8003432002041AD010898B6010830B585B0C0
:108AC80004AC002524F8025D0091ADF806002146AB
:108AD8001020FFF713FC9DF806002146FFF70EFC57
:108AE8009DF807002146FFF709FC9DF80000214684
:108AF800FFF704FC9DF801002146FFF7FFFB9DF8F6
:108B080002002146FFF7FAFB9DF803002146FFF714
:108B1800F5FB9DF80E00C043C0B22946FFF7EEFBF7
:108B280005B030BD10B5054C206806F071FC18B1D1
:108B3800206806F06AFCF6E710BD00BF5C1A00204A
:108B48002DE9F04F2DED0C8B87B08246039390F8FA
:108B58005030029191461BB1322BA8BF322300E05E
:108B6800012307EE903AB8EEE7BADFEDD77AD74B94
:108B7800DFEDD7BA1B88D74D019587EE8BBA002B4E
:108B880008BF0123D44F07EE903AF8EEE79A2B88F6
:108B98009FEDD2CA69EEABBA13F0020F3BEE2BBAC7
:108BA8008BEE8BBA26D0B7F90030B7F9022083EAEA
:108BB800E37182EAE270A1EBE371A0EBE270884214
:108BC8000446B8BF0C46B4F5E17F16DA8842DFEDFB
:108BD800C4AA05DD002AD8BF524207EE902A04E055
:108BE800002BD8BF5B4207EE903AF8EEE77AC7EE63
:108BF800AAAA04E0F0EE4CAA01E0F7EE00AA9FED65
:108C0800B79AB84DD0464FF0000BB0EE49AAB64C13
:108C180034F91B300CEE903AF8EEECCAF5EE047A13
:108C280037F91B306CEEA7CA08EE903A019BFDEEAF
:108C3800ECCA1988F8EEEC7ADFEDACCA89074FEA7E
:108C48004B0667EEACCAF8EEE88A00F08580A849C2
:108C580031F91B3007EE903AF8EEE77AB0EE007A79
:108C6800E8EE877AC9F10000FDEEE77A17EE901A70
:108C7800814203DB4945A8BF494608469D49039BF5
:108C8800715E401A33F91B10084407EE900AB8EEDB
:108C9800E78A09F05FFF50B19749B2EE049A88EE6F
:108CA800090A11F80B0008F059FD20EE098A9AF814
:108CB8001C30DFED926A0AEE103A9AF8083007EE97
:108CC800903AF8EE677AB8EE4AAA68EE277AB1EEDB
:108CD800047A67EEA67A2AEE077AFDEEE77A17EEAF
:108CE800901AF1EE477ABDEEE7AA1AEE103A9942C9
:108CF80008DBBDEEC7AA1AEE103A8B42A8BF0B4696
:108D08000AEE103A7E4901EB8B01D1ED007AE8EECC
:108D18002B7ABBEE0E7AF4EEC77AF1EE10FAB8EEC3
:108D2800CAAA09D4B3EE0E7AF4EE477AF1EE10FA35
:108D3800C8BFF0EE477A01E0F0EE477AC1ED007A5D
:108D48009AF8123009EE103AB8EE499A67EE897A25
:108D58009FED6C9A27EE899A019B1988CA0751D40E
:108D6800A05F0028B8BF4042B0F5206F02DD85ED56
:108D780000CA26E09FED647A98F8013068EE877A99
:108D880007EE103AB8EE477A87EE877AD5ED007A83
:108D980037EE6C7AE7EE2B7A9FED5C7AF4EEC77AC1
:108DA800F1EE10FA09D49FED5A7AF4EE477AF1EE13
:108DB80010FAC8BFF0EE477A01E0F0EE477AC5ED49
:108DC800007A98F80B30D5ED007A08EE103AB8EE34
:108DD800488A8B0768EE277A9FED4E8A27EE888AA5
:108DE80014D578EECA8AF0EE4A7AEAEEA87A38EE16
:108DF800498AF0EE678AF0EE497AEAEE887AB0EEB0
:108E0800678A03E0B0EE498AF0EE4A8A42499FED4C
:108E1800437A1BF8013007EE903AF8EEE77A4FEA0A
:108E28008B0067EEEC7A0C1D0444E7EE878A043564
:108E380008F1010894ED007AC4ED00CA3CEEC77A47
:108E480001F10C0487EE2B7A20441431344C1BF8C2
:108E58000130D0ED007A37EE677AB0EE68DAEBEEE3
:108E6800077A08EE903AF8EEE88AC0ED007A67EEE5
:108E7800A87ADFED2C8A3DEE080A67EEA88A30EE64
:108E8800680A0DF05DFBBDEECDDAA0531DEE103A79
:108E9800254E264846F82B30BDEEC88AF1EE688A82
:108EA80018EE103AFDEEE88A214940F82B3018EE0A
:108EB800903A049041F82B300591BBF1000F39D15D
:108EC8004FF0010BA3E600BF83F9223EE810002013
:108ED800BD3786359C1A0020D811002000000000FC
:108EE8000000E143E01A002014110020CDCC4C40D2
:108EF80018340020DC2F00202C9501086F12033C49
:108F0800EC1A00200AD7A33D0000A043000040C38C
:108F1800000040430AD7233CF41A0020A69B443B98
:108F28004C2B0020F7CC9238542B0020602B0020CB
:108F38006C2B0020029AB7F9043095796D0028351A
:108F48005D434B4BB3F9043000EE103ABAEECF0A4A
:108F58000DF0F6FA6D11281A002D07EE900AB8BF29
:108F68006D42322DF8EEE76A424A02DD0023936033
:108F780026E0FDEEE99A19EE903A23F0030307EE96
:108F8800903AF8EEE79ADFED3C7A9AF80D30C9EEA0
:108F9800A77A07EE103AB8EE477A936826EE877AF2
:108FA80067EE277AFDEEE77A17EE901A0B443349FD
:108FB8008B42A8BF0B4632498B42ACBF936091608D
:108FC80093685B13B3F5807FA8BF4FF480736FF08D
:108FD800FF029342B8BF134607EE903AF8EEE78ACD
:108FE800FDEEE67A9AF8032017EE903A53439B1168
:108FF80007EE903A234B1B78032BB8EEE78A14D977
:10900800BAF84E20B2F5FA7F0FD2FDEEC87A534275
:1090180017EE901A994204DB914217EE903AA8BFD6
:10902800134607EE903AB8EEE78A78EE287AFDEE16
:10903800E77ACDED017ABDF80430A3801BB200EECB
:10904800103AB8EEC00A0DF07BFA049B059AA0808E
:10905800FDEEE88ABDEEC88AC3ED028A002386EDDC
:10906800028A936007B0BDEC0C8BBDE8F08F00BF9F
:1090780014110020182B002000803B45FEFFFF0F35
:10908800020000F0D42B00202DE9F04F2DED028BCB
:1090980089B000260693C44B0591B3F90270B3F961
:1090A80000300392002FB8BF7F42002BB8BF5B424D
:1090B8009F42B8BF1F46B7F5FA7F8046A8BF4FF456
:1090C800FA770190B3460296B2463446B74D2B88DC
:1090D80099075AD0B44BB64A33F8143032F91420F1
:1090E800022013FB0022039B5B429A424FEA440191
:1090F80003DB039B9342A8BF1346AE4A31F90290A3
:10910800069A32F91420C9EB030303EB020909F0AC
:1091180021FD88B107EE909AA74BB8EEE70AB2EEA8
:10912800048A185D80EE080A08F018FB20EE080A89
:10913800FDEEC07A17EE909A98F80830642203FB87
:1091480009F393FBF2F398F81C206FF0040A0AFB6A
:1091580002FA534504DB02EB820A9A45A8BF9A46F5
:10916800964A52F8241009EB010342F210718B421F
:10917800A8BF0B4692498B42B8BF0B4642F8243031
:1091880098F8122053431B1302932D8805F003030C
:10919800012B38D0844B8B4933F914B0019B51F81B
:1091A80024E093F801C0884B33F9140080EAE07397
:1091B800A3EBE073B3F5206F4FEA840616DC0BEBE4
:1091C8008B031A0192FBFCF3042290FBF2F0181AAD
:1091D8008644BEF57A5FA8BF4FF47A5E7B4B9E4506
:1091E800ACBF41F824E041F8243002E0002341F804
:1091F80024308B597D2693FBF6F6019BDB7A73436B
:10920800402693FBF6F6AA0711D50298C7F5FA721D
:1092180007FB0BF907FB06F54FF4FA7102FB0A99F5
:1092280002FB005599FBF1F395FBF1F505E0EB071F
:109238004DBF029D35465B46534662006449049221
:10924800614A605C32F814C004220FFA8CFE9EFB5F
:10925800F2F909FB00F06FF04F0990FBF9F9994416
:1092680001F1200333F9140023F814C0C0EB0E0EEB
:1092780001F124002C319EFBF2F251F8243050F811
:1092880024E041F824E0734498F8501040F8242072
:1092980013444FEA840C00EE103A79B14D4B4E4816
:1092A800D3ED000ACDF81CC0B8EEC00A00EBC4002C
:1092B800FEF796F8DDF81CC0BDEEC00A474A0498D0
:1092C800125D474910EE103A5343202293FBF2F304
:1092D80009EB0502D21A42524248434A4CF8005060
:1092E800424D4CF802905B424CF80530019B01332B
:1092F80001930CB90124E9E62B4B98F80D70B3F9EA
:109308000440059B9B790F335B0063435B112E4C34
:10931800002B4FF00406B4F9044094FBF6F4294EF0
:10932800A3EB0404B8BF5B42322BD6F808E00BDC91
:109338002F4B07FB04E7BB42A8BF3B462D4FBB4260
:10934800ACBFB360B76001E00023B36098F80330A6
:109358005C43294B1B78032B4FEAA4140CD9B8F8AB
:109368004E30B3F5FA7F07D25F42BC4203DB9C4222
:10937800A8BF1C4600E03C46B368946043F34F33F3
:10938800B3F5807FA8BF4FF480736FF0FF06B34238
:10939800B8BF3346E618836000238E80AB6009B0FF
:1093A800BDEC028BBDE8F08FD81100209C1A00207C
:1093B80018340020DC2F00202C9501080C1B0020FD
:1093C800F0D8FFFF182B00201411002080C1FFFFE8
:1093D800F41A0020482B0020302B0020081B002006
:1093E8004C2B0020602B0020542B00206C2B0020DD
:1093F800FEFFFF0F020000F0D42B00202DE9F04FF4
:109408002DED028B85B081460293AE4B01911C88ED
:10941800009204F00204A4B294B1AB4BB3F9024039
:10942800B3F90030002CB8BF6442002BB8BF5B42D0
:109438009C42B8BF1C46B4F5007FA8BF4FF4007427
:10944800CA460025A04BA14833F81520A04B50F878
:10945800256033F9153083EAE377A7EBE37711B298
:10946800B7F5206F4FEA450B4FEA41014FEA8508EF
:1094780011DC042793FBF7F3CB1A1E44B6F57A5F89
:10948800A8BF4FF47A56934B9E42ACBF40F8256074
:1094980040F8253002E0002340F8253050F80860F5
:1094A8009AF80B309AF80170F6115E43854B1B88C9
:1094B8004F439B074FEAA6164FEAA71756D0864B8D
:1094C80033F90B30022112FB0132009B5B429A42B6
:1094D80003DB009B9342A8BF1346804A3BF9022056
:1094E8009A1A029B33F91530D31808EE103A09F08E
:1094F80031FB68B1B8EEC80A794BB2EE048A80EE47
:10950800080A585D08F02AF920EE080ABDEEC08A5C
:10951800744918EE102A58F8013042F210701344BA
:109528008342A8BF0346704899F808208342B8BF11
:10953800034648F8013018EE101A4A4399F81C10EF
:1095480001EB8101D2114842824203DB8A42A8BF63
:109558000A46104699F8122053431B13F61A3F1A6D
:109568006643674303EB662600EB67275F4A584B61
:1095780012F805C03BF803004FF0040E03B293FB4A
:10958800FEF101FB0CF1A7EBA11702F134013BF945
:1095980001C02BF8010002F138004032CCEB030384
:1095A80058F8021093FBFEF358F800E048F802E080
:1095B8007144194400EE101A99F8501048F8003018
:1095C800434B69B14A4A4B48D2ED000A0393B8EEBF
:1095D800C00A00EBC500FDF703FF039BBDEEC00A00
:1095E800454A4648525D10EE101A51434911BA19BE
:1095F800521A2BF80020424A48F80270414F48F8A6
:109608000760414E494248F806100AF1010A11461E
:109618000DB9012516E72C4AB3F90430B2F9044014
:10962800019A99F80D5092790F3252006243521103
:10963800002A4FF0040493FBF4F3244CA2EB030339
:10964800B8BF5242322AD4F808E00BDC2F4A05FB97
:1096580003E5AA42A8BF2A462D4DAA42ACBFA26084
:10966800A56001E00022A26099F803205343294A2B
:109678001278032A4FEAA3130CD9B9F84E20B2F591
:10968800FA7F07D25542AB4203DB9342A8BF134689
:1096980000E02B46A2688B6042F34F32B2F5807F20
:1096A800A8BF4FF480726FF0FF04A242B8BF2246F1
:1096B8009C1800238480BA60B36005B0BDEC028BAF
:1096C800BDE8F08F9C1A0020D8110020182B00202C
:1096D8001411002080C1FFFF18340020DC2F002067
:1096E8002C9501080C1B0020F0D8FFFFF41A00206D
:1096F800482B0020302B0020081B00204C2B00207A
:10970800542B0020602B00206C2B0020FEFFFF0F45
:10971800020000F0D42B00202DE9F04F2DED028B34
:1097280087B000260593A14B0392B3F90270B3F9F1
:1097380000300090002FB8BF7F42002BB8BF5B42BB
:109748009F42B8BF1F46B7F5FA7F8246A8BF4FF4BD
:10975800FA77B1460196B0463446954D2B8899075D
:109768005BD0022C59D0914B924A33F8143032F91D
:109778001420022013FB0022039B5B429A424FEA0B
:10978800440103DB039B9342A8BF13468A4A31F97D
:1097980002B0059A32F91420CBEB030303EB020B5A
:1097A80009F0D8F988B107EE90BA844BB8EEE70A09
:1097B800B2EE048A185D80EE080A07F0CFFF20EEAB
:1097C800080AFDEEC07A17EE90BA9AF808306422BB
:1097D80003FB0BF393FBF2F39AF81C206FF00408D9
:1097E80008FB02F8434504DB02EB82089845A8BF52
:1097F8009846734A52F8243042F210715B448B4207
:10980800A8BF0B466F498B42B8BF0B4642F82430BD
:109818009AF8122053431B1301932B8803F0030279
:10982800012A01D1022C3FD16748604A30F914005F
:1098380032F914906549009A51F824E0567880EA84
:10984800E075A5EBE075B5F5206F4FEA84021EDCE4
:10985800022C16D009EB8901090191FBF6F60421C7
:1098680090FBF1F0361AB644BEF57A5F574958486E
:10987800A8BF4FF47A5E8645ACBF42F801E050506D
:1098880007E089EAE975A5EBE975642DE2DD0020BA
:1098980088504E497D26525892FBF6F6009AD27AA5
:1098A8007243402692FBF6F69A0713D5022C11D084
:1098B8000198C7F5FA7207FB06F507FB09F302FBE7
:1098C80008334FF4FA7102FB005293FBF1F392FB59
:1098D800F1F508E0DB0704D5022C02D0019D4346D0
:1098E80001E035464B4662003A490492364A605CCC
:1098F80032F814E04FF0040C0FFA8EF292FBFCFBE6
:109908000BFB00F06FF04F0B90FBFBF0034402934E
:1099180001F148034FEA840B33F9140023F814E0EB
:10992800121A01F150005C3150F824E051F824304B
:1099380041F824E092FBFCF273449AF8501040F886
:109948002420134400EE103A59B1234B2348D3ED99
:10995800000AB8EEC00A00EBC400FDF741FDBDEEF9
:10996800C00A1F4A1F49125D049810EE103A53436B
:10997800202293FBF2F3029A2A44D21A42521A4A3C
:1099880002994BF80210194A4BF80250184A5B42E8
:109998004BF80230009B01340133032C00937FF411
:1099A800DCAE07B0BDEC028BBDE8F08FD81100200B
:1099B8009C1A002018340020DC2F00202C95010868
:1099C8000C1B0020F0D8FFFF14110020182B0020DA
:1099D80080C1FFFFF41A0020482B0020302B002004
:1099E800081B00204C2B0020542B0020602B00204B
:1099F8006C2B00202DE9F04F2DED088B85B009EE7A
:109A0800902A0193C84B02931A8812F0020F8346DA
:109A1800B7EE009A4CD0169BC448DC89B0F90030E8
:109A28001B1B03F2F31540F2E632954203D8002BD4
:109A3800B8BF5B4201E04FF4FA73B0F90220121B81
:109A480002F2F31440F2E630844203D8002AB8BF89
:109A5800524201E04FF4FA729BF84C0058B393421B
:109A6800B8BF1346C3F5FA7307EE903A9FEDB07A84
:109A7800F8EEE77A6423C7EE877A93FBF0F307EEF4
:109A8800103A77EEC97AB8EEC77AF0EE498AE7EE6F
:109A9800878AF7EE006AF5EEC08AF1EE10FA0AD46A
:109AA800F4EE668AF1EE10FAC8BFF0EE668A04E0BA
:109AB800F0EE498A01E0DFED9F8A9F4DCB1C0093B1
:109AC800D9464FF00008AA46009B9C4F13F8014F57
:109AD8000093B8F1020F4FEA4806B2EE04AA0DD17E
:109AE800B7F904109FED967A0A3401FB04F307EEE8
:109AF800903AF8EEE77AC7EE877A64E0F8EE697A8A
:109B08009FED8B6A37F91830C7EE867A06EE903AE1
:109B18008C4B33F9183007EE103A19EE903AF8EEFC
:109B2800E66AB8EEC77A5B42A6EEA77A07EE903AE5
:109B3800F8EEE77AB4EEE77AF1EE10FA08D4F8EE28
:109B4800E97AB4EEE77AF1EE10FAD8BFF0EE477A88
:109B58007D4B9B5F08EE103A019BB8EEC88A33F93B
:109B6800183077EEC87A08EE103AB8EEC88A37EEA1
:109B7800888A88EE0A8A08F0EDFF40B1734B13F823
:109B88000800B0EE480A07F0E9FDB0EE408A029BF3
:109B98001988CA0704D5DBED117A68EE277A12E036
:109BA800BB5F9FED677A1434634307EE903AF8EE93
:109BB800E77A8B07C7EE877A42BF9BED127A28EEC9
:109BC800078AE8EE287A624B62499B5FDAED236ADE
:109BD800D9ED08AAD1ED000A9FED5F8A07EE103A89
:109BE800B8EEC77A5D4BE7EE667A18F80320D9ED30
:109BF8000B6A27EEAA7A0AEE902AF8EEEAAAB0EEE5
:109C080048BA67EE2AAA27EEA07ACAEE88AA27EEF3
:109C1800267AD5ED006AE7EE0A6A9FED517AF4EEEE
:109C2800C76AF1EE10FAB0EE66AA09D49FED4D7A34
:109C3800F4EE476AF1EE10FAC8BFB0EE47AA01E0A9
:109C4800B0EE47AA89EE208A47494FEA88042144A2
:109C580091ED000A85ED00AAC1ED007A37EEC00A41
:109C68009BF8501020EE080A31B14048039300EBEE
:109C7800C800FDF7B5FB039B13F80830F0EE087A2F
:109C880080EE270A08EE103AD9ED0E7AB8EEC88AA7
:109C980060EE277A27EE880ADFED357A80EE0B8AA8
:109CA800B4EEE78AF1EE10FA09D4DFED327AB4EEB9
:109CB800678AF1EE10FAC8BFB0EE678A01E0B0EE2D
:109CC800678A3AEE8A0A08F1010830EE080A0CF0B1
:109CD80037FC294BB0F57A7FA8BF4FF47A709842C9
:109CE800B8BF1846FDEEEAAA244B1AEE902A9853FC
:109CF800BDEECAAA224BBDEEC88AE250214B1AEE2D
:109D0800102AE250204B18EE102AB8F1030FE25047
:109D180009F1040905F104057FF4D6AE05B0BDECE0
:109D2800088BBDE8F08F00BF9C1A0020203000206F
:109D38000000FA4300000000E01A0020D8110020BB
:109D48000000484218340020DC2F00202C95010820
:109D580014110020482B00200000C842142B0020BA
:109D680000007AC300007A43701B0020302B0020CB
:109D7800000096C30000964318FCFFFF4C2B002000
:109D8800542B0020602B00206C2B0020426A806A34
:109D9800131A5842584170474171704743799B07DD
:109DA8000AD5436A8269D154436A01690133B3FB16
:109DB800F1F201FB12334362704707EE900AF8EEA6
:109DC800E77ADFED0C6A9FED0C0AF5EEC07AF1EE4A
:109DD80010FAD4BFB1EE677AC7EEA67A08B5D8BF35
:109DE800C7EE267A27EE800AFDF7C0FD034B83ED08
:109DF800000A08BD8096184B35FA8E3C7800002082
:109E080038B50D4B0D4D1A8A0D4B1968498811420A
:109E18001C4603D005F0F6F9286007E005F0F2F9D2
:109E28002B68984282BFC01A064B1860236858688E
:109E3800BDE8384002F03EB9000400487C1B002011
:109E4800B00700200400002003460A4690F84602A6
:109E5800D96A9B7901F006BA437913F0010310B56A
:109E680004460DD000F0CCFD58B1236A6269E16860
:109E7800D05C0133B3FBF1F201FB1233236210BD56
:109E8800184610BDF8B59B4B1B680446187818B1E6
:109E9800012800F068819BE2242C974D0CD006D84D
:109EA8000A2C00F0D9800D2C00F0D68046E12A2C2F
:109EB80006D02C2C04D041E128716871A8714EE1BC
:109EC8008E4B69792F798C4A002058542FBB19780A
:109ED800D771472921D1597850291ED19978472916
:109EE80007D1D978472904D11979412901D101210C
:109EF800D1719978814A522903D1D1784D2900F03E
:109F0800918299787D4A472907D1D178532904D17C
:109F18001279562A04BF0322EA71EA79764E022A98
:109F280039D0032A4CD0012A40F08580BA1E072A6E
:109F380000F28180DFE802F004080F131A257F2A57
:109F480007F09AFDA86076E01B78532B73D1AB68B5
:109F58005B42AB606FE007F08FFDE8606BE01B7859
:109F6800572B68D1EB685B42EB6064E01B78302BC1
:109F7800634B1A788CBF42F0020222F002021A7078
:109F880059E0002007F0D8FD287454E0002007F0BD
:109F9800D3FD68824FE0072F06D0082F4BD1012050
:109FA80007F0CAFDF08246E0012007F0C5FD41F246
:109FB800184358434FF47A73B0FBF3F0B0823AE099
:109FC800022F07D0032F0AD1002007F0B5FD4D4B13
:109FD800187030E0002007F0AFFD30762BE02AD96A
:109FE8003A1F9210337E0132D2B2013B02EB830357
:109FF800DBB2102B1FD8F91EC2F1010201EB82025D
:10A00800D2B2012A0BD0042A11D100205E1E07F01B
:10A0180093FD3D4B98553D4B00229A5507E05E1E37
:10A028003B4A0020935507F087FD3A4B98553A4A2A
:10A03800136801331360304B2A2C18BF9A7907F143
:10A0480001074FF000000CBF012254402F716871C6
:10A058000CBF5A769C7182E0687E002847D02F4B4F
:10A0680013F8012D2E495A708B42F9D1234A224CFC
:10A0780013785278402B85BF373B1B011B01DBB29D
:10A0880098BF03F0F003402A8CBF373A303AD2B277
:10A098001344AA79DBB29A4226D121230B702149B5
:10A0A800E0790B681E4A013301280B600AD00228A8
:10A0B8001CD1722313701C4BA28A1A801B4BE28A94
:10A0C8001A8013E0672313700D4B1B789F070ED57A
:10A0D800174BA2681A60E2685A60164B227C1A7005
:10A0E800154B628A1A8002E03F230B700020002380
:10A0F8006B7634E0D40700207C1B00201030002051
:10A10800D819002074110020A511002095110020F5
:10A1180075110020851100202C2A0020D80200206B
:10A12800C4020020382A0020DA1900205C1100201F
:10A13800E0190020DE190020DC1900206B79687E08
:10A148000E2B9FBFA34A591C5171A34A98BFD454E0
:10A15800A04A18B993795C40947100E0002000305F
:10A1680018BF0120F8BD9B4B997E0022082900F2F8
:10A178002F81DFE801F0050B0F15202B48606A00DE
:10A18800B52C40F02581DA7601223AE0622C08BF2E
:10A19800022236E003229A761C775C779C7717E1D7
:10A1A80004229A765A7F997FDC772244D2B25A7772
:10A1B8000A449A770CE105229A765A7F997F1C8483
:10A1C8002244D2B25A770A449A7701E106229A7653
:10A1D8005A7F997F2244D2B25A770A449A771A8CC6
:10A1E80002EB0424A4B2B4F5AC7F88BF794A1C847E
:10A1F80084BF0121D17600225A84002C40F0E880E7
:10A2080007229A76E4E05A7F997F2244D2B25A779D
:10A218000A449A775A8CB2F5AC7F3CBF6D498918CD
:10A2280002F1010238BF81F82440198C92B29142A0
:10A238005A84E5D9CCE008229A765B7FA34200F0E5
:10A24800C780644B0122DA760DE0644D9A7615F8E2
:10A25800012D6A70624A9542F9D1997F5D4AA142FF
:10A2680006D03F232B705F4A536801335360AFE039
:10A278005D48016801310160D07E10B13E232B702A
:10A28800A6E021212970D17F062941D004D80229CE
:10A2980007D0032923D0F8BD122959D0302967D017
:10A2A800F8BD502129705149946A4C60D46A0C60F9
:10A2B800516B4FF47A7491FBF4F14D4C218092F874
:10A2C8007C114C4A19B1117841F0020102E0117871
:10A2D80021F002011170012283F87D2169E05321E8
:10A2E800297092F82910CE0705D592F82820D51E96
:10A2F8006A426A4100E0024602F0010183F87C11DB
:10A30800002A56D13B490A7822F002020A7050E02E
:10A318004F21297092F82F10CC0705D592F82E20DE
:10A32800D11E4A424A4100E0024602F0010183F888
:10A338007C1122B92F490A7822F002020A702E4AAB
:10A3480093F8531011702D4AB3F85010118030E073
:10A35800562129702A49946B0C8042F21074D16BF3
:10A3680091FBF4F1274C2180012182F87E1120E035
:10A378004921297092F82810234A102988BF1021F2
:10A388001170224914780022A2420ED2204D0E7A72
:10A398005655204D4E7A56551F4DCE7A56551F4D5F
:10A3A80011F80C6F56550132EEE71D490A68013263
:10A3B8000A6093F87D31074A002B3AD092F87E3133
:10A3C800BBB3002182F87D1182F87E111846F8BDD2
:10A3D8000020F8BD7C1B002010300020D80200208F
:10A3E800C4020020B4070020382A0020E019002009
:10A3F800DC190020D8190020DE1900208200002076
:10A40800DA1900205C11002074110020A01B002024
:10A41800751100208511002095110020A51100203C
:10A428002C2A00201279432A7FF46BAD0222EA71AC
:10A4380067E5F8BD0449054B0968187000225A61A0
:10A4480099611A77704700BF08300020B4070020D0
:10A4580010B5121A07EE902A5B1A2DED028BF8EE52
:10A46800E78A07EE903A184B059CB8EEE78AD3EDD9
:10A47800007A28EE278A28EE080AA8EEA80A0CF027
:10A4880005FBDFED127A049B20EE270AF0EE480A5E
:10A49800BCEEC00A83ED000AB1EE680A0CF052F96E
:10A4A800DFED0B7A9FED0B7AE0EE077ABDEC028BBD
:10A4B800FDEEE77A17EE903A002BBCBF03F50C438C
:10A4C800A033236010BD00BF780000202C7D8E3F94
:10A4D80000A00C46A00CB34544F25063984203DD3B
:10A4E800A0F50C40A0387047034B9842BCBF00F55C
:10A4F8000C40A030704700BFB0B9FFFF73B51A4CCD
:10A50800036823600B686360184D0068184EFFF7F6
:10A5180054FC184B009395E8030094E80C0001964E
:10A52800FFF796FF144B32681A606868636813492E
:10A538001B1A07EE903A124B286893ED007A2368AD
:10A548001B1A0B600F4BF8EEE77A1A600E4B67EE9A
:10A55800877A1B68FDEEE77ADA880C4BC1ED017A41
:10A568001A8002B070BD00BFF02E0020E019002054
:10A57800FC2E0020F82E0020382F0020002F00206D
:10A5880078000020302F0020201000202C2F0020E1
:10A598004279DFED2A5A2A4B9FED2A5A07EE902A74
:10A5A800F8EE677AC27BC7EEA57AB2EE047AC3EDFD
:10A5B800007A07EE902AF8EE677A234ADA60C7EE47
:10A5C800A57AC3ED017A8179204B07EE901AF8EE4F
:10A5D800677A017CDA60C7EE877AC3ED007A07EE06
:10A5E800901A817E06EE101AF8EE677AB8EE466A7F
:10A5F800C7EEA57A86EE056AC3ED017A83ED026A95
:10A60800C179134B06EE901A417CDA60F8EE666A5F
:10A61800C6EE876A07EE101AC17EC3ED006A07EE20
:10A62800901AB8EE477AF8EE677A87EE257AC7EE81
:10A63800857A83ED017AC3ED027A70470000C8423B
:10A64800082F002000007A440000FA44182F002048
:10A658003C2F002010B50C4C23789B0713D50B4BCF
:10A668001B78042B0FD90A4A0A4B106852685A60A3
:10A678001860FFF7A2FB084B1A88084B1A8023784A
:10A6880043F00103237010BDD8190020DE19002003
:10A69800E019002060110020D01100204C2F00206C
:10A6A8001C4B1B681B0307B530D51B4A1B4BD2ED4F
:10A6B800007A1B788DF80030B2EE047A67EE877A5C
:10A6C800174B9FED187A1B788DF80130FCEEE77A6E
:10A6D8000A2017EE903AD2ED017A8DF8023067EE33
:10A6E800877A6946FCEEE77A17EE903AD2ED027A5D
:10A6F8008DF80330FCEEE77A17EE903A8DF80430C7
:10A70800094B1B788DF80530FDF734FE03B05DF872
:10A7180004FB00BFE42F0020F82F0020D62F0020D4
:10A72800F42F002000007A44DA2F0020054A13781D
:10A7380083F001031370044A00231360034A136073
:10A74800AEE700BFDA2F0020F02F0020EC2F00200A
:10A75800094A13781844C0B210F0800F18BF803827
:10A7680010701346054A19781378994201BF0023DF
:10A778001370014A13707047512F0020502F00208A
:10A7880010B50A4B0A4A1B7842609C18094A0460B3
:10A7980012789A4225BFD31A0B60C3F180030023B5
:10A7A8002EBF4B600B604A6010BD00BF512F0020C8
:10A7B800522F0020502F00201FB5684602A9FFF72E
:10A7C800DFFF044B02981B6803440398184405B044
:10A7D8005DF804FB280600202DE9F04F89B0824679
:10A7E80001930023029103929946039A934205DA52
:10A7F800029A52F8232001339144F6E7019B4D4613
:10A80800002B56D100F0E8FD002852D101987CE0D9
:10A8180002223F4E8DF81C201A0C4FF480578DF8F9
:10A828001D2006201A0A8DF81E208DF81F3000F012
:10A83800F7FD3785062006F0A7FE364BB7610122E3
:10A848001A700020378507A9042206F0C5FE029F6A
:10A85800D04626464FF0000B039B9B451EDABC46AC
:10A8680057F8042B4FEA8B03002A47D0B24235D35E
:10A8780032465AF80310CDF814C00020049306F0AD
:10A88800ABFE049BDDF814C05AF8032032444AF8A2
:10A898000320DCF800309E1BCCF800601C4B4FF402
:10A8A80080529A611C4A13682D1B1C44019B14603A
:10A8B8004BB345B3184B1B68DCB22A19B2F5807F3D
:10A8C800164AD2688CBFC4F580742C4693429FD335
:10A8D800134A00231370134A137014E00020D8F8A9
:10A8E800001006F079FE57F8043CD8F80020F61A54
:10A8F8001344C8F80030002347F8043C0BF1010B5F
:10A9080008F10408A8E7C5EB090009B0BDE8F08F15
:10A918000004004825060020280600201C0000200E
:10A92800502F0020512F002030B50B4C0B4D2278B2
:10A938002B789A4285B00CD0684602A9FFF720FF11
:10A948000123684602A90222FFF746FF00232B7065
:10A95800237005B030BD00BF512F0020502F0020BC
:10A9680030B50E4D0E4C2A7823789A4285B011D016
:10A97800684602A9FFF704FF002302A902226846DD
:10A98800FFF72AFFFFF7E4FE20782B781B1A5842BE
:10A99800584100E0012005B030BD00BF512F002014
:10A9A800502F002038B50E4C4FF4805545F2082042
:10A9B80000F036FD2585062006F0E6FD094BA56169
:10A9C80001221A70C720258506F0DEFD064AA5611A
:10A9D80000231370054A1370054A136038BD00BF81
:10A9E8000004004825060020502F0020512F002089
:10A9F80028060020FFF704BAFFF702BAFFF700BAEB
:10AA0800437913F001031FBFC36803F1FF32C36921
:10AA1800006A1DBF181A1040C0B21846704790F857
:10AA28003B3210B57BB990F83A3290F83942A342DC
:10AA380009D2B0F8401201229A400A430133A0F823
:10AA48004022DBB2F3E710BD8379DB07D0F834315D
:10AA580044BFB1FA81F149095A681B8909B1936168
:10AA68007047138570476E4B6E4A9FED6F7AD2ED33
:10AA7800007ADFED6E4ADFED6E3A30B51C88B3F927
:10AA88000AE01D8A06EE904AB8EEE76AF8EE666AB2
:10AA9800DFED687AB3F9044067EEE67AB7EE004A6C
:10AAA800E6EE077A9FED647A67EE666A9FED637A51
:10AAB800E6EE076A27EEA77A07EE904AB3F9024056
:10AAC8009FED5F6AF8EEE77A67EE277A07EE104A9D
:10AAD800B8EEC77ADC89E6EE877AB6EE007AFDEE44
:10AAE800E76A87EE866AC3ED066AF8EEE66AD2ED93
:10AAF800017A9A89E6EE874A06EE90EAB3F908E009
:10AB08009FED507A05EE90EAF8EEE66AF8EEE55A1F
:10AB180066EEA46A65EEA45A66EEA46AB3F806E087
:10AB2800E6EE875A65EE875AA5EEA34AF0EE445A38
:10AB380004EE10EAB8EE444A25EE844AB5EE404ADF
:10AB4800F1EE10FA5BD02DB205EE905A24B224EE45
:10AB5800A45A07EE104AF8EEE55A12B265EE255AE5
:10AB6800B8EEC75A65EEA35A64EE854AB0EE007A8D
:10AB7800E4EE875AB5EE007A65EE875A07EE102A9A
:10AB8800B8EEC75A9FED307ADFED306AB3F9162078
:10AB9800E5EE075AF8EEE77A9FED2D7A76EEE77A3A
:10ABA800DFED2C6AE5EEC77A05EE902AB0EE677AFB
:10ABB800DFED297AB3F91420B3F9123067EE277A5A
:10ABC80007EE102AC7EE847AF8EEE55AB8EEC77A8F
:10ABD80065EEA75A27EE877A65EEA75A27EE237AFD
:10ABE800A5EEA67AF0EE476A07EE103AB8EEC77AF5
:10ABF80036EE877ADFED196AE7EE267A01E0DFEDB7
:10AC0800187A18B1FDEEE77AC0ED007A31B1FDEEA1
:10AC1800C67A642217EE903A53430B6030BD00BFEA
:10AC280098020020FC1C00200000003700007AC7B2
:10AC380000000038000000390000803A0000803829
:10AC48000000A04500000036000080470000804951
:10AC580000008039000000300050C3450000803DEE
:10AC680000000000704770471FB50123ADF8083099
:10AC7800ADF80410002301A9ADF80A30ADF80C3086
:10AC8800ADF8062001F0DBFA05B05DF804FB38B535
:10AC9800A0F513746379A579DB0744D594F83832A5
:10ACA80005F00105EBB1226B1068C36A5B084362CB
:10ACB80094F83C3223B1B4F842320133A4F842325A
:10ACC800917A6A00FFF7D0FF012384F83B32002312
:10ACD80084F8393284F83A3284F83832A4F84032A9
:10ACE80038BD94F83B32012B04BF94F8393284F80C
:10ACF8003A322046FFF793FE94F83B22236B3AB989
:10AD0800012284F83B221868997A05FA02F207E0D2
:10AD1800002284F83B2295421868997A08BF0222DB
:10AD2800BDE83840A0E738BD10B5A0F5127494F816
:10AD38003C22BAB9A36A616A994228D0591CA06911
:10AD4800A162C35C2069DBB25B0043F400738142FB
:10AD5800A4F83E324FF00A0384F83D3228BFA262BD
:10AD6800012312E094F93D327BB1B4F83E124B084E
:10AD7800A4F83E32204601F00101FFF765FE94F881
:10AD88003D32013B84F83D3201E084F83C3294F8CE
:10AD98003832002B4ED194F839320133DBB2092B0B
:10ADA80084F8393203D12046BDE8104037E60A2B33
:10ADB80040D194F83B322BB9B4F8403243F0010348
:10ADC800A4F840326379D9071CD5B4F8400282054B
:10ADD80001D4C30705D4B4F844320133A4F844328B
:10ADE80010E0E36AC0F347000BB198470AE0E36953
:10ADF8006269D054E369E1680133B3FBF1F201FB06
:10AE08001233E361012284F8382294F83B220023AC
:10AE1800012A84F839320DD1A27984F83B32236BA8
:10AE280012F0010F1868997A0CBF02220022BDE8BF
:10AE3800104019E710BD7620F421312203F09ABFA3
:10AE480013B50622044603211E206B4603F016FFA5
:10AE580000283ED19DF800209DF801309DF8021091
:10AE680043EA02231BB21C4A07EE903A92ED007A9D
:10AE7800F8EEE77A012067EE877A92ED027AFDEE26
:10AE8800E77A17EE903A23809DF8033043EA0123CE
:10AE98001BB207EE903AF8EEE77A9DF8041067EED9
:10AEA800877A92ED017AFDEEE77A17EE903AA38061
:10AEB8009DF8053043EA01231BB207EE903AF8EEFD
:10AEC800E77A67EE877AFDEEE77A17EE903A6380C5
:10AED80000E0002002B010BD3000002007B5F721C7
:10AEE8006B460622762003F0C9FE9DF800309DF8D7
:10AEF80001100C4A1B0343EA01139DF8021043EAB0
:10AF0800111353609DF803309DF804101B0343EAA6
:10AF180001139DF8051043EA1113136003B05DF89F
:10AF280004FB00BFFC1C00201FB5044602210C20B6
:10AF380001220DF1070303F0A1FE08B900203BE050
:10AF48009DF80730DB07F9D50321062202AB0C2058
:10AF580003F094FE0C20092101220DF1070303F0F0
:10AF68008DFE0028EAD09DF8073013F00C0FE5D1CC
:10AF78009DF809209DF8083043EA0223C3EB833388
:10AF88009B009DF80B2023809DF80A3043EA02239A
:10AF9800C3EB83339B009DF80D2063809DF80C3034
:10AFA80043EA0223C3EB83339B00A3800C200A21CE
:10AFB800012203F0DFFE012004B010BD07B50A210D
:10AFC80000220C2003F0D6FE142004F042F90A21D6
:10AFD8000F220C2003F0CEFE0A2004F03AF901AB50
:10AFE800102103220C2003F049FE0A2004F031F955
:10AFF8000A2100220C2003F0BDFE0A2004F029F9E2
:10B008000DF10303022101220C2003F037FE0DF19C
:10B018000303092101220C2003F030FE0A2101223A
:10B028000C2003F0A7FE03B05DF804FB074B1B6878
:10B038001869074B20F01F0200F01F01D2580123A6
:10B048008B401A4201D001F035B87047B802002091
:10B05800140401402DE9F0437C4A136887B09046F8
:10B0680093B11A681AB17A49486902434A619A88C1
:10B07800ADF8002002228DF8032098680022694666
:10B088008DF8022003F0E4FC322004F0E2F80021FD
:10B0980011221E2003F06EFE012160221E2003F003
:10B0A80069FE642004F0D5F802A8FFF7C9FE002461
:10B0B8000A2726462546022101221E2003F05AFEB1
:10B0C800322004F0C6F802A8FFF7BAFEBDF908203E
:10B0D800BDF90A10BDF90C308A421444A8BF0A46CB
:10B0E80093421D44A8BF134613F5805F0E4404DD48
:10B0F800013FE0D14FF0010901E04FF000091E20A7
:10B108000021122203F036FE0A27022101221E2006
:10B1180003F030FE322004F09CF802A8FFF790FEFE
:10B12800BDF90820BDF90A10BDF90C308A42A4EB1C
:10B138000204A8BF0A469342A5EB0305A8BF13461D
:10B1480013F5805FA6EB010602DD013FDDD101E0CA
:10B158004FF0000907EE904A9FED3E7A3E4FF8EE19
:10B16800E77A0021C7EE277A70221E20F0EEE77AF0
:10B17800C7ED007A07EE906AF8EEE77AC7EE277A0D
:10B188009FED367AF0EEE77AC7ED017A07EE905A2E
:10B19800F8EEE77AC7EE277AF0EEE77AC7ED027A9B
:10B1A80003F0E8FD012120221E2003F0E3FD1E200C
:10B1B8000221002203F0DEFD642004F04AF8B9F110
:10B1C800000F04D14FF07E533B607B60BB60D8F822
:10B1D80000301E4C1A7B002A35D01A7D002A32D046
:10B1E8001B498A6942F001028A61187B197D01F0C6
:10B1F80011F823689A689B88128A134223D018484A
:10B2080004F0EAF82368186900F054FF23681B6902
:10B21800049300260C23012504A88DF815308DF819
:10B2280014608DF8165006F02BFA23688DF8066026
:10B238005B7D8DF8043001A803238DF805308DF867
:10B24800075006F0FFF907B0BDE8F083B802002008
:10B258000010024000406F463000002001C05E46EA
:10B2680035B000082DE9F04F544D1E464FF41473C5
:10B2780005F10804434385B080469146E718A24685
:10B2880010B92B444E4A03E0012805D14D4A2B44FE
:10B298009A631032C3F83C214FF4147303FB08F38C
:10B2A800EC180AEB030203F59C734748A06034329C
:10B2B80053446163E261236200224FF0010B4FF4B3
:10B2C8008071D4F83C3161610320A2626262A1619D
:10B2D8002263E26284F8442284F840B284F841226E
:10B2E800A4F84A22A4F84C22C4F810906073A673FC
:10B2F80084F84E8204F59C7258681B8901924FF0BD
:10B30800020C03A9ADF80C308DF80EB08DF80FC003
:10B31800CDF800C003F09CFBA36BDDF800C0597B9F
:10B3280058681B898DF80E1003A9ADF80C308DF8FC
:10B338000FC003F08DFB59463846FFF785FB3220D6
:10B3480003F087FF019A214BD2F804B0B3FBF9F15F
:10B35800B1F5803F03D3012BF8D95B08F6E74FF42A
:10B36800147404FB08F805EB0809584689B248220A
:10B3780008F5127804F0BCFD0AEB0804144BC9F870
:10B38800503200225846214604F008FED9F83850B9
:10B3980016F0010F0CBF022200222868A97AFFF7D5
:10B3A80063FC0C4BC9F854322846211D002204F0D6
:10B3B800F5FD384605B0BDE8F08F00BFFC1C002045
:10B3C8006CA701088CA70108C08D010800A24A04D7
:10B3D80031AD000897AC00080F4B73B518781C46C0
:10B3E80098B105230D4D8DF800304FF48056002399
:10B3F8008DF8013001A82E856946022206F0ECF886
:10B40800AE619DF8050000F0010000F00100207019
:10B4180080F0010002B070BD25060020000400483D
:10B42800064B70B51D6806461C46FFF7D5FF18B9D0
:10B4380023685B1BB342F8D970BD00BF08300020F9
:10B44800F7B503238DF80430030C8DF805308DF81B
:10B458000700030A06200F4614468DF80630FFF74A
:10B46800DFFF78B1084D4FF4805601A904222E85DC
:10B47800002006F0B1F838460021224606F0ACF864
:10B48800AE61204603B0F0BD0004004802464021EA
:10B498003C2003F06FBC70B500EB8000094CA0F1B4
:10B4A800A1059C3825440444074B15F8010F1E7864
:10B4B8007040FFF7EBFFA542F6D13046BDE870407B
:10B4C800E4E700BFD88D01082034002010B5441EE1
:10B4D80014F8010F10B1FFF7DEFFF9E710BD0246BF
:10B4E80080213C2003F046BC10B5D420FFF7F7FFBD
:10B4F8008020FFF7F4FFA820FFF7F1FF3F20FFF7B8
:10B50800EEFFD320FFF7EBFF0020FFF7E8FF402016
:10B51800FFF7E5FF8D20FFF7E2FF1420FFF7DFFFBD
:10B52800A120FFF7DCFFC820FFF7D9FFDA20FFF7DB
:10B53800D6FF1220FFF7D3FF8120FFF7D0FFCF20DF
:10B54800FFF7CDFFD920FFF7CAFFF120FFF7C7FFAC
:10B55800DB20FFF7C4FF4020FFF7C1FFA420FFF75F
:10B56800BEFFA620FFF7BBFFAF20FFF7B8FFA6205E
:10B57800FFF7B5FFAE20FFF7B2FF2020FFF7AFFFC0
:10B588000020FFF7ACFFB020FFF7A9FF4020FFF72E
:10B59800A6FF0020FFF7A3FF1020FFF7A0FF4FF43E
:10B5A8008064013C0020A4B2FFF770FF002CF8D1A2
:10B5B8008120FFF794FFC820FFF791FFAF20FFF726
:10B5C8008EFF012010BD08B55038C0B2FFF787FFC5
:10B5D8000020FFF784FF1020BDE808407FE75039BE
:10B5E80010B50446C8B2FFF77AFF04EB44004000E8
:10B5F80004EB440400F00E00FFF771FFC4F3C3002E
:10B608001030BDE810406AE7026BC168034610B508
:10B61800406942B11A6C8C1A013A005D08BF0A46AB
:10B62800C0B21A6410BD1A6A805C01328A4228BF0F
:10B638000022C0B21A6210BD436B13B190F84400E7
:10B648007047836A406A1B1A584258417047036B17
:10B6580013B15B68016C01E0C369016A8B423CBFAE
:10B66800C2689B18581AC0B27047836A8169426BD6
:10B678001944D160416A99429DBF0169CB1A536050
:10B68800CB1A96BF0023536083624FF0000380F803
:10B698004430136888BF816243F001031360704728
:10B6A800436A8269D154436A02690133934228BFCD
:10B6B80000234362436B1BB11B68DB0705D4D4E747
:10B6C800026D136843F0800313607047F0B5046D92
:10B6D8008668236823F0010323608379054613F005
:10B6E800020F40790CBF4FF0000E4FF4005E13F0CC
:10B6F800040F14BF4FF48067002710F0010F14BF28
:10B70800042100218307206820F00100206062687E
:10B7180022F440524EEA02026260226822F4B053D8
:10B7280023F00C0348BF41F008013B430B4323605F
:10B73800A36895B023F44073A360684600F042FE06
:10B74800284B9C4201D10C9B0EE0274B9C4201D117
:10B758000D9B09E0254B9C4201D10E9B04E0244B34
:10B768009C420CBF0F9B109B2268A879170448BF06
:10B778005B00B3FBF6F206FB1233B3EB560F2368FC
:10B7880028BF01321E0441BF4FF6F073C2F34201D5
:10B79800134041EA03026B7992B213F0020FA281BF
:10B7A80000F0010114BF4FF400320022DC0748BF4B
:10B7B80042F480322B6D11B159680A4302E059688E
:10B7C80021EA02025A609A6801074CBF42F0080257
:10B7D80022F008029A601A6842F001021A6015B055
:10B7E800F0BD00BF00380140004400400048004060
:10B7F800004C0040417169E7816067E7026D036BA7
:10B8080070B50446D5699BB9A90611D5C36A1BB1A1
:10B81800908C80B298470BE0E169928C40694E1C8D
:10B82800D2B2E6614254E169E268914228BFE3611D
:10B83800616BA1B92A0612D5636AA26A9A42236D7E
:10B8480009D0501CA669A062B25C1A852369984287
:10B8580005D3A16203E01A6822F080021A602B0760
:10B8680042BF236D08221A6270BD0D4B0D484FF47C
:10B8780000525A600C4A11684FF6FE730B40136071
:10B88800426B11684FF6FE730B401360426A836A7D
:10B898009A4200D0E9E6012380F84430704700BF9F
:10B8A80000000240302E0020440002402DE9F047FD
:10B8B8001E46A64B8CB09842894690469DF850503B
:10B8C80040F08580A24BA34A1A60A34A5A6102F548
:10B8D80080729A614FF48072DA601A619F4A1A6323
:10B8E800143A5A63A2F54842203ADA6404329A6458
:10B8F800C3F8088018659A4B9A6942F480429A61A5
:10B908005A6942F001025A6102238DF80830032374
:10B9180015F0010A8DF809304FF000038DF80A3050
:10B9280014BF022301232C078DF80B3019D54FF0D3
:10B9380090444FF4007701978AF001038DF80A309C
:10B94800636A23F0F0036362636A43F0700363621F
:10B95800204601A900F0A8FEBAF1000F27D1A7617F
:10B9680025E0B00710D50CA94FF4007341F82C3D21
:10B978004FF09040436A23F0F0034362436A43F078
:10B988007003436200F090FEF10710D50CA94FF444
:10B99800806341F82C3D4FF09040436A23F4706374
:10B9A8004362436A43F4E063436200F07DFE0E2382
:10B9B8008DF800300022012368468DF801308DF89B
:10B9C80002208DF80330624C05F03CFE0BE1654B1C
:10B9D800984276D1644B5F4A1A604FF48072DA60FD
:10B9E8001A61624A5A6102F580729A615C4AC3F828
:10B9F80008801865D36943F40033D36102238DF8B6
:10BA08000830032315F0010A8DF809304FF00003C0
:10BA18008DF80A3014BF022301232A078DF80B3052
:10BA280019D54FF090444FF4804701978AF00103ED
:10BA38008DF80A30636A23F070636362636A43F0C7
:10BA4800E0636362204601A900F02EFEBAF1000F00
:10BA580027D1A76125E0B30710D50CA94FF480437F
:10BA680041F82C3D4FF09040436A23F070634362E5
:10BA7800436A43F0E063436200F016FEF70710D50F
:10BA88000CA94FF4004341F82C3D4FF09040436A15
:10BA980023F070434362436A43F0E043436200F09B
:10BAA80003FE26238DF800300022012368468DF816
:10BAB80001308DF802208DF803302B4C05F0C2FDC3
:10BAC80091E02B4B984240F00F812A4B214A1A6093
:10BAD8004FF48072DA601A61274A5A6102F580725F
:10BAE8009A611F4AC3F808801865D36943F4802314
:10BAF800D36102238DF80830032315F0010A8DF86D
:10BB080009304FF000038DF80A3014BF02230123D7
:10BB18002C078DF80B3033D5184C4FF480670197FC
:10BB28008AF001038DF80A30636A23F47063636254
:10BB3800636A43F4E0636362204601A900F0B4FD40
:10BB4800BAF1000F40D1A7613EE000BF00380140C4
:10BB5800302E00207C900108A421002058000240CB
:10BB68000010024000440040DC2D0020A4230020E7
:10BB780000480040882D0020A4250020000400482B
:10BB8800B0070FD50CA94FF4806341F82C3D5848F5
:10BB9800436A23F470634362436A43F4E063436295
:10BBA80000F082FDF1070FD50CA94FF4006341F8AE
:10BBB8002C3D4F48436A23F470434362436A43F47D
:10BBC800E043436200F070FD27238DF80030002227
:10BBD800012368468DF801308DF802208DF8033076
:10BBE80005F030FD434CC4F82C900027012384F85D
:10BBF80044302762E761A76267626671C4F808800B
:10BC0800A5712046FFF762FDF20734D5236B002BA0
:10BC18002AD001A800F05AFAE36C01934FF480533C
:10BC28000A9380230693E368ADF810302023099324
:10BC3800206B636902930B970597079708970397FB
:10BC480000F06FFA01A9206B00F04DFA236B216D0B
:10BC58001A6842F001021A608A6842F040028A605B
:10BC68005B689BB2236406E0236D20221A621A687F
:10BC780042F020021A60B3072FD5636B43B301A8C3
:10BC880000F024FAA36C01934FF480530A938023A5
:10BC980006932369ADF8103000251023606B0393D9
:10BCA8000B95059507950895099500F03AFA606B8C
:10BCB80001A900F018FA636B1A6842F002021A60D0
:10BCC800226D5D605D60936843F08003936004E0DB
:10BCD800226D136843F080031360226D136843F0EC
:10BCE80001031360204600E000200CB0BDE8F08797
:10BCF80000040048882D00201FB50123ADF8083046
:10BD08000023ADF80C30ADF80A30094BADF804103B
:10BD18001B78ADF80620012B08BF032301A908BF33
:10BD2800ADF80C3000F08BFA05B05DF804FB00BFED
:10BD38002C010020084BDA68D10709D4DA68D2064A
:10BD480008D4DB6813F0040F14BF032004207047E5
:10BD580001207047022070470020024003788B4280
:10BD680086BF024B33F8110000207047A827002037
:10BD780070B5344C054603F045FAA369A061C31AAF
:10BD8800B3F5FA5FE36182BF002384F8203084F8BA
:10BD9800213094F820302BB9A12D02BF294A012166
:10BDA80082F8211094F82110264A31B1D118EDB249
:10BDB800013381F8225082F8203094F8205094F80A
:10BDC8004330AB423CD11F4B93F84430052B02D093
:10BDD800062B03D02FE0002006F0E8FD94F823306E
:10BDE8001E2B28D100200246C1B26B1E99421ADAD6
:10BDF800214491F822300821DBB283EA0206F607D3
:10BE080044BF83F01803C3F3460301F1FF3154BF65
:10BE18005B0843F0800311F0FF01C2F34702ECD145
:10BE280001301A46E0E7234493F822309A4202D1BF
:10BE3800032006F0BBFD002384F8213084F820306D
:10BE480070BD00BFA827002010B50446B0F9000057
:10BE580005F01AFBB4F9020005F016FBB4F904006A
:10BE6800BDE8104005F010BB10B50446006805F0A9
:10BE78000BFB606805F008FBA068BDE8104005F002
:10BE880003BB2DE9F74F0120FBF7D6F9002488B34F
:10BE9800012C2FD8194E4FF04C0909FB04FA06EB78
:10BEA8000A0808F19007BD7815B10134E4B2EEE74D
:10BEB80090F9003090F804E01846114B03228DE801
:10BEC800240001212A4653F82E30FBF78BF88346CD
:10BED80060B106F14800504429464A460AF021F963
:10BEE80001231C44C8F848B0BB70E4B20120FBF73A
:10BEF80089F9CCE703B0BDE8F08F00BFA827002080
:10BF08009490010800212A2210B511480AF009F975
:10BF1800104B002219461048105C83F8F2010424E3
:10BF28000520013283F8F74182424FF0000483F87C
:10BF3800F60183F8F94183F8F80103F10803EAD11F
:10BF48000123A1F8F431522381F8F03110BD00BF6C
:10BF5800D0130020E011002065AD010810B5FFF7EF
:10BF6800E9FE4FF43024012806D11CB1FFF7E2FEA8
:10BF7800013CF8E7052010BD002C08BF052010BDC6
:10BF880070B50646441E14F8011F89B1094D2846AC
:10BF98000AF0FDF80028F6D005F1080398423FBFE3
:10BFA800054B401BC018A31B38BF80F88631EAE751
:10BFB80070BD00BF00B90108E011002007B51C4B97
:10BFC80003F1E402C3F8E0201A4A92F88E215AB12C
:10BFD800012A14D1032183F8E610072183F8E82009
:10BFE80083F8E7100C2208E0022183F8E610032109
:10BFF80083F8E82083F8E710072283F8E4200E4B43
:10C008000E4A1A604020FBF717F970B1012200238D
:10C0180090F9000040218DE80C00094A4FF4E13303
:10C02800FAF7E0FF003018BF012003B05DF804FB09
:10C03800A8270020E01100203C0000206D270108FF
:10C04800212801080120002105F028BFF0B5184A71
:10C0580092F8E930D2F8EC701546042B11D807EBAA
:10C06800C3025E1C941CF6B209D013469288D1070D
:10C0780005D5104203D008E00131052908D133461F
:10C08800EBE785F8E9300020F0BD93F802E00021E5
:10C09800074C0C2204F1F00C02FB01F31CF80320FE
:10C0A8009645E9D1234484F8E960D3F8F400F0BD5B
:10C0B800A827002020F01F01012300F01F00024ADA
:10C0C80083408B50704700BF140401400023036075
:10C0D800436083608381036143618361C361036259
:10C0E8004362836270478A68036810B50C6A144318
:10C0F8000A6914434A6914438A691443CA69144390
:10C108004A6A14438A6A23F4FF4323F070032243E4
:10C11800134303608B8943600B6883604B68C3607B
:10C1280010BD02684FF6FE731340036000230360DE
:10C1380043608360C360294B984201D1284A27E0B5
:10C14800284B984201D1264A2AE0274B984201D130
:10C15800234A2DE0254B984201D1214A30E0244B57
:10C16800984201D11E4A33E0224B984204D11C4A1E
:10C17800536843F470032EE01F4B984204D1184AC9
:10C18800536843F0706326E01C4B984204D11C4A64
:10C19800536843F00F031EE01A4B984204D1184A23
:10C1A800536843F0F00316E0174B984204D1144A41
:10C1B800536843F470630EE0144B984204D1104A5C
:10C1C800536843F4704306E0114B984204D10C4A7B
:10C1D800536843F470235360704700BF080002405F
:10C1E800000002401C0002403000024044000240AF
:10C1F800580002406C0002408000024008040240DF
:10C20800000402401C04024030040240440402407E
:10C218005804024001F0030301F0FC0101F18041E0
:10C2280001F5803110B59B008C680F229A4024EAF2
:10C2380002028A608A68984002438A6010BD0A88B0
:10C248008B88F0B54C880E89CD88C2B9026A22F075
:10C25800010202628269016A22F0F3021A4342EA89
:10C26800061344F0010421F00A02144383610462B6
:10C27800836923F00C03836183691D431FE0042A4B
:10C28800016A1ED14FF6EF720A4002628269016AA2
:10C298001B0222F4734243EA06332401134344F099
:10C2A80010044FF65F720A40A4B22243836102620F
:10C2B800836923F440638361836943EA05258561C3
:10C2C800F0BD082A1DD14FF6FF620A400262C2691A
:10C2D800076A4FF60C7111404FF2FF523A4042EA9A
:10C2E800042443EA06130B4344F480749BB2A4B2BB
:10C2F800C3610462C2694FF6F3731340C361C36933
:10C308001FE04EF6FF720A400262C169026A40F6F7
:10C31800FF470F4045F6FF7111401A0242EA063303
:10C3280041EA04343B4344F480549BB2A4B2C36151
:10C338000462C2694FF2FF331340C3612D02C3691F
:10C34800ADB21D43C561F0BD036A23F0010303626A
:10C35800036A70B5446882690D6822F4803222F05D
:10C36800730215438A8923F0020313438A8813430F
:10C37800134A90420FD002F5006290420BD002F5AA
:10C388004062904207D002F58062904203D002F5E5
:10C39800806290420DD1CA89CE8823F008031343E6
:10C3A8000A8A24F4407414434A8A23F0040333436A
:10C3B80014438A68446085614263036270BD00BFAC
:10C3C800002C01409B4A536803F00C03042B2DE911
:10C3D800F04105D0082B06D097490160B3B916E0A3
:10C3E800954B036012E053685468C3F38343991C68
:10C3F800E30349BFD36A914B8F4C03F00F0344BF4B
:10C408000133B4FBF3F34B43036000E000235168AE
:10C418008B4FC1F3031139440D790168EDB221FA4C
:10C4280005F444605668C6F302263E44367924FA79
:10C4380006FEC0F808E05668C6F3C2263E443679C0
:10C44800F6B2F440C460D2F82C80C8F3041808F09F
:10C458000F0C07EB4C0C18F0100FBCF814C01FFAA7
:10C468008CFC07D0BCF1000F04D0B3FBFCFCC0F877
:10C4780010C000E00161D2F82CC0CCF3442C0CF0C1
:10C488000F0807EB48071CF0100FBF8ABFB204D093
:10C498001FB1B3FBF7F7476100E04161176BFF0677
:10C4A8005ABF654F87618161176BBF065ABF624FDC
:10C4B800C761C161176B7F065ABF5F4F0762016290
:10C4C800176BFF0506D5994204D1AE4202D14F0041
:10C4D800476200E04462176BFF0406D5994204D115
:10C4E800AE4202D14F00876200E08462176BBF053D
:10C4F80006D5994204D1AE4202D14F00C76200E08E
:10C50800C462176B7F0506D5994204D1AE4202D1A9
:10C518004F00476400E04464176B3F0506D5994215
:10C5280004D1AE4202D14F00876400E08464176BE7
:10C53800BF0406D5994204D1AE4202D14B00C36470
:10C5480000E08464156B3B4BAD0701D1046315E033
:10C558001C6B04F00304012C01D101630EE01C6B79
:10C5680004F00304022C02D14FF4004305E01B6BD6
:10C5780003F00303032B01D12F4B0363146B2D4BE3
:10C5880014F4403F02D1C0F834E018E01C6B04F406
:10C598004034B4F5803F01D1416310E01C6B04F4D2
:10C5A8004034B4F5003F02D14FF4004306E01B6B62
:10C5B80003F44033B3F5403F01D11F4B4363146B81
:10C5C8001C4B14F4402F02D1C0F838E018E01C6B63
:10C5D80004F44024B4F5802F01D1816310E01C6B72
:10C5E80004F44024B4F5002F02D14FF4004306E0D0
:10C5F8001B6B03F44023B3F5402F01D10E4B83632B
:10C60800146B0C4B14F4401F02D1C0F83CE021E03D
:10C618001C6B04F44014B4F5801F01D1C16319E008
:10C628001C6B04F44014B4F5001F0BD14FF4004305
:10C638000FE000BF0010024000127A0000093D0020
:10C648003C0000201B6B03F44013B3F5401F01D1DD
:10C65800134BC363126B134B12F4400F03D1C0F892
:10C6680040E0BDE8F0811A6B02F44002B2F5800F99
:10C6780002D10164BDE8F0811A6B02F44002B2F500
:10C68800000F02D14FF4004306E01B6B03F4400394
:10C69800B3F5400F01D1024B0364BDE8F08100BF40
:10C6A80000127A0000100240F0B500230E681C4604
:10C6B8000125A54005EA060EAE452BD10F797A1E55
:10C6C800012A15D8856803229A4025EA0202826069
:10C6D8004D7982689D4015438560828892B222EA2E
:10C6E8000E0282808A798588A2402A4392B282808B
:10C6F800032205689A40D2431540056005689F40AB
:10C708002F430760C7681740CA7902FA03F547EA5A
:10C718000502C2600134102C03F10203C8D1F0BD38
:10C7280038B52DED048B4A4C0368C4F82C31838846
:10C73800A4F83031013A0D46072A42D8DFE802F062
:10C74800040A101822292F35B4F82C310B80B4F8BC
:10C758002E3113E0B4F82E310B80B4F82C3105E0FB
:10C76800B4F82C315B420B80B4F82E315B4205E003
:10C77800B4F82E315B420B80B4F82C316B80B4F8DE
:10C7880030311DE0B4F82C315B420B80B4F82E3107
:10C7980012E0B4F82E310B80B4F82C310CE0B4F868
:10C7A8002C310B80B4F82E3105E0B4F82E315B4201
:10C7B8000B80B4F82C315B426B80B4F830315B42AB
:10C7C800AB80244B93F83430002B3ED1B5F90030C0
:10C7D80094ED500AD4ED4D7A09EE103AB5F90230CD
:10C7E80008EE103AB8EEC88AB5F90430B8EEC99A1E
:10C7F80028EE000A08EE903AA7EE890AF8EEE88AD1
:10C80800D4ED537AA7EEA80A09F09AFE94ED510ADE
:10C81800D4ED4E7A288028EE000AA7EE890AD4EDD6
:10C82800547AA7EEA80A09F08BFE94ED520AD4EDCB
:10C838004F7A688028EE000AA7EE890AD4ED557A67
:10C84800A7EEA80A09F07CFEA880BDEC048B38BDD1
:10C85800A82700203C000020104BDFED117A1B6850
:10C868009A89104B1B6883F31003D31A07EE103A0A
:10C87800B8EEC77A27EE277A07EE902AF8EEE77A1D
:10C88800C7EE277AFDEEE77A17EE900A6428A8BF6C
:10C89800642020EAE070C0B2704700BFC0190020D1
:10C8A8000000C842D0190020094B1A68137844F6D2
:10C8B800FB7103EB431300FB03135078C0EB00300C
:10C8C800B3FBF0F39078B3FBF0F080B2704700BF91
:10C8D800C019002008B50A4890F8593100EB430305
:10C8E8000A22B3F8681189B2A0F8701100F5BC707B
:10C8F80002F094FD80B2FFF7D7FF024B188008BD05
:10C90800A8270020C419002008B5084809F04DFCE4
:10C91800C0B209280246054B04DC01302021C0B210
:10C928009954F6E700221A5408BD00BF152A0020C2
:10C9380008B5074809F039FCC0B21428044B04D8DC
:10C94800421C20211954D0B2F7E700221A5408BD1E
:10C95800152A00202DE9F74FA74C02F053FC266852
:10C968006568A768861BF643451BC71BED43FF4355
:10C97800F60F8046ED0FFF0F2EB93FB9002D00F0DE
:10C988008682B9462CE04FF0000929E0B14627E03D
:10C9980003EB8A0BBBF802301A050ED413F4805F40
:10C9A8001DBF964A9BF801101268954A954B14BF13
:10C9B80052F82120126843F82A20BBF80230D80523
:10C9C80016D499050AD5904B1B7813F0040F0CBFA9
:10C9D8008E4A8F4A8B4B126843F82A2009F10109C5
:10C9E800207B8C495FFA89FA82450B68D0D326E010
:10C9F800894A5046594603F03DFB884B1B885A0626
:10CA080003D550465946864A16E0580703D550467E
:10CA18005946844A10E0190703D550465946824AB8
:10CA28000AE09A0703D550465946804A04E0DB07D6
:10CA3800D4D57F4A5046594603F01CFBCEE7DFF8B1
:10CA480008E20093BEF906307822A3F57A735343BF
:10CA58004FF47A7293FBF2F303F22B130193002243
:10CA6800F3465FFA82FE864517D2009B03EB820EDF
:10CA7800BEF802E01EF4806F0DD0DFF88891019BAC
:10CA880039F822E040F2671A9E449EFBFAFC0AFB42
:10CA98001CEE29F822E00132E3E74DB308F5C33371
:10CAA800A0336360637B544A13BB9373614B1B6869
:10CAB80013F0020F0AD0DFF894E19EF800E0BEF10F
:10CAC800000F03D04FF0010E82F80EE0DA0506D50C
:10CAD800594BDB781BB1A37B43F00203A3734A4B8A
:10CAE8001B7813F0050F02BFA37B43F00403A37365
:10CAF80094F80EE0BEF1000F03D13F4B5B7B002B97
:10CB08004FD094F80DC01CF0010FACF10C031DD1EF
:10CB1800BCF1030F07D8DFF8E8903C4A1EF0040F79
:10CB280008BF4A4600E0364AACF1040CBCF1070FD6
:10CB380005D8DFF81CC11EF0010F18BF6246DBB232
:10CB4800032B0ED81EF0020F3C4B06E0DBB2032B82
:10CB580006D82F4B2A4A1EF0020F18BF1A4600E0CB
:10CB6800274A4FF0000C5FFA8CF383420DD20B6812
:10CB780003EB8C035B881B0642BF224BD2F8009064
:10CB880043F82C900CF1010CEDE785B1BEF1000FD4
:10CB980008D0637B184A0133DBB2142B06D100237B
:10CBA80004E025B1637B002BF3D100E05373002E22
:10CBB80052D0234AB2F90250B2F90020002DB8BF72
:10CBC8006D42002A4FF03203B8BF524295FBF3F58D
:10CBD80092FBF3F2EDB2D3B2AB4238BF2B46194AFF
:10CBE80013B192FBF3F300E0134643442360E37B65
:10CBF800014A7BBB01232EE0A8290020042A00203B
:10CC08003CA80108920E00201F340020A8980108B3
:10CC180098980108A01A0020B49001089C1A0020D6
:10CC2800BA900108C0900108C6900108CC9001088C
:10CC3800D2900108E42F0020C4330020B0980108E6
:10CC4800D8110020400D030020300020241A0020B5
:10CC5800B89801080023D3738E4D8F4B2D78E27B53
:10CC6800ADB9002F00F00E818C4B267B1A788C4BC7
:10CC78008C4D93F800C08C4BD3F800E00B6802F0A1
:10CC880004020021D2B203EB86060F46B5E01AB9BA
:10CC9800864A1A61002508E0854AFAE70A68AB0067
:10CCA800D6187688760604D40135EBB28342F5D3DC
:10CCB800D7E7804EB6F90060192E25DD12F803E09B
:10CCC80094F814C026690EF00F09E1450CDCDFF872
:10CCD800C8C19CF815C0BCEB1E1FDEBFDFF8D8E149
:10CCE800D6F800C043F80EC012F803E094F816C056
:10CCF8000EF00F09E14533DBDFF89CC19CF815C045
:10CD0800BCEB1E1F2CDC26E0193629DA12F803E0EA
:10CD180094F814C026690EF00F09E1450CDCDFF821
:10CD280078C19CF817C0BCEB1E1FA2BFDFF888E1D2
:10CD3800D6F800C043F80EC012F803E094F816C005
:10CD48000EF00F09E1450BDBDFF84CC19CF817C06A
:10CD5800BCEB1E1F04DBD6F800E0574E43F806E094
:10CD6800544EB6F90260192E1BDD12F803C094F870
:10CD780014E026690CF00F09F1450CDCDFF8189176
:10CD880099F81590B9EB1C1FDEBFDFF82CC1D6F857
:10CD9800009043F80C90D25C02F00F0CF4451EDDB5
:10CDA80082E7193680DA12F803C094F816E026698B
:10CDB8000CF00F09F1450CDBDFF8DC9099F81590C1
:10CDC800B9EB1C1FDEBFDFF8F0C0D6F8009043F8BF
:10CDD8000C90D25C02F00F0CF445FFF665AF94F8A6
:10CDE80017E0BEEB121FA2BF334A36689E505BE7BE
:10CDF8005888000504D404330435B342F8D122E03E
:10CE08004AB101EB0C0A06209AFBF0F900FB19A0C5
:10CE180001280DDC01E057B9012793F801900EEBCA
:10CE280089003EF829A090F80290C07803E01746E0
:10CE3800002081468246013125F802AC85F8009031
:10CE48006870C9B2D7E7164A1378013B13F0FF039D
:10CE580008BF06231370114B1B785B0741BFBBF952
:10CE68000630A3F57A7303EBC3034FF47A7243BF1A
:10CE780093FBF2F30133DBB20123104A92FBF3F385
:10CE88004344A36003B0BDE8F04F01F003BD03B015
:10CE9800BDE8F08F430F0020A82900201F34002090
:10CEA80074000020940E0020042A0020B498010881
:10CEB8003CA80108D8110020920E0020400D030064
:10CEC80038B500240B4D6059254405F08DF8696884
:10CED80011B10948FAF7B8FCA96811B10748FAF77F
:10CEE800B3FC0748103405F07FF8B4F5F07FE9D1BA
:10CEF80038BD00BFD89001086AAD010870AD0108BF
:10CF0800E3BA010870B50546284609F04EF9064609
:10CF180058B91A4B1A485A791A4B03EB8203BDE8E1
:10CF28007040D3F8DC11FAF78FBC28461649324610
:10CF380009F044F960B91548154C05F055F854F84E
:10CF4800041F19B11348FAF77FFCF8E7124805E007
:10CF58000024124B53F8241021B91148BDE8704041
:10CF680005F042B82846324609F028F9013400286D
:10CF7800EFD1024B0B4D5C71C6E700BFE0110020FA
:10CF880076AD0108D890010882AD010887AD010887
:10CF9800B49201089AAD0108E3BA0108B8920108F1
:10CFA80042AC01086FA90108F0B585B0044609F044
:10CFB800FCF8082826D1621EE01D1F4912F8013F1F
:10CFC80009681944497801F00301022908BF203B88
:10CFD80082421370F1D1254604F1080715F8016B58
:10CFE8001648314609F0D3F820B12846314609F0F1
:10CFF800CEF810B1F9F784FB1CE0BD42EED1204613
:10D00800FEF7BEFF0E4804F0EFFF00230D4A1A4456
:10D0180004A992F886210A440849595C02F80C1CB4
:10D028000133082BF2D1002307488DF80C3001A9F1
:10D03800FAF70AFC05B0F0BD9000002000B901081D
:10D048009EAD0108E011002087B90108264B274C46
:10D058001D68206880B5F9F7A7FF2846F9F7A4FFEF
:10D06800206841798A0703D441F0020102F0C4F92B
:10D078001F4B08229A611F4B1A6812F4003F1F4683
:10D088001FBF06236371E37923F001031CBF43F03C
:10D098000203E371206802F0BBF990B1144E082333
:10D0A8003385124B186802F0B0F98046FCF7EAFEA7
:10D0B80008B103F0A9F82846414602F0ACF9082364
:10D0C800B361284602F0A4F938B12846266802F070
:10D0D8009CF90146304602F09EF93B689B03D9D57E
:10D0E80000F02BFFD6E700BF64300020C0290020E5
:10D0F80000040048E42F00202DE9F041054609F01E
:10D1080054F82C4B04469E6888B92B4804F06CFFF1
:10D118002A4B53F8241041B10123A340334202D0D3
:10D128002748FAF791FB0134F2E7264821E0284620
:10D138002549224609F042F858B92448244C04F0FD
:10D1480053FF54F8041F0029EFD01D48FAF77CFB61
:10D15800F7E72B782D2B03BF013504F1FF344FF08F
:10D1680001084FF000080026144B53F8267027B921
:10D178001848BDE8F04104F037BF28463946224632
:10D1880009F01CF898B90120B040B8F1000F03D09D
:10D19800FAF7B0FC104802E0FAF7B4FC0F4804F0C4
:10D1A80023FF39460E48BDE8F041FAF74DBB01367A
:10D1B800DAE700BFE0110020A4AD010820930108C0
:10D1C8009AAD0108E3BA010882AD0108AEAD0108C5
:10D1D8001C93010842AC0108BAAD0108C3AD0108AF
:10D1E80086B9010810B5084804F0FEFE074B002474
:10D1F8001C741C64064B1C7002F092FA05F0A6F829
:10D20800044B1C6010BD00BFCBAD0108C029002035
:10D21800213400206430002070B5064600240B4BF2
:10D22800E518AA8816420AD0E1580948FAF70CFB13
:10D238002846002104F065FE064804F0D5FE1434A3
:10D2480040F66C439C42EAD170BD00BF609A010869
:10D25800F7AD0108E3BA010808B50848FAF7F4FA87
:10D26800FDF7A0FBFEF7B8F818B9642001F0F1FF4C
:10D27800F8E70348BDE80840FAF7E6BA01AE010846
:10D288000EAE01082DE9FF410A48068885684488E2
:10D29800B0F80480C768FDF78FFACDF800800290D7
:10D2A800019731462A4623460348FAF7CDFA04B0D7
:10D2B800BDE8F0811C00002016AE0108F0B5047826
:10D2C8008BB005460CB1002436E04B4B19680E2391
:10D2D80003FB041101F58C70B1F91D51B1F9192145
:10D2E800B1F91B31009591F82051019591F8215120
:10D2F800029590F90700039001F590713F4891F964
:10D308000210049121460134FAF79EFA082CDCD168
:10D3180070E02D2B14D1072C1BDC284608F09CFF4D
:10D328000AAB661C03EB440424F8100C15F8013F03
:10D33800303B092BFAD934462B78002BE9D104E08D
:10D34800A3F13002092A09D8E5E7082CBDF818200E
:10D3580009D00BB0BDE8F040F9F7D2B9202BF8D1CD
:10D3680001352646E7E7072AF3D8BDF81A00224B0D
:10D37800A0F2EE2189B240F2DC55A9421B68E8D838
:10D38800BDF81C10A1F2EE24A4B2AC42E1D8BDF85D
:10D398001E6004B237B2A742DBDB0DB2AF42D8DC65
:10D3A800A542D6DBBDF8247007F16404A4B2C82CEA
:10D3B800CFD8BDF826E00FFA8EF4112CC9DCBDF8E1
:10D3C8002050B42DC5D8BDF82240B42CC1D812B213
:10D3D8004FF00E0C0CFB0233A3F81901A3F81B1134
:10D3E800A3F81D6183F8205183F8214183F81F7148
:10D3F80083F822E10BB0F0BD3011002073AE0108B4
:10D40800F0B504468FB0204608F0CFFEC5B225BB64
:10D41800AF48B04C04F0E8FD94F8D21009B9AE4812
:10D4280054E049B294F8D02094F8D130009194F89F
:10D43800D310019194F9D410029194F9D510039165
:10D4480094F8D6100491A54829460135FAF7FCF955
:10D45800102D04F10704DFD1E1E72046A049052299
:10D4680008F0ACFE0546B8B929469E48702208F077
:10D4780058FE9D4B196828460E2303FB0013013004
:10D488000022082883F8232183F8242183F8252102
:10D4980083F82621F0D119E120469449042208F0A6
:10D4A8008DFE05462046002D4AD1202108F06FFE4A
:10D4B800002800F00B81461C304608F076FE2C460A
:10D4C80007468B4B53F824502DB98A480FB0BDE856
:10D4D800F040FAF7B9B930462946FAB208F06EFEBC
:10D4E80001340028EDD17B4A02F170011646002371
:10D4F80082F8D63082F8D23082F8D13082F8D03033
:10D5080007328A42F3D17C4901EBC40191F8A02289
:10D51800934210DAD1F8A472C3EBC302B0183A44AC
:10D5280000F1D0011768C0F8D0709088888092798F
:10D538008A710133E7E729467048FAF785F996E0DA
:10D548006F49072208F03AFE05462046002D4AD1C9
:10D55800202108F01CFE064608F027FEC4B274BB62
:10D568006848FAF771F9214667480134FAF76CF907
:10D578000E2CF8D15848FAF767F900246348214679
:10D58800FAF762F90025584A614811680E2202FB31
:10D5980004120123D2F823215E49AB4013425E4BAB
:10D5A80005F1010508BF1946FAF74EF90E2DEAD123
:10D5B80049480134FAF748F9082CDFD186E03046AB
:10D5C800564908F04DFE2C46002852D0022C55D062
:10D5D80008F042FE06AB514943F82400002008F049
:10D5E8003FFE0134F0E74D4908F03AFE002460B1EF
:10D5F800082C3ED008F030FE06AB484943F824001A
:10D60800002008F02DFE0134F1E7082C31D1069BEB
:10D618000F2B2ED8DDF81CE0BEF1070F29D8089F84
:10D628000D2F26D8099E06F16402C82A21D80A9D22
:10D63800FF2D1ED80B9864281BD80C99642918D87C
:10D64800884216DA0D9C032C13D8224AC3EBC30375
:10D65800134483F8D0E083F8D17083F8D26083F85C
:10D66800D35083F8D40083F8D51083F8D6402C4CD7
:10D67800C9E60FB0BDE8F040F9F742B8069B072BA2
:10D6880020D807990D291DD80278722A0DD06E2A44
:10D6980018D1154A12680E2000FB032301228A4084
:10D6A800D3F8231121EA020209E00F4A12680E207A
:10D6B80000FB032301228A40D3F823110A43C3F84D
:10D6C800232101E0F9F71CF80D4C9CE60FB0F0BDE2
:10D6D8009BAE0108E0110020E3BA0108C6AE0108BC
:10D6E80012AC0108B0120020301100203DAC010836
:10D6F800B892010842AC0108D890010851AC010861
:10D7080093AE010874AD0108E2AE010898B60108AD
:10D71800E7AE010843BD0108FDBD0108EBAE0108F5
:10D728006FA901082DE9F743047805468CB9324DF5
:10D7380095F8AF12B5F8AC2295F8AE322F480091A3
:10D7480021460134FAF780F8102C05F10405EFD1D1
:10D758004EE008F081FD0F28044636DC28462021DB
:10D7680008F015FD264EE4B2D6F84480451CA40006
:10D778000027284608F070FD5FFA87F9B9F1010F14
:10D7880083B208D0B9F1020F0BD0B3F5B47F24D21D
:10D79800726C13530AE0FF2B1FD8736C23449870E4
:10D7A80004E0FF2B19D8736C2344D87028462C2129
:10D7B80008F0EDFC054608B1013502E0B9F1020FA9
:10D7C8000BD10137032FD4D112E00E4800210F22CC
:10D7D80003B0BDE8F043F8F710BF08EB04000021E0
:10D7E800042208F09EFC03B0BDE8F043F8F788BFB8
:10D7F80003B0BDE8F08300BFE0110020EDAE0108E2
:10D80800C0290020D0AB01082DE9F0412DED048B93
:10D81800B1498AB0044608F08DFCB049002820467A
:10D828000CBF0126072608F085FCAD4900282046D4
:10D8380008BF022608F07EFC002808BF0426F1076E
:10D8480040F1F080A748A84C04F0CEFB002004F07B
:10D85800D1F9A64804F0C8FBA54804F0C5FB6279D5
:10D86800A44BA54803EB82032546D3F8DC11F9F74E
:10D87800EBFFA248F9F7E8FF4FF00008274695EDBF
:10D88800048AB5EE408AF1EE10FA04D19C48F9F703
:10D89800DBFF002570E09B48D5ED059A95ED069ACB
:10D8A800D5ED078A4146F9F7CFFFB5EEC08AF1EE0C
:10D8B80010FA02D5202004F08FFBB0EE480A06A823
:10D8C800F9F742FE01469048F9F7BEFFF5EEC09A17
:10D8D800F1EE10FA02D5202004F07EFBB0EE690AC2
:10D8E80006A8F9F731FE01468748F9F7ADFFB5EE0E
:10D8F800C09AF1EE10FA02D5202004F06DFBB0EECC
:10D90800490A06A8F9F720FE01467F48F9F79CFF67
:10D91800F5EEC08AF1EE10FA02D5202004F05CFB87
:10D92800B0EE680A06A8F9F70FFE08F101080146EB
:10D938007648F9F789FFB8F10C0F05F110059ED16B
:10D94800A4E749B294F8D02094F8D130009194F823
:10D95800D310019194F9D410029194F9D510039140
:10D9680094F8D61004916A4829460135F9F76CFFF6
:10D97800102D04F1070403D094F8D2100029E0D147
:10D988006448654C04F030FBD7F8088054F8041F4D
:10D9980019B16248F9F758FFF8E70D46604B53F89C
:10D9A800254054B10123AB4013EA080F03D05D486A
:10D9B8002146F9F749FF0135F0E75B4804F014FB0D
:10D9C80021467B180AAA93F886311344574A8A5C81
:10D9D80003F8102C01310829F3D1002306A9544873
:10D9E8008DF82030F9F730FF524804F0FDFA52481C
:10D9F800F9F75CFB514804F0F7FA4F48F8F786FE50
:10DA08004F4804F0F1FA4C48FFF78CFE4D48F9F7FF
:10DA18001BFF4020FFF700FC4B4804F0E5FA46489E
:10DA2800F9F7A4F9B20739D5484804F0DDFA4848AF
:10DA380004F0DAFA404804F01DF9464804F0D4FA34
:10DA48003D48F8F7E7FD444804F0CEFA3A48F9F7BC
:10DA5800DFF84248F9F7F8FE3748F8F763FF40481F
:10DA680004F0C2FA3448FFF729FC00270E257D434D
:10DA780000243C4A926C2A440123D2F80A20A3408D
:10DA880013421ED101340E2CF3D10137082FEDD1EA
:10DA98002C48F9F7D9FE8020FFF7BEFB730716D58F
:10DAA800314804F0A1FA314804F09EFA224804F003
:10DAB800BBF82448F9F7C8FE4FF48070FFF7ACFBB9
:10DAC80005E0394622462A48F9F7BEFEDAE70AB0E9
:10DAD800BDEC048BBDE8F08101AF010879B3010802
:10DAE80008AF01080EAF0108E01100201CAF0108C3
:10DAF8002EAF0108D89001083AAF010845AF0108D8
:10DB080052AF01085FAF010873AD010887B901087A
:10DB180077AF010867AF01081C93010896AF0108A9
:10DB280020930108A4AF0108B1AF010800B90108AA
:10DB3800BDAF0108C6AF01086FA90108D5AF01083C
:10DB4800E1AF0108E3BA0108EFAF0108FCAF010833
:10DB58000FB001081DB0010827B0010836B0010850
:10DB680044B00108C029002050B0010861B0010884
:10DB780073B0010830B50028104C114AB8BF4042B4
:10DB88003C2590FBF2F304FB030068430D4D90FB2A
:10DB9800F2F22D682D7B25B903EB830303EB830396
:10DBA80001E0C3EB031302EB83030B8004FB0202C7
:10DBB8004FF47A7392FBF3F24A8030BD806967FFB5
:10DBC80080969800C8190020022803D0431E5842A6
:10DBD80058417047064B1B681B7823B1054B1868E2
:10DBE800C0F3C0407047044B1878C0F380007047FA
:10DBF80004060020F41000201F34002010B50A4C41
:10DC08005E280146206805D15D2101F004FC2068EA
:10DC18003E2105E05D2903D101F0FDFB20683D218F
:10DC2800BDE8104001F0F7BB0C2A002010B50446EF
:10DC3800C0B2FFF7E3FFC4F30720BDE81040DDE7FB
:10DC4800024B5E21186801F0E6BB00BF0C2A0020D9
:10DC580038B5064C05465E21206801F0DCFB2068DB
:10DC68002946BDE8384001F0D6BB00BF0C2A002089
:10DC780013B5044601A90068FFF77CFF1320FFF7DE
:10DC8800E7FFBDF90400FFF7D1FF1B20FFF7E0FF16
:10DC9800BDF90600FFF7CAFF2320FFF7D9FF236865
:10DCA800002BB4BF53204E20FFF7C0FF01A96068C6
:10DCB800FFF760FF1220FFF7CBFFBDF90400FFF765
:10DCC800B5FF1A20FFF7C4FFBDF90600FFF7AEFF46
:10DCD8002220FFF7BDFF6368002BB4BF5720452003
:10DCE800FFF7A4FF02B010BD674B73B51878674DF6
:10DCF800FFF76AFF2B788342044620D0C8B1644BF3
:10DD08001B68E3B193F9000002230093614B1B6881
:10DD18005B78003318BF0123019304214FF4165395
:10DD28000022F9F75FF95C4B186040B101232B70B2
:10DD380005E0594E3068F9F742F934602C70574BBA
:10DD4800574D1878FFF740FF2B788342044618D0C8
:10DD580088B1544B1B68A3B10022012493F9000039
:10DD680000944FF4964301920821F9F73BF94E4B82
:10DD7800186028B905E04C4E3068F9F720F934608E
:10DD88002C704A4B4A4D1878FFF71EFF2B788342B8
:10DD980004462E4642D0002837D0464B1A68002A3F
:10DDA8003CD0D37992F90000434C002B08BF0223E2
:10DDB80002220092002254F8233001921021F9F730
:10DDC80011F93E4B0546186040B33D4C94F84A3073
:10DDD800022B0BD094F89620022A01D14C3405E08E
:10DDE80023B1002A04F14C0418BF0024354B1C60F1
:10DDF80044B1204600214C2208F093F90223256003
:10DE080084F84A300123337008E02C4E306803F060
:10DE1800F1FF3068F9F7D3F834602C702A4B2B4D9A
:10DE28001878FFF7D1FE2B788342044629D000B337
:10DE3800274B1B682BB3274A93F9000012685278C6
:10DE4800002A0CBF082209220323009301924FF4F1
:10DE5800614320210022F9F7C5F81F4B186080B1F3
:10DE68001E4A012313702B701D4B1A681D4B1A6034
:10DE780007E0194E3068F9F7A2F8184B34601C70A7
:10DE88002C7002B070BD00BF0C060020B811002035
:10DE980008060020C81900200C2A00200D060020C2
:10DEA800E81900206C1A00205C1A002018060020CF
:10DEB800721A00201406002094900108741A002099
:10DEC800F0270020781A002024060020881A002055
:10DED800200600201C0600208C1A0020901A002022
:10DEE80008300020941A0020642928BF6421F8B55E
:10DEF80010FB01F56424064695FBF4F40027E4B210
:10DF0800FBB2A34204D29F20FDF7C5FA0137F7E719
:10DF1800B4420BD2C4EB84101421C4EB800095FBEF
:10DF2800F1F5663D2844C0B2FDF7B5FA0134E4B214
:10DF3800B44201D29A20F7E7F8BD2DE9F743934C94
:10DF480001F060F96368C31A002BC0F2688300F51A
:10DF5800433303F5A07363608D4B1D78237AC5F3B3
:10DF68008005EB1A18BF012325724DB1002B00F074
:10DF78005683884B5A789A7001225A701A702BE08F
:10DF8800844A2BB1D37843F00203D370937853704B
:10DF9800D67806F0020101F0FF0339B97D49896896
:10DFA800411A002903DB06F0010300E0012303F016
:10DFB8000107784917707BB1F2070DD50A7901324C
:10DFC800D2B20523B2FBF3F303EB8303D31ADBB21C
:10DFD800714A0B71D35C4B706E4EDFF80882337850
:10DFE8007BB3F37823F00203F3706C4B0344AE2049
:10DFF800B360FDF774FA08B1FDF776FA88F8000007
:10E00800002800F00C83B020FDF769FA4020FDF7E6
:10E0180066FA0020FDF763FA1020FDF760FA4FF466
:10E028008067013F0020BFB2FDF730FA002FF8D11A
:10E038003846FDF7C8FA7278594B53F82200FDF7B5
:10E0480045FA98F80030002B00F0E9827378062B27
:10E0580000F2B382DFE813F00700B102180078007D
:10E068006C018901EE014F494F4A504B5048F9F76E
:10E07800D6FB0120FDF7A7FA4D48FDF727FA022045
:10E08800FDF7A1FA4B48AEE14B4F3B689B0735D5EE
:10E09800DFF85481DFF85491B8F8001044480A2397
:10E0A800B1FBF3F203FB121399F80010009192B23E
:10E0B80042499BB2F9F7B3FBFEF73AFC0120FDF7A2
:10E0C80082FA3B48FDF702FA3D4B99F800201868A0
:10E0D800B8F80030067906FB123164234B43C17847
:10E0E8008E1B56430220B3FBF6F6F6B2FDF76BFA29
:10E0F80031461520FFF7F8FE032600E001263B68AD
:10E108001F0540F15A822F4B2F491F68096800915B
:10E1180064232E4997FBF3F2254803FB1273F9F7A2
:10E128007EFBFEF705FC3046FDF74DFA2048FDF76B
:10E13800CDF9FEF791FB0746701CFDF744FA152050
:10E148003946FFF7D1FE38E20120214FFDF73BFAAF
:10E158002048FDF7BBF93B68980749D51E4A144883
:10E16800B2F90210B2F900300091B2F904201B494B
:10E1780001921B4AF9F753FBFEF7DAFB0220FDF781
:10E1880022FA0B48FDF7A2F9032632E00C2A0020F8
:10E198001F340020C4290020ABB50108404B4C00B7
:10E1A80008950108B0B50108B9B50108BDA901086D
:10E1B800152A0020C0B50108E42F0020CBB50108BE
:10E1C800C0190020CC190020D0190020E3B501089F
:10E1D800D4190020F8B50108C21100200EB60108B4
:10E1E8001DB6010879020020C41900208000002013
:10E1F80002263B68D9071AD57C4A7D48B2F9021035
:10E20800B2F900300091B2F904207A4901927A4AB1
:10E21800F9F705FBFEF78CFB3046FDF7D4F9744897
:10E2280006F10108FDF752F95FFA88F846463B689F
:10E238001A0718D5714A6E48B2F90210B2F90030BF
:10E248000091B2F904206B4901926D4AF9F7E7FA97
:10E25800FEF76EFB3046FDF7B6F96548771CFDF70B
:10E2680035F9FFB23E46674A6249B2F90030B2F961
:10E2780002200092644A5E48B2F900200192634A83
:10E28800634FF9F7CCFAFEF753FB3046FDF79BF9DD
:10E298005748FDF71BF997ED000A5548F9F754F967
:10E2A800534807F082FF06F101085FFA88F8C0B208
:10E2B800B946092809D8431C2044DBB220224272FF
:10E2C800E218002191721846F3E7494F99ED010AC7
:10E2D8003844F9F739F9FEF72BFB4046FDF773F997
:10E2E8003846FDF7F3F899ED020A3846F9F72CF9A4
:10E2F800384607F05AFF0236F6B2C0B2092809D8E4
:10E308002318421CD2B220215972A31800219972F5
:10E318001046F3E73F4AB2F9003000EE103A3844AD
:10E32800B8EEC00AF9F710F9FEF702FB304657E0DD
:10E338000026394F3B78B34240F23F810E2E00F061
:10E348003C8170080130FDF73EF9304603F01AFCB5
:10E358003B78B34206D92020FDF79DF8701CC0B267
:10E3680003F010FC0236F6B2E3E72C4E2C4996F87F
:10E37800B4271F48F9F753FA0120FDF724F91C4880
:10E38800FDF7A4F8274B28491F7819483A46F9F7AA
:10E3980046FA0220FDF717F91548FDF797F80C2300
:10E3A80003FB0766214996F8B72796F8B637104851
:10E3B800F9F735FAFEF7BCFA0320FDF704F90C4823
:10E3C800FDF784F896F8BC1796F8BA2796F8BB3785
:10E3D800074800911649F9F722FAFEF7A9FA04202E
:10E3E800FDF7F1F80248FDF771F8E6E01411002096
:10E3F800152A00200EB6010821B601081A110020BE
:10E4080016C50108DC2F0020D011002025B6010810
:10E4180078080020840800208C280020E0110020C3
:10E4280029B601084830002035B6010846B601086B
:10E4380057B601087B4B1B681B0640F1BA80236A5C
:10E44800616A794A8B421FBF536292F828300133C0
:10E4580003F003034FF001014FF0000018BF82F8EA
:10E468002830FDF7BCF894F82830704AD05CFDF7E6
:10E4780012F802200121FDF7B2F800266C4B9B5DD3
:10E488003620C3EBC30393FBF0F0C0B2062828BFC5
:10E4980006206038C0B20136FCF7FDFF102EEDD122
:10E4A800644B65491B78654813F0020F644B1A7872
:10E4B80014BF59234E23F9F7B2F9FEF739FA0220AF
:10E4C800FDF781F85D48FDF701F85E495E4B4E683F
:10E4D8000A685A4892FBF3F25C4996FBF3F3F9F7A2
:10E4E8009EF9FEF725FA0320FDF76DF85348584EBC
:10E4F800FCF7ECFF574B58491A885048F9F78FF941
:10E50800FEF702FA0420FDF75EF84C48FCF7DEFF40
:10E51800524B53491A884948F9F781F9FEF7F4F93B
:10E5280004210A20FDF75BF84448FCF7CFFF4D496A
:10E53800E26A4248F9F773F9FEF7E6F90520FDF7B4
:10E5480042F83E48FCF7C2FF7268B36846493B4848
:10E55800F9F765F9FEF7D8F905210A20FDF73FF824
:10E568003648FCF7B3FF3369F26840493348D21A9A
:10E57800F9F755F9FEF7C8F90620FDF724F82F48F2
:10E58800FCF7A4FFB2683A492C48F9F748F9FEF7B6
:10E59800BBF906210A20FDF722F82848FCF796FF68
:10E5A80034492648152207F02DFEFEF7ADF907205D
:10E5B80016E7F37843F00203F370002D2FD12E4BAA
:10E5C80093F82030052B9BBF2C4A9B183F251D7FB5
:10E5D80000211220FDF703F82846FCF75CFF132002
:10E5E8000021FCF7FCFF264B1B78002B254B1B78E2
:10E5F80014BF72202120002B18BF5220FCF74BFFBC
:10E6080014200021FCF7EBFF94F83050074B585DBD
:10E61800013505F00305FCF73EFF84F8305003B0E0
:10E62800BDE8F083E42F00200C2A002069B6010819
:10E63800A5110020D81900206EB60108152A00205F
:10E64800DE190020E0190020809698007FB60108A6
:10E65800B4070020DA1900208CB601085C110020EC
:10E6680094B601089BB60108A2B60108ABB601082A
:10E67800B2B60108C4020020C4330020089501087E
:10E68800430F0020A80F002010F80A3C0133DBB22A
:10E698000A2B84BF10F8131C044A00F80A3C82BFF6
:10E6A800002322F8113000F80A3C7047103300208C
:10E6B800334A136C90681944081A40F68C23984220
:10E6C80070B513469160D06051603BD9127893F9C8
:10E6D80045108A4210460BD1111F082908D893F813
:10E6E8004610182901D8013103E083F8442002E0DC
:10E6F800002183F8461093F944402149A24219D1D8
:10E7080091F84740B4B10C310024944206DA1D4D0B
:10E7180051F8046F25F814600134F6E70C2805D089
:10E728001849002421F810400130F7E7164801780D
:10E738000131017083F84520002201211A7083F805
:10E74800471070BD92F84710C9B1A0F2EF2440F20B
:10E75800DA518C4208D811780B2905D80B1D0131E4
:10E76800117042F8230070BD002283F84720074B40
:10E7780003F13002002143F8041F9342FAD170BD1F
:10E788003001002010330020340600203C01002016
:10E79800024A136C01331944116470473001002098
:10E7A800024B53F820301B6819607047A42B0020D7
:10E7B800064B53F820301A681B89A1F57A71594322
:10E7C8004FF47A7391FBF3F111607047A42B00208A
:10E7D800054B98420CBF054A054A138801339BB282
:10E7E80013800020704700BF00540040F010002044
:10E7F800F210002038B510F80E2C50F8043C0446EE
:10E808005AB9012200F80E2C20F80C1C997A1868C5
:10E818000222BDE83840FDF76FBA30F80C2C20F81A
:10E828000A1C891A89B220F8081C084A10F80F0C2B
:10E83800002522F8101004F80E5C1868997A2A4608
:10E84800FDF75AFA04F8065C38BD00BF1033002003
:10E85800044B53F820301BB107289CBF1B68196074
:10E86800704700BF58020020074A13689B060AD564
:10E87800064B00211970064908684FF6FE730340DD
:10E888000B60202353607047000002401E340020B4
:10E898001C0002402DE9F047664D2B6866490A784E
:10E8A800581C02F0FF068E460AB10346F6E72B60B5
:10E8B800687BAB6895F80C80AA7B374639B220296B
:10E8C80000F09B80DFF880C10CEB81033CF821103D
:10E8D800DC789B78C3F1FF039BB2002B65D0C3F1B2
:10E8E800FF0363434FF03C0C1B12B1FBFCF9B9F179
:10E8F800050F5DD8DFE809F0030B1A293A4AE01A38
:10E90800DAB24143B1FBFCF01044C0B251E0B1FBB4
:10E91800FCF00CFB101189B2DAB2C1F13C01E31A28
:10E928004B432046B3FBFCFC94442CE0B1FBFCF0C9
:10E938000CFB10115FFA83F8E21A89B24A43B2FB62
:10E94800FCF24244D2B2204632E0B1FBFCF90CFBA7
:10E95800191189B25FFA83F8E01AC1F13C01484302
:10E96800B0FBFCF04044C0B2224621E0B1FBFCF809
:10E978000CFB1811D8B289B2E31A01FB03F2B2FBFF
:10E98800FCFC224684445FFA8CF412E0B1FBFCF8EC
:10E998000CFB181189B2D8B2C1F13C01E31A4B4300
:10E9A800B3FBFCF20244D2B203E02246204600E068
:10E9B80044464FEA042C4CEA004C4CEA020C17235C
:10E9C80006F117014FF0010808FA03F8C91A18EA06
:10E9D8000C0F89B2DFF8748014BF4FF011094FF0A3
:10E9E800090913F1FF3308F80190E9D21836013705
:10E9F800B6B2BFB2114BA04660E7AA73AB60104A2B
:10EA0800E98001238EF800300E4985F80C8040F229
:10EA18002A336873AE80536000234B620B889BB225
:10EA280043F001030B80136843F001031360BDE852
:10EA3800F08700BF402A00201E3400204C2A002006
:10EA48001C000240002C0140920E0020D902002038
:10EA580073B506460D46002401232A88A3401342B5
:10EA68001AD0AA78009302F003038DF80430EB78EB
:10EA7800022B03D0032B0CBF032301238DF8053091
:10EA88003046C2F301136946C2F381028DF806309D
:10EA98008DF80720FDF708FE0134102CDCD102B0F8
:10EAA80070BD2DE9F04F734EF57B07460C4687B0D5
:10EAB80011469A4600686B1C914622464FF0020B9D
:10EAC800F37301F0C7F93B897868ADF8043001A900
:10EAD8008DF806B08DF807B0FFF7BAFF0023ADF840
:10EAE8000A30ADF81230ADF8163070230193BA7AB7
:10EAF8003C68CDF80CA0012306F110082D01ADF8F3
:10EB080008304FF48073A844ADF810B0ADF8143055
:10EB18000C2A7ED8DFE802F0077D7D7D0F7D7D7DA4
:10EB2800387D7D7D5E00204601A9FDF70DFCA369B7
:10EB380043F0080326E0236A4F4823F010032362BA
:10EB4800236A6168A26922F0807222F4E642844254
:10EB580042F4E04206D000F50060844202D043F05F
:10EB6800300307E023F0E00321F4406143F0300371
:10EB780041F480616160A261C4F838A02362A3698E
:10EB880043F40063A36144E0236A3B4823F48073A1
:10EB98002362226A6168E369844223F0730343F0C5
:10EBA800700306D000F50060844202D042F440723F
:10EBB80007E022F4606221F4405142F4407241F4CB
:10EBC80080516160E361C4F83CA02262E36943F0CC
:10EBD80008031DE0236A284823F480532362226A2D
:10EBE8006168E369844223F4E64343F4E04342F472
:10EBF800405203D000F50060844201D141F48041C5
:10EC08006160E361C4F840A02262E36943F40063F1
:10EC1800E3613A7B3B681AB15A6C42F400425A6489
:10EC28001A8892B242F001021A80BA7A0C2A18D8CD
:10EC3800DFE802F0071717170B1717170F17171723
:10EC48001300721903F134010AE0721903F1380153
:10EC580006E0721903F13C0102E0721903F1400168
:10EC6800116135444046A5F818906B6107B0BDE8BE
:10EC7800F08F00BF402A0020002C0140F8B53A4E22
:10EC88003A4C4000C7B24FF420453068C4F8D05021
:10EC9800D0F818E01EF4004F05D0AE46013DBEF195
:10ECA800000FF5D116E0D0F804E0314D0EEA050565
:10ECB80045F490353D4345604FF42045C4F8D050A5
:10ECC800D0F818E01EF0020F2DD1AE46013DBEF17E
:10ECD800000FF5D1C4F8D0501FE02946013D0029A6
:10ECE800F8D081694906F8D5C4F8D050204945685C
:10ECF800294041F0007141F4105141EA0241394381
:10ED080041604FF42041A2B1306885696D071ED477
:10ED180011F1FF31F9D2C4F8D010FFF759FD0030D6
:10ED280018BF0120F8BD4FF420458162C4F8D050C7
:10ED3800D7E73068C4F8D0100B46826992060CD425
:10ED48001A46013B002AF8D1C4F8D030E5E7416AF9
:10ED580003F8011B013AD2B2D3E7C4F8D03020231C
:10ED6800C3610120F8BD00BFEC100020402A00203C
:10ED7800009800FC400070B5C5B23248324B0068BC
:10ED88004FF42044C3F8D0408669360404D526469B
:10ED9800013C002EF8D113E046682C4C344044F076
:10EDA800807444F490342C4344604FF42044C3F8F6
:10EDB800D0408669B60729D42646013C002EF8D1F2
:10EDC800C3F8D0401CE02146013C0029F8D08169F5
:10EDD8000E06F8D544681D49214041F0007141F400
:10EDE8008031294341604FF42041C3F8D010846931
:10EDF800A40711D40C460139002CF8D1C3F8D0105F
:10EE0800FFF7E6FC003018BF012070BD4FF4204426
:10EE18008162C3F8D040DAE782624FF42042C3F837
:10EE2800D0208169890606D41146013A0029F8D113
:10EE3800C3F8D020E4E7C3F8D0202023C361012021
:10EE480070BD00BFEC100020402A0020009800FC94
:10EE5800034B4FF4004208B19A6170471A85704716
:10EE680000080048034B4FF4004208B11A85704768
:10EE78009A617047000800482DE9F04F2DED028B8C
:10EE880085B006460393894B1B889807914636D56B
:10EE9800109B8748DC89B0F900301B1B03F2F3157F
:10EEA80040F2E632954203D8002BB8BF5B4201E03E
:10EEB8004FF4FA73B0F90220121B02F2F31440F275
:10EEC800E630844203D8002AB8BF524201E04FF42A
:10EED800FA729342B8BF1346C3F5FA73052293FB3F
:10EEE800F2F30A22643B5343327FD2105343642225
:10EEF80093FBF2F3134423EAE373DBB200E06423E9
:10EF08000093CB1C0293B2460024029BDFF8C08119
:10EF180013F8015F0293022C4FEA440705D1B8F9B0
:10EF280004201B3555436D114AE0624938F8143006
:10EF380031F91410022013FB0011C9F100039942A2
:10EF480003DB49450B46A8BF4B465B4931F907B07F
:10EF5800CBEB030B039B33F914309B4403F0FAFD0E
:10EF680088B107EE90BA554BB8EEE70AB2EE048ABC
:10EF7800185D80EE080A02F0F1FB20EE080AFDEEAB
:10EF8800C07A17EE90BA494B1988CA0714D438F9D1
:10EF980007301B355D438B074FEA251510D5B37C29
:10EFA8009DF9002003FB0BFB02FB0BFB64239BFB7F
:10EFB800F3FB05EB2B1503E0357A05FB0BF52D115B
:10EFC800DFF810E13E4B0422DB5F93FBF2F314F809
:10EFD8000E2090469AF80120EB1A5A4341464A43BC
:10EFE800642192FBF1F2D2110192364A9AF80B5041
:10EFF80010880EF1040C00FB03F25CF82410D21206
:10F0080005FB0215B5F5001F2F4AA8BF4FF40015E0
:10F018000EF110019542B8BF154651F8242041F869
:10F0280024309A1A00094FF6FF7396F85010B3FB74
:10F03800F0F0424393114CF824504FEA840B6D13BF
:10F0480000EE103A59B10EF11C00B8EEC00A00EB00
:10F05800C400DEED0D0AF8F7C3F9BDEEC00A9AF850
:10F0680015300199019810EE102A534342465A432D
:10F078006918642392FBF3F3144A1B121944D15301
:10F0880002F1080101344BF8010002F114012032A9
:10F09800032C4BF801504BF802300AF1010A7FF4B7
:10F0A80034AF05B0BDEC028BBDE8F08F9C1A002090
:10F0B8002030002018340020DC2F00202C95010877
:10F0C80014110020E81000200000E0FF4C2B002065
:10F0D800D8110020142B002010B5447800780022A5
:10F0E80002FB02F3193B634303F6C413534340F690
:10F0F800C411434393FBF1F3034921F81230013261
:10F10800072AEDD110BD00BF782B00200430114B29
:10F1180033F91000B0F5617F10B506DB40F6330314
:10F1280098420246A8BF1A4601E04FF461720C7873
:10F13800192340F2833013FB0404944207DA497818
:10F1480013FB01039342B4BF0020012010BD00202F
:10F1580010BD00BF2030002010B500F15003027828
:10F168008A4203D18478C278944204D30430984206
:10F17800F5D1002010BD012010BD0B4B1B6813F406
:10F18800805F0A4BB3F9063005D0C089421A934212
:10F1980007DD084400E0008A8342B4BF0020012054
:10F1A80070470120704700BFE42F00202030002066
:10F1B8001FB5094B1B681B030AD58DF804000123F2
:10F1C8000D2001A98DED030A8DF80530F9F7D2F865
:10F1D80005B05DF804FB00BFE42F00201FB5084B05
:10F1E8001B681B0309D58DF80400029100230D202C
:10F1F80001A98DF80530F9F7BDF805B05DF804FBF5
:10F20800E42F002010B50A4A0A4B11689B6800BF1A
:10F2180012689142F7D1084A546F4FF47A7000FB94
:10F2280004F2D31AB3FBF4F300FB013010BD00BFA6
:10F238000830002010E000E0142B002038B5044608
:10F24800FFF7E0FF0546FFF7DDFF401BA042FAD3BA
:10F2580038BD10B504462CB14FF47A70FFF7EEFFB5
:10F26800013CF8E710BD024A136801331360704788
:10F2780008300020054B9A6F10B51C4602B1904724
:10F28800E36F13B1BDE81040184710BD142B0020E0
:10F29800014B1B68184700BF0434002010B500203C
:10F2A800FFF7F6FF074B00241C7003F02DFC064BFC
:10F2B80083F88040C3F88440A3F88840C3F88C40A2
:10F2C80010BD00BFE8330020142B002010B510B982
:10F2D800BDE81040E2E700230C225A430C4C1119F8
:10F2E800125D824203D00133102BF5D110BD094BBA
:10F2F800D3F88C0018B14A784078824206D20022AE
:10F30800C3F88C10A3F88820C3F8842010BD00BF70
:10F31800C0980108142B002010B540001428A8BF7D
:10F3280014200023074A022199540B4499181424E5
:10F33800834201F8014CF5DBFF21D1540F20BDE8D1
:10F348001040C3E7743000202DE9F84307460B242A
:10F35800013C35D01D4B08229A617D1C32264FF0A6
:10F368000508DFF86890B9F814309BB283F00803F9
:10F37800A9F814300120FFF78BFF3046FFF769FF2B
:10F38800B9F814309BB283F008030020A9F81430B0
:10F39800FFF77EFF3046FFF75CFFB8F1000F08D09B
:10F3A800B8F10108DDD14FF4FA70FFF752FFFA26E1
:10F3B800D7E7013DD5D14FF47A70FFF74AFFC7E789
:10F3C800034B044ADA60BDE8F88300BF0004004834
:10F3D80000ED00E00400FA0506498B6F0A4623B1E8
:10F3E800CB6F0BB10020AFE7012302EB83039867D3
:10F3F800704700BF142B002003685B691847036837
:10F408001B6918470368DB68184703689B68184737
:10F4180003685B68184703681B6818472DE9F84FAD
:10F42800B0F90230934218BF00232DED028B18BFAC
:10F438000370057804460E469146002D40F08B80F7
:10F4480007EE902A9FED770AF8EEE77AB6EE008A83
:10F4580027EE800ADFED747A20EE270AA04620EE18
:10F46800080A07F0E3F8DFED716A60EE266AB7EE86
:10F47800006AB0EE667AA0EE007A40F2DC5363656B
:10F48800D0EE006A1023A4F8523037EE067A76EEF2
:10F49800866AC6EE077A1823A4F85030274684ED0A
:10F4A800046A27EE807A27EE007A77EE075A84ED11
:10F4B800017AC4ED025A70EE005A84ED037AB8EE70
:10F4C800007AA5EE807A27EE877A67EEA67A84ED31
:10F4D800057AC4ED067ADFED567A98ED047A27EEC0
:10F4E800277AF0EE678AB5EEC07AF1EE10FA4CBFD3
:10F4F80077EE487A77EE087A013517EE900A03F02E
:10F508009DFBD8ED017A67EEA87AC7E90E01F5EE02
:10F51800C07AF1EE10FA4CBF77EEC87A77EE887AA7
:10F5280008F1040817EE900A03F088FB032DC7E9D9
:10F53800080107F10807CED1A6F2DC531B042367A4
:10F54800E3676367C4F88030A367C4F88430012395
:10F55800A4F802902370D4F85490B4F95280636AE6
:10F56800276A206FE26FD4F840C0D4F88010C4F83E
:10F578008020C9EB060606FA08F64FEAE67B7343D5
:10F5880007FB0B332667A7FB06671F44636C656F91
:10F5980060674FEAE27B53430CFB0B3EACFB022354
:10F5A8007344B61A67EB0307E36AA26AC4F88410C7
:10F5B8004FEAE07B434302FB0B3EA2FB002373446C
:10F5C800B6185F41E36CA06CB4F95020A5674FEA08
:10F5D800E17B4B4300FB0B33A0FB01011944636B38
:10F5E800361A206B4FEAE57B05FB03F300FB0B3370
:10F5F80067EB0107A0FB050119448019794103F065
:10F60800F3FA08F1FF3201239340E067C01841EB99
:10F61800E371424603F0E8FABDEC028B4844BDE8CA
:10F62800F88F00BF6F12833ADB0F4940F404B53FEF
:10F638000000804B2DE9F8430024244B93F8C06068
:10F64800E0B2B0420DD203EB8003214AD3F89030E8
:10F6580032F810101BB10B2801D8DB689847013429
:10F66800EBE71C4B1B685B032DD500242346E2B255
:10F67800B24228D2DFF8549009F190074FEA840883
:10F6880057F8242055689D4215D0284600F05AFCAA
:10F69800EFF31283502282F3128828216A6A01FB51
:10F6A80000900132C0F8E8206A6942F001026A61FC
:10F6B800DBB283F3118857F808301B6800221A6000
:10F6C80001342B46D3E7BDE8F88300BF142B002094
:10F6D80034110020E42F002008B50E4B1B6813F4EA
:10F6E800805F0D4B14BFD3F8DC21D3F8E02193F8E9
:10F6F800C01092880023D8B2884204D2074820F864
:10F7080013200133F7E7FFF795FF3220BDE80840E3
:10F718009FE500BFE42F0020142B002034110020A7
:10F728000A4B1A680A4B30B502F48052D3F8DC4110
:10F73800D3F8E05100230AB1A18800E0A988054860
:10F7480020F8131001330C2BF5D130BDE42F002025
:10F75800142B00204A30002070B5124D0024214699
:10F7680005F2E510702285F8E44106F0DAFC21463E
:10F77800D5F858320B4A0B4493F9020080B102F2D3
:10F78800E5141E680E5108199C8884809B79837142
:10F7980092F8E43107310133702982F8E431E7D176
:10F7A80070BD00BF142B0020094B1A680E2303FB01
:10F7B8000020437AFF2B07D0064A12789A4203D9D1
:10F7C800054A32F8130000E0808800B2704700BF95
:10F7D800082A00208C2800202030002038B5294C29
:10F7E8002DED048B94ED978AB0EE480A0546F8F79C
:10F7F800BDF8F0EE408AB0EE480AF8F754F894EDF8
:10F80800989AB0EE408AB0EE490AF8F7AFF8F0EEF1
:10F81800409AB0EE490AF8F746F895ED017AD5ED29
:10F82800027A95ED006A68EE676A27EE088AE7EEC5
:10F83800286A68EE000A67EE807AE6EE290AB0EEDA
:10F84800660AE7EEA80A06F07DFFDFED0F7A20EEE4
:10F85800270ADFED0E7A80EE270AD4ED997A30EE8A
:10F86800270AF2EE047A80EE270A06F069FEBDEC5C
:10F87800048B83B21A0444BF00F5B47083B218B283
:10F8880038BD00BF142B00200000E144DB0F4940C5
:10F8980001380A4B042804D8DFE800F00507090BF3
:10F8A8000D00074A08E0074A06E0074A04E0074A4D
:10F8B80002E0074A00E0074A1A6070478400002007
:10F8C8002197000881EE0008FD99000805940008BA
:10F8D80091900008498B00086C4B6D4A2DE9F04F58
:10F8E8005E8914684FEA062AB4EB0A0A9C884FEA34
:10F8F80004481C894FF000054FF0000B65EB0B0B1B
:10F90800A4FB0A6704FB0B77F40944EA476418EB85
:10F9180004065C884FF000094FEAE7154FEAC4383F
:10F92800DC8849EB050787B0CDE90467A4FB0A67C3
:10F9380004FB0B77340A44EA076418EB04064FEA21
:10F9480027259C894FF0000949EB0507CDE9006799
:10F95800AAFB046704FB0B77F40D44EA472414F56B
:10F96800FA664FEAE75545F10007B6F5FA6F77F101
:10F978000003CDE90267964667DAA4FB046704FB37
:10F9880005F34FF0050C07EB4307DDE90489A6FBF7
:10F998000C230CFB07335F104FEA3206B8EB06085E
:10F9A8004FEA920669EB070946EA83769F10DDE97C
:10F9B8000023921B63EB0703DDE90267CDE900230F
:10F9C800344A4FF0FF33964277EB0303CDE90489BD
:10F9D80028DA40F6AC52A4184FF000035D4104FB4E
:10F9E80005F3A4FB044505EB43056FF006026642E8
:10F9F80002FB0566A4FB0223334418EB020649EB1D
:10FA08000307CDE904670B26A4FB062306FB053391
:10FA1800DDE900455B104FEA3202A41A65EB0305E5
:10FA2800CDE900450AFB0BF3DDE90245AAFB0AAB69
:10FA38000BEB430B4FEADA7242EA4B02A41A4FEA85
:10FA4800EB7365EB0305CDE90245DEF80440009B46
:10FA5800019DA4FB032304FB05334FEA52584FEAE8
:10FA6800635948EAC328DDE90423B8EB020269EBCD
:10FA780003039946D30B43EA494300B1036009B134
:10FA8800029B0B6007B0BDE8F08F00BF8602002024
:10FA98007C2D002024FAFFFF054B1A7A02F0FF01A3
:10FAA80022B10122027000221A7270470170704759
:10FAB8007C2D0020772048210122FFF75BB97720B1
:10FAC80058210122FFF756B907B5002101AB0322DF
:10FAD8007720FFF7D3F89DF805309DF804001B0246
:10FAE80043EA00439DF80600184303B05DF804FBA1
:10FAF80008B5FFF7E9FF014B586008BD7C2D0020D1
:10FB080008B5FFF7E1FF014B186008BD7C2D002008
:10FB180013B506220446432168206B46FFF7AEF86A
:10FB2800A8B19DF800209DF8013043EA0223238004
:10FB38009DF802209DF8033043EA022363809DF874
:10FB480004209DF8053043EA0223A380012002B077
:10FB580010BD13B5062204463B2168206B46FFF70B
:10FB68008DF8A8B19DF800209DF8013043EA0223E2
:10FB780023809DF802209DF8033043EA0223638026
:10FB88009DF804209DF8053043EA0223A380012054
:10FB980002B010BD094B1B681869094B20F01F0201
:10FBA80010B5D258012400F01F0304FA03F31A42D7
:10FBB80003D0FCF77FFA034B1C7210BD80020020B3
:10FBC800140401407C2D0020F0B52B4D6B7A85B0D4
:10FBD800002B4ED1294C2368002B4AD01A68284E96
:10FBE80012B171690A4372619A88ADF80020022245
:10FBF80098688DF80320694600228DF80220FEF7E8
:10FC080027FFB3691D4F43F00103B3612368187BD5
:10FC1800197DFCF7FFFA2268936894881B8A1C40B8
:10FC280002D001236B7224E01648FFF7D5FB3B682E
:10FC38001869FCF73FFA3B688DF80C401B69029382
:10FC480008230DEB030001268DF80D308DF80E60AA
:10FC580001F016FD3B688DF806405B7D8DF8043099
:10FC680001A803238DF805308DF8076001F0EAFC40
:10FC7800D7E705B0F0BD00BF7C2D00208002002032
:10FC8800001002409DFB000808B5FFF79DFF6B219F
:10FC980080226820FFF76EF86420FFF7DAFA6B21FC
:10FCA80003226820FFF766F8124B19211A7868209A
:10FCB800FFF760F80F20FFF7CCFA0F4B1A211A78DC
:10FCC8006820FFF757F81B2118226820FFF752F821
:10FCD8001C2110226820FFF74DF8372100226820E8
:10FCE800FFF748F8682038210122BDE80840FFF7EF
:10FCF80041B800BFB40200200000002008B5FFF79B
:10FD080063FF074B1B7813B1012B03D008BD4FF4D9
:10FD1800006201E04FF48052024B1A8008BD00BF18
:10FD2800840200202C0000202DE9F0410369C768F7
:10FD380005460E461F40002F35D0B7FA87F24FF020
:10FD48000043D340DB432B611F40A2F11B03042B6C
:10FD5800F1D8DFE803F0221F1C190300746A24B1EC
:10FD6800013C0023A4B2736201E0EC6AA4B2D6F8A5
:10FD78002080B8F1000FDED0D8F800304046214688
:10FD88009847D8F80480F4E73068696B07E0706832
:10FD9800A96B04E0B068E96B01E0F068296C0368BE
:10FDA80089B29847C7E7BDE8F08107B52320FFF778
:10FDB80050FA6820752101220DF10703FEF75EFF56
:10FDC80028B19DF80700A0F168035842584103B0D4
:10FDD8005DF804FB01480249A6E700BF004801405E
:10FDE800C82C0020014802499EE700BF004001409E
:10FDF800782C00200148024996E700BF000800401F
:10FE0800502C0020014802498EE700BF0004004042
:10FE1800282C00204FF08040004985E7002C002066
:10FE280010B5054C05482146FFF77EFF04F1C801CF
:10FE38000348BDE8104077E7D82B0020002C01408C
:10FE480000440140014802496EE700BF002C014010
:10FE5800D82B0020224B10B5224C5A43224BB3FB1F
:10FE6800F2F203880139013AA04289B292B29BB2F8
:10FE78000ED004F50064A0420AD0B0F1804F07D03C
:10FE8800A4F59834A04203D004F58064A04202D1BE
:10FE980023F070039BB2154CA04206D004F5806491
:10FEA800A0421CBF23F440739BB203800D4BC16278
:10FEB800984202850FD003F5006398420BD003F5F2
:10FEC8004063984207D003F58063984203D003F556
:10FED8008063984201D1002303860123436110BD4A
:10FEE80040420F00002C014000A24A0400100040CC
:10FEF80073B505460068FFF7ADFF2A6813889BB203
:10FF080043F001031380EB7A8DF8043001240026B6
:10FF180001A88DF805408DF806608DF8074001F0BE
:10FF280091FBEB7A1B2B0BD1192301A88DF8043018
:10FF38008DF805408DF806608DF8074001F082FBCA
:10FF480002B070BD134B800A984220D00AD84A3BB1
:10FF5800984212D00133984211D0B0F5801F14D1C5
:10FF6800012070470C4B98420BD0013398420AD0BD
:10FF7800023B984209D104207047022070470320B1
:10FF880070470520704706207047FE207047002004
:10FF9800704700BF4B00100051001000F8B504680E
:10FFA800064620460F461546FFF7CCFF06284BD8D5
:10FFB800B27A910847B902238B40D4F80CE0DB43AE
:10FFC8009BB203EA0E03E3600A23204A03FB0013F3
:10FFD80042F82370043342F8235015463FB1B17AF2
:10FFE800E268890802238B409BB21343E36028220E
:08FFF80002FB00522032EFF37E
:020000040801F1
:100000001286502383F3128803B203EB8303DB00D1
:1000100003F10C011C3329442B4451F8047F17B120
:1000200017600A6804329942F7D100231360F3B2D3
:1000300083F31188282303FB0050036A1BB1E36894
:1000400043F0010303E0E2684FF6FE731340E36000
:10005000F8BD00BFD82B00200148FBF7D3BB00BF81
:10006000882D00200148FBF7CDBB00BFDC2D002010
:100070000148FBF7C7BB00BF302E002010B54B88EE
:10008000DC0641BF2F4B14791B6853F8244044BF52
:100090002D4B43F820404B889B0641BF294B547998
:1000A0001B6853F8244044BF274B43F820404B883B
:1000B0001C070ED5254B0C781B78B3EB141FA1BF82
:1000C000204BD4781B6853F82440A4BF1E4B43F840
:1000D00020404B889B070ED51D4B0C781B78B3EB4B
:1000E000141FDFBF174B54781B6853F82440DCBF44
:1000F000154B43F820404B88DC070FD5154C0B7887
:10010000247803F00F03A342DFBF0E4B14781B6863
:1001100053F82440DCBF0C4B43F820404B885B076E
:100120000FD50B780C49097803F00F038B42A1BF60
:10013000044B92781B6853F82220A4BF024B43F86B
:10014000202010BD042A0020920E0020BF2900208C
:10015000BD290020BC290020BE290020254A2648B0
:1001600026490023F0B5156803700B701C461A462B
:100170002E1976884EB92F5D3FB9037000230A709F
:100180004B7007781C461A460CE0360548BF013212
:1001900004F1040403F1010348BFD2B2802CDBB2A6
:1001A000E6D1EAE7E0B2B8420CD215F8240006091D
:1001B0009E4200F00F00A8BF731C9042A8BF421CD3
:1001C0000134EFE78A704B70C2F3470102F001027D
:1001D0000A444C1E0A490B480A70C3F3470203F055
:1001E0000103134404700849501E084A0870137034
:1001F000F0BD00BFA01A0020B4290020842E0020EA
:10020000BE290020BC290020BF290020BD290020D4
:100210002DE9F04FC24BDA682DED028B1A61C14A0D
:100220001168D960C0490B6843F020030B60BF4BD5
:100230001978012990460CBF002201221A70BC4B8C
:100240001A78910789B040F13D83BA4909780429A9
:1002500040F23883B849097801F0040101F0FF0049
:1002600011B922F001021A701B78DB0702D408B121
:10027000FAF7F4F9B149CA78531C052293FBF2F25C
:1002800002EB82029A1AAE4BCA701B78039392005B
:100290000023AC4CDFF8CCC2DFF8D8925CF8231016
:1002A00091FBF9F504F1080004F1100640F8235021
:1002B000A54844F8231000FB051142F2107091FB91
:1002C000F0F080B226F813004FF0140E04F114067B
:1002D00004F13C0A0EFB036E5AF823605EF80270CC
:1002E0004EF80210F61B314444344AF82310052618
:1002F00091FBF6F109FB051144F82310039C012C36
:100300004FEA830BE24605D10238B0F5797F98BFFA
:100310004BF80C100BB90123BBE7884CD8F8003020
:10032000226D9FED8A7A8A4E8A4D9B1A07EE903A8B
:10033000F8EE677AD8F800302365C7EE877A7C4BF1
:100340001B78B7EE008AF4EEC87AF1EE10FA58BFC7
:10035000F0EE487A13F00103C4ED157A12D005AA25
:1003600000927D4B06AA01920CCB9AE80300FAF7A3
:1003700073F86421059A069BB2FBF1F293FBF1F34B
:10038000328000E033802B8094F858306B48002B8B
:100390003BD0D0ED157AC26DDAF80030C8EE276A8E
:1003A0009B1A026E022507EE103AB8EEC77ADAF809
:1003B000043027EE267A9B1AFDEEC77AB0F9662044
:1003C00017EE901A07EE903A644BB8EEE77AD3ED49
:1003D000007A67EE277A67EEA67AFDEEE77A17EEE7
:1003E000903A02FA83F3B0F9642093FBF5F302FA32
:1003F00081F29BB292FBF5F292B2A0F86A30A0F8BB
:100400006820A0F86630A0F86420012384F85830F2
:10041000534BDAF804101B88DAF80000474D514EB0
:10042000216603F03003E065002B00F04B8205F1FC
:100430007403009305F178030193EA6E2B6FFAF7CA
:100440000BF872682B6F9B1A07EE903A434B326899
:1004500093ED007AEB6EF8EEE77A9B1AEB67384B78
:1004600067EE877A1B78FDEEE77A012BC5ED207ADF
:1004700003D0022B00F0DF8024E2D5ED287A3A4B3E
:10048000D5ED215A95ED255A95ED156A95ED264A3B
:10049000D5ED274A35491D68B1EE677ABDEEC77ABA
:1004A000FDEEE77A17EE10EA17EE90CA0020304A08
:1004B00091ED007A52F8207007EE907AF8EEE77A24
:1004C000A2F1140367EEA57A33F81060FDEEE77A27
:1004D000283217EE903A9B1B9BB222F810301BB2C9
:1004E00007EE903AF8EEE77A3B4467EE857A4400EF
:1004F000FDEEE77ACDED037A07EE903AF8EEE77A73
:10050000BDF80C8067EE847AA7EE867AFDEEC77A96
:1005100017EE902A724531DB6245A8BF62462EE095
:10052000B407002008300020D41900205E110020FC
:10053000D8190020DE1900201F340020842E00204E
:100540001C100020882E0020806967FF00007A447C
:10055000521A0020541A0020601100207800002058
:100560009C1A0020E01900202010002050100020CC
:10057000002F002080969800DB0FC940724607EEDE
:10058000902AF8EEE77A5FED046AC1ED007AFDEE9D
:10059000E77A313617EE903A43449AB2AB78D1ED10
:1005A000027A07EE103AB8EE477A4B684F6027EEB2
:1005B000267AFB1A88EE077AB6B2622E06EE903AD9
:1005C000F8EEE66A37EE067AC6EE866A86EE077AB7
:1005D00076EEE76AE7EE267AC1ED047AC1ED027A9B
:1005E0000FD964EEA77ABA4EFDEEE77A17EE903A8D
:1005F000B3F5FA6FA8BF4FF4FA63B342B8BF3346FE
:1006000000E0002313441BB240F6B8329342A8BF67
:100610001346B04A9342B8BF1346AF4AA352AF4AFB
:10062000142303FB002351F8142B1A60002840F018
:10063000498101203BE7AA4BD5F874801F68D4F8A4
:1006400078903E89DFEDA78A4FEA58039E4228BF83
:100650001E46B5F8A8301AB29642C3BFD5ED157A3A
:100660009FEDA17A67EE877AB6B2C1BFFDEEE77A59
:1006700017EE906AF618B6B2C8BFA5F8A860D4F80D
:10068000AC50C5EB09052846F9F72AFF0028D8BF6A
:10069000404241F293129042CCBF0020012088B327
:1006A00007EE905AB8EEE70A20EE280AF7F7FFF8AF
:1006B00007EE908AF8EE677A40F6B83320EE270A04
:1006C000FDEEC07ACDED037ABDF80C20A4F8B02081
:1006D00012B29A42A8BF1A467E4B9A42ACBF09EBAF
:1006E00002034B4448F6A042934203DDA3F50C43BA
:1006F000A03B04E0002BBCBF03F50C43A033C4F8BF
:10070000B43001E0C4F8B490D4F8B450C5F50C533B
:10071000283307EE903AF8EEE77A67EEA88AB0EE53
:10072000680AF7F727F98DED070AB0EE680AF7F7C0
:10073000BEF8D4ED317AD4ED2E4AD4ED155A94EDAD
:100740002F4A94ED305A65498DED060AB1EE677A6D
:10075000BDEEC77AFDEEE77A0DF1180E17EE10AA7E
:1007600017EE90BA0020614AFEEC016A32F91030AF
:10077000DFF88C9107EE903A07EE106AF8EEE77A10
:10078000B8EEC77A3C32D6EE877A4FEA400CFDEEDF
:10079000E77ACDED037ABDF90C30B3F57A7FA8BFC7
:1007A0004FF47A734B45B8BF4B461FFA83F922F8D2
:1007B00010900FFA89F207EE902AF8EEE77A27EE0A
:1007C000A47ABDEEC77A8DED037A27EE847AD1ED57
:1007D000007ABDF80C90E7EE257AFDEEE77A17EE89
:1007E000902A524503DB5A45A8BF5A4600E05246BC
:1007F00007EE902AF8EEE77A9FED3D6AC1ED007AA8
:10080000BA7891ED027A06EE902AF8EE666A4A68A6
:100810004B6066EE866A9A1AC8EE266A143106EEB6
:10082000102AB8EEC66A76EEA56A86EE256AC5EE8F
:10083000A66A36EE476AA6EE867A01ED017A01EDE8
:10084000037A25EE077ABDEEC77A17EE103ABDEEB1
:10085000E77A4B4417EE102A13441BB240F6B83225
:100860009342A8BF13461B4A9342B8BF13461A4A85
:100870002CF802301F4A142303FB0023C3ED007A37
:1008800008B901206FE73B7923B1642395FBF3F5A9
:10089000194B1D803B8898450DD9D4F8AC30A06F1A
:1008A000C01AF9F71DFE80EAE072A2EBE07242F294
:1008B00010739A4206DD114B01221A700E4BB4F8E8
:1008C000C8201A8009B0BDEC028BBDE8F08F00BFD4
:1008D00030F8FFFF48F4FFFFA4100020781000203C
:1008E00020100020D30237390000C842EC2E00202F
:1008F000DB0FC94050100020181000201C100020F1
:1009000018FCFFFF10B5134B93F8DC37012B0146A1
:1009100019D1114B114C1878421CD2B21A70120620
:1009200044BF00221A700E4A1B7812782154934259
:1009300036BFC2F180029B1A9B183F2B09D9BDE834
:100940001040FAF711B8074BBDE810401868FEF7E1
:1009500066BD10BDE0110020502F0020522F002056
:10096000512F002098300020F0B5974D2B78023B96
:1009700087B0082B00F28A81DFE813F009002E000F
:100980004F0064007C008E000A016E0179018F4BDC
:100990008F4C1A68636864339A4240F2778100266C
:1009A0008C4B8D4A1B789E420ADA2368884FD05CB4
:1009B00030B1FFF7A7FF3B68013301363B60EFE73B
:1009C0002168834B525C002A40F060811A604FF02E
:1009D000FF325A6003231BE0262300937F4B0193D1
:1009E00003F10C0202924920A3F10A0250210233C2
:1009F000F7F7E0FF002840F04981794B1B6813F0BE
:100A000080024FF0FF31724B04D083E803000423CF
:100A10002B703BE11A6059602AE0724A02230021E0
:100A2000009301910291482002F10803F7F7C2FFF9
:100A3000002840F02B81664B4FF0FF3218605A605F
:100A40000523E5E707230093674B019303F10C02AD
:100A500002924720A3F1080200210433F7F7AAFF0E
:100A6000002840F013815A4B4FF0FF3218605A6053
:100A70000623CDE75D4A05230021009301910291F1
:100A8000532002F10803F7F795FF002840F0FE809D
:100A90004F4B18600723BBE74D4C236813B96360C5
:100AA000012323604B4B1A7863681344402BA8BF83
:100AB0004023132B636040F3E980454B1B680D2BEB
:100AC00000F2EA80DFE803F060070B0E121923281A
:100AD0002D3134404B51464800F0DEFC51E0454892
:100AE00045493FE045484649464A48E0464B474865
:100AF00093F8DA1793F8DB2741E0434B444893F827
:100B0000B4270C2101FB023393F8B6172AE03E4BC1
:100B10004048B3F8401125E03B4B3F48B3F8421141
:100B200020E03E4B3E4819691CE03E483E4B18E031
:100B30003E4B1B68D80404D5334B3D4893F87811DD
:100B400010E00C2323601FE02F4B3A4893F87C11F0
:100B500093F87D2193F87B3100F008FD11E03648D1
:100B6000364B198800F002FD0BE01D4B1B68190580
:100B70000AD5254B3248B3F88011B3F97E2100F035
:100B8000F5FC6368181A60602368013323607DE018
:100B90002C4B1B689A0114D52B4B1B888BB92B4B04
:100BA0001B6804932A4B0E201B68059304A9F7F7D2
:100BB000E5FB284B4FF480521A8009232B70F7F77E
:100BC00057FCF7F7BDFB61E08C30002008300020B7
:100BD0004C3200208C000020309501089A950108C5
:100BE000E42F00205897010870970108BC9701086E
:100BF000E7B6010804B70108BDA901081CB7010840
:100C0000A8A90108B4A90108E011002033B7010820
:100C100047B7010854B7010866B701085C1B0020FC
:100C200078B701088BB701082C000020343200206F
:100C300098B70108A8B70108C4B7010830320020EE
:100C4000D2B70108F4100020403200203C320020CE
:100C50000034002054320020154B1B78002BAED0FE
:100C6000144B1B689B01AAD408232B70A9E7124BD5
:100C70001A68124B5B68C8339A4203D900F030FB04
:100C80000123C5E600F046FB0028F7D100F012FB77
:100C900060B101232B7009E000F03CFB0028F5D087
:100CA000074B4FF480521A800923B1E607B0F0BD1C
:100CB00038320020F4100020083000204C32002090
:100CC000543200200846FFF71DBE0F4B1A786A2ADF
:100CD00016D15A88B2F5FC6F12D11A79BE2A0FD1FB
:100CE00093F8DD27EF2A4FF000000BD113F8012B0A
:100CF0005040064A9342F9D1B0FA80F0400970475B
:100D000000207047704700BF00F80308E0FF0308A9
:100D10002DE9F04F2DED028BE84C85B000214FF40A
:100D2000FC62204605F001FAE54B04F53B721A60BF
:100D3000E44B00251D70E44B04F2B6721A606A237E
:100D40002370022003236371F6F7E0FE4FF48070F6
:100D5000F6F7DCFE4FF416732022A4F8623184F813
:100D60006621FA236E22A4F8643184F87821BC232A
:100D70000A22A4F8603184F879214FF4FA732B2207
:100D8000A4F86A3184F87B210123212284F85E31A2
:100D900084F87A3184F87C2184F88231232200237C
:100DA00084F87D21C4F820324FF4C872C4F824328C
:100DB000052384F8B457A4F86E51A4F86C51A4F834
:100DC000705184F8545184F8555184F85651A4F860
:100DD0005851A4F85A51A4F85C5184F85F5184F832
:100DE000675184F86851A4F88051A4F87E21A4F8D2
:100DF000845184F81D5284F81C5284F8285284F8D7
:100E00002B3240F2DC53A4F8943140F24C43A4F866
:100E1000963140F26C73A4F8983140F27533A4F81F
:100E20009A3140F6430384F8295284F82A5284F810
:100E30008E5184F88F51A4F89C3122462B462546CA
:100E4000032BCCBF0121002103F1010382F89E1185
:100E500014BF1E217521122B82F89F1102F102028C
:100E6000EED14FF4FA63A5F8C431A5F8C831A5F85E
:100E7000CC31A5F8D03140F27E41052340F27E5EB0
:100E800085F8DE31A5F84011C82340F23A71A5F883
:100E900048E1DFF82CA2A5F8E23140F2EA5E002634
:100EA00001274FF47A791E2019224FF4C8734FF0AE
:100EB000320BA5F84211A5F84AE140F2DC5140F2AC
:100EC000B45E85F89101039085F8DF210192A5F8C1
:100ED000E631A5F846110291A5F84CE185F890613C
:100EE00085F89261A5F8C291A5F8C691A5F8CA91B6
:100EF000A5F8CE9185F8D26185F8DC6185F8DD71C1
:100F000085F8E07185F8E17185F8E47185F8E861AC
:100F100085F8EA71A5F84491A5F84EB1A5F85031CD
:100F2000A5F852B185F8EB6185F8EC6185F8ED71B3
:100F300085F8EE61FAF7EAFFDAF8003003986F738C
:100F40002E73D87218735520019AD8700F205871DB
:100F5000DA712220212298715A740E2053224FF008
:100F6000170E1874DA7635200A224FF0280883F815
:100F700015E083F816E098764FF02D0E5A209A74FB
:100F800001924FF0780C642283F80DE018721A7702
:100F900083F80AC01E7083F8018083F80280DE7532
:100FA00083F804B09E731E76DE735E7683F8098044
:100FB00083F814E04FF4FA7EA3F84EE0DFF820E166
:100FC000C3F838E0C3F83CE0DFF818E1C3F828E0E4
:100FD000DFF814E1C3F834E0DFF810C1DFF810E106
:100FE0009FED3A8AC3F82CC0C3F830C0C3F848E07C
:100FF000F7EE087ADFF8FCC002999F774FF04B0EAE
:1010000083F85080C3ED087AC3ED097A83ED108A26
:10101000C3F844C083F84CE085F8B607A5F8C017BC
:101020004120042185F8B70785F8B8B785F8B96776
:1010300085F8BD6785F8BE6785F8BA6785F8BB6730
:1010400085F8BC6783F85C101521A3F85860A3F8F5
:101050005A60A3F85660C3F860C083F8648083F8D0
:10106000658083F868101A49D9661A4919671A49C0
:10107000596783F878701948FAF786FFDAF8003074
:10108000019A83F811614FF44871A3F8161183F89F
:10109000126183F8138183F8147183F8186185F85D
:1010A000D421C82285F8D5216422A5F8D69185F8E7
:1010B000D861A5F8DA2119461EE000BFE011002032
:1010C000301100204830002058110020000000009E
:1010D0009A99193FF6287C3F3D0A773FF7B80108F7
:1010E0008FC2F53C000060406666663FCDCCCC3ECA
:1010F000000040400000A0400E2202FB06326FF0CC
:10110000170082F81901032082F81A016FF02F00EE
:1011100082F81B01072082F81C016FF0230082F87F
:101120001D01052082F81E0101365A2081F8200198
:1011300081F821016422FF20082E81F81F2181F807
:10114000220101F10E01D7D1002183F88911C821B4
:10115000A3F88A11142183F88C11A3F890211E2181
:101160004FF4967283F88D11A3F892210121282261
:1011700083F88E11A3F894212F4B18EE102A44F80F
:10118000102F9C42F9D12D480021402204F0CDFFC0
:1011900000232B4D2B4C59591A1904330868C2F8F7
:1011A000AC02382BF5D104F50B700021802204F03D
:1011B000BCFF05F13801702204F50B7004F0AAFFA2
:1011C000FEF7CCFF4FF40020F6F7A0FCDAF8006041
:1011D0000125314604F284404FF4CC7284F8DC5788
:1011E00084F8DA5784F8DB5704F094FF04F21C60AB
:1011F00031464FF4CC7204F08DFF134B1B681A6814
:10120000C4F8C2275A68C4F8C6279A68C4F8CA271F
:101210001A68C4F8CE275A68C4F8D2279A68C4F866
:10122000D627022384F8D85484F8703605B0BDEC74
:10123000028BBDE8F08F00BFA01200208C140020AC
:10124000E4970108E0110020581100201549D1F859
:10125000883043F47003C1F88830134B1A6842F0A9
:1012600001021A605868114A02405A601A6822F056
:10127000847222F480321A601A6822F480221A6082
:101280005A6822F4FE025A60DA6A22F00F02DA6229
:10129000186B074A02401A6300229A604FF00063FD
:1012A0008B60704700ED00E0001002400CC07FF83A
:1012B000CCFC00FF074B93F8DC37012B08D1064A22
:1012C000064BD0681B68834234BF00200120704762
:1012D00000207047E01100201C000020280600209C
:1012E00038B5094B93F8DC5765B9084C2068F5F719
:1012F0006AFE074B25601B78022B03D1BDE83840FE
:10130000FAF7C3BD38BD00BFE011002098300020BF
:1013100094300020064B93F8DC371BB1012B05D12C
:10132000F9F722BB034B1868FEF76DB80020704731
:10133000E011002098300020F8B5011F0646002378
:10134000083051F8042F02F120043F2C3BD802F161
:1013500008040F2C06D80232032A04D9002B08BF38
:10136000012300E002238142EBD1012B30680ED033
:10137000022B1AD0736803F003039B0000F00300F4
:1013800043EA0010B36803F00303184317E000F0CA
:101390000F0040F04000FFF7B5FAB068736800F046
:1013A0000F0040EA0310C0B209E000F03F0040F037
:1013B0008000FFF7A7FA3079FFF7A4FA307ABDE88A
:1013C000F840FFF79FBA06F10C0734463A4600256D
:1013D00052F8043D03F18001FF294FEA850510D939
:1013E00003F50041B1F5803F02D245F0010508E068
:1013F00003F50003B3F1807F34BF45F0020545F0EB
:101400000305B242E4D165F03F00C0B2FFF77AFABB
:1014100005F00303022B207807D0032B0CD0012BFF
:1014200013D1FFF76FFA60780FE0FFF76BFA60787F
:10143000FFF768FAA07808E0FFF764FA6078FFF732
:1014400061FAA078FFF75EFAE0780434FFF75AFA01
:10145000BC424FEAA505DBD1F8BD10B50446C0B2C9
:10146000FFF750FAC4F30720BDE81040FFF74ABA6F
:1014700010B504467F2C06D964F07F00C0B2FFF798
:1014800041FAE409F6E7E0B2BDE81040FFF73ABAE6
:10149000430083EAE070EBE72DE9F047304B93F827
:1014A000DC37012B86B0074601D004464AE004F041
:1014B00080FE03A9054606466846F9F765F9039BD1
:1014C000049A029713442B443F2B059519D9002306
:1014D000684603A90322F9F783F9039B3BB9049BF0
:1014E0002BB9204A13705370059BABB301E0F9F799
:1014F00033F9039B049A059E134433447F2B2BD866
:10150000029FDFF86090CA4639461AF8024BC4F1D0
:101510008008B04528BFB0460AEB04004444E4B25A
:10152000424604F0F7FD802C89F8004014D1C8EB46
:101530000606504607EB0801324604F0EBFD89F839
:10154000006009E0254614F8011B21B1064B18681C
:10155000FDF765FFF6E7ED1B284606B0BDE8F0870E
:10156000E0110020502F0020983000200FB407B564
:1015700004AB064953F8042B01930020F6F766F8F4
:1015800003B05DF804EB04B0704700BFC50C010860
:1015900040F2E9330F4A1289920704D4013B9BB20F
:1015A000002BF7D10BE00C4A40F2E93310700949E7
:1015B0000989C9070AD4013B9BB2002BF7D1074A1E
:1015C000138801339BB21380FF2070471078C0B29C
:1015D000704700BF003800400C380040D42F002076
:1015E00030B5174B9B894FF47A733AB311B10D782C
:1015F000013107E0FF2505E0013B9BB24FF6FF7488
:10160000A3420FD00E4C2489A407F5D50D4C2570AC
:101610000B4D2D89ED070BD4013B9BB24FF6FF75A7
:10162000AB42F5D1084A138801339BB2138005E021
:10163000247808B104700130013AD6E7012030BDAA
:10164000003800400C380040D42F00200C4B0D49CE
:10165000DA684378D243C2F30222C2F10402934013
:1016600002781B010A44DBB282F8003303780122BE
:10167000580903F01F0302FA03F341F820307047C2
:1016800000ED00E000E100E0036823F01F0202F13A
:10169000804202F5823270B503F01F011468012305
:1016A00003FA01F124EA0101116002682A4C22F0D8
:1016B0001F0502F01F02295903FA02F221EA020271
:1016C0002A510279016802F1804221F01F0402F5DB
:1016D000823201F01F01155903FA01F1294311511A
:1016E00002681E4D22F01F0402F01F02615903FA26
:1016F00002F221EA020262510268194C22F01F062E
:1017000002F01F02315903FA02F221EA0202417982
:1017100032511029026812D122F01F0102F01F027B
:101720004E5903FA02F232434A51026822F01F0175
:1017300002F01F020859934003430B5170BD01F1A1
:10174000804122F01F0001F5823102F01F020C5887
:10175000934023430B5070BD040401400804014032
:101760000C040140F0B5BE4CA3782DED028B013B7B
:10177000012B85B000F26F81E578854240F06B81E6
:101780002379022B00F06781B64B5B5D6371A3790F
:101790006D00F2EE048A1BB16319B3F9083009E059
:1017A0006319D4ED037AB3F90830F1EE677AC4ED2A
:1017B000037A5B4208EE103A2369A94EB8EEC88A54
:1017C0001A0388EE288A35D5D6ED037AFDEEE77A3E
:1017D00028EE280A17EE903AD6ED057A8DF80A30F1
:1017E000FDEEE77A17EE903A8DF80B3004F0F2FE3A
:1017F000FCEEC07A96ED060A17EE903A20EE280A23
:10180000ADF8083004F0E6FEFCEEC07A96ED070A6B
:1018100017EE903A20EE280AADF80C3004F0DAFE0C
:10182000FCEEC07A0C2017EE903A02A9ADF80E300B
:10183000F6F7A4FDD4ED077A894BF5EE407AF1EE88
:1018400010FA60D1D3ED067AB4EEE78AF1EE10FA21
:1018500004DDDA6883ED068A5A61E8E0F5EEC07AC5
:10186000F1EE10FA40F3E38093F8202042B1022A0F
:1018700000F2DD805A6B83ED078AFA329A63D6E074
:10188000D3ED037A38EE678AF7EE007AB4EEE78A92
:10189000F1EE10FAACBF01210021D3ED0A7A69B153
:1018A0009FED717A27EE877ADFED707AB4EEE77AF2
:1018B000F1EE10FA58BFF0EE477A03E09FED6C7A34
:1018C00067EE877AC3ED0A7A2369654A1B0311D54F
:1018D0008DF808105379116B0B440B205A788DF852
:1018E0000920DA7A8DF80A205B7D8DF80B3002A989
:1018F000F6F744FD0123226B84F82030637913440A
:101900000022DA7291E0B4EEE78AF1EE10FA48BFF5
:1019100083ED078AA16B636B94ED067AD4ED076AB9
:10192000591AC943C90F77EE667A59B9B7EE006AFA
:10193000F4EEC67AF1EE10FA79DDB4EEE68AF1EE55
:1019400010FA74DDD4ED056A454BB4EEE67AF1EE9B
:1019500010FACCBF0126002666B1D3ED097A9FEDBF
:10196000427A67EE877A9FED427AC3ED097AD3ED2A
:101970000B7A0AE0B0EE007AF4EEC77AF1EE10FAD4
:1019800008DDD3ED0B7A9FED387A67EE877AC3EDE9
:101990000B7A07E0D3ED097A9FED357A67EE877A07
:1019A000C3ED097AD4ED097A206B627967EEA87AE3
:1019B0001044FCEEE77ACDED017A9DF804304370D7
:1019C000D4ED0B7A2769FCEEE77A3F03CDED017A7F
:1019D0009DF8042042750ED546EA41018DF80810A5
:1019E0008DF80930C37A8DF80A300B2002A98DF8E2
:1019F0000B20F6F7C3FC94F82020194B022A11D1D2
:101A0000D3ED0A7A9FED1B7A196B67EE877A002275
:101A100083F82020FCEEE77A5A7917EE903A0A44D0
:101A2000D37202E0022283F82020F8F783FEA27925
:101A30000B4B0AB1104A00E0104ADA602544D4ED9D
:101A4000037AB5F9083000EE103AB8EEC00A80EE1D
:101A5000280A37EEC00A05B0BDEC028BF0BD00BF0E
:101A6000D42F0020BC980108EC51783F6F12833AC4
:101A70000AD7833F00007A440000A0410000A0C1C3
:101A80002B4BF0B52B4D1E6805F110002F78F31984
:101A90002C46597801F00401013501F0FF0219B11B
:101AA0008542F3D10020F0BD224D631B022B0ADDDD
:101AB0001AB102EB82025200D2B215F8013B303B60
:101AC0001A44D2B2F1E70021AC420AD919B101EBB4
:101AD00081014900C9B215F8013B303B1944C9B234
:101AE000F2E72E2F16D10134042000232578771930
:101AF00003EB83037F785B007F079BB244BF303DDD
:101B00005B1900F1FF3044BF01349BB210F0FF00BD
:101B1000ECD100E0002308484143642000FB03139C
:101B20000620B3FBF0F3054800FB0230F0BD00BF18
:101B3000900000201030002040420F008096980056
:101B400030B500231A4610498C1894F83C40BCB1BB
:101B50002E2C06D1013298B18C180444002584F84B
:101B60003C5011440A2491F83C106343A1F1300425
:101B7000092C9CBF303B5B180E2A03D80132E2E7E8
:101B8000184630BD002030BDD42F0020104B10B5BA
:101B90000446185CF9F783FC0E4800EB4400B0F9EA
:101BA0004C10B1F57A7F05DBB1F5FA6FA8BF4FF4A1
:101BB000FA6101E04FF47A71A1F57A710A230920E4
:101BC00091FBF3F1BDE81040C9B2FCF791B900BF39
:101BD00000B90108D42F0020031EB8BF2D2210B574
:101BE000B8BF58420C46B8BF01F8012B0A22F5F7DE
:101BF00019FD00230370204610BD00BF07B5064B3A
